:020000040800F2
:1000000000000820B91A0208FB0D0208030E0208BE
:100010000B0E0208130E02081B0E0208000000005F
:10002000000000000000000000000000E1DD010809
:10003000230E020800000000F1DF010859E001086A
:10004000311B0208311B0208311B0208311B020858
:10005000311B0208311B0208311B0208311B020848
:10006000311B0208311B0208311B0208311B020838
:10007000311B0208311B0208311B0208311B020828
:10008000311B0208311B0208311B0208311B020818
:10009000590E0208311B0208311B0208311B0208ED
:1000A000311B0208311B0208311B0208311B0208F8
:1000B000311B0208311B0208311B0208311B0208E8
:1000C000311B0208311B0208311B0208311B0208D8
:1000D000311B0208311B0208311B0208311B0208C8
:1000E000311B0208311B0208311B0208311B0208B8
:1000F000311B0208311B0208311B0208311B0208A8
:10010000311B0208311B0208311B0208311B020897
:10011000311B0208311B0208310E0208311B020894
:10012000311B0208311B0208311B0208311B020877
:10013000311B0208311B0208311B0208311B020867
:10014000311B0208311B0208311B0208450E020850
:10015000311B0208311B0208311B0208311B020847
:10016000311B0208311B0208311B0208311B020837
:10017000311B0208311B0208311B0208311B020827
:10018000311B0208311B0208311B0208311B020817
:10019000311B0208311B0208311B0208311B020807
:1001A000311B0208311B0208311B0208311B0208F7
:1001B000311B0208311B0208311B0208311B0208E7
:1001C000311B0208311B0208311B0208311B0208D7
:1001D000311B0208311B0208311B0208311B0208C7
:1001E000311B0208311B0208311B0208311B0208B7
:1001F000311B0208311B0208000000000000000053
:1002000000000000000000000000000000000000EE
:1002100000000000000000000000000000000000DE
:1002200000000000000000000000000000000000CE
:1002300000000000000000000000000000000000BE
:020000040801F1
:1000000081F0004102E000BF83F0004330B54FEAC9
:1000100041044FEA430594EA050F08BF90EA020F36
:100020001FBF54EA000C55EA020C7FEA645C7FEAC9
:10003000655C00F0E2804FEA5454D4EB5555B8BFEC
:100040006D420CDD2C4480EA020281EA030382EA5D
:10005000000083EA010180EA020281EA0303362DEF
:1000600088BF30BD11F0004F4FEA01314FF4801CC2
:100070004CEA113102D0404261EB410113F0004FD4
:100080004FEA03334CEA133302D0524263EB43038B
:1000900094EA050F00F0A780A4F10104D5F1200E29
:1000A0000DDB02FA0EFC22FA05F2801841F1000184
:1000B00003FA0EF2801843FA05F359410EE0A5F158
:1000C00020050EF1200E012A03FA0EFC28BF4CF089
:1000D000020C43FA05F3C01851EBE37101F000453F
:1000E00007D54FF0000EDCF1000C7EEB00006EEB4C
:1000F0000101B1F5801F1BD3B1F5001F0CD34908D6
:100100005FEA30004FEA3C0C04F101044FEA44522C
:1001100012F5800F80F09A80BCF1004F08BF5FEAB3
:10012000500C50F1000041EB045141EA050130BD93
:100130005FEA4C0C404141EB0101013C28BFB1F5A5
:10014000801FE9D291F0000F04BF01460020B1FAF0
:1001500081F308BF2033A3F10B03B3F120020CDAC3
:100160000C3208DD02F1140CC2F10C0201FA0CF0A1
:1001700021FA02F10CE002F11402D8BFC2F1200C06
:1001800001FA02F120FA0CFCDCBF41EA0C019040BC
:10019000E41AA2BF01EB0451294330BD6FEA040405
:1001A0001F3C1CDA0C340EDC04F11404C4F12002F0
:1001B00020FA04F001FA02F340EA030021FA04F302
:1001C00045EA030130BDC4F10C04C4F1200220FA59
:1001D00002F001FA04F340EA0300294630BD21FA97
:1001E00004F0294630BD94F0000F83F4801306BF5D
:1001F00081F480110134013D4EE77FEA645C18BF51
:100200007FEA655C29D094EA050F08BF90EA020FE7
:1002100005D054EA000C04BF1946104630BD91EADF
:10022000030F1EBF0021002030BD5FEA545C05D1E2
:100230004000494128BF41F0004130BD14F5800421
:100240003CBF01F5801130BD01F0004545F0FE4195
:1002500041F470014FF0000030BD7FEA645C1ABFCA
:10026000194610467FEA655C1CBF0B46024650EA01
:10027000013406BF52EA033591EA030F41F400212D
:1002800030BD00BF90F0000F04BF0021704730B5B3
:100290004FF4806404F132044FF000054FF0000188
:1002A00050E700BF90F0000F04BF0021704730B549
:1002B0004FF4806404F1320410F0004548BF40421E
:1002C0004FF000013EE700BF42004FEAE2014FEA73
:1002D00031014FEA02701FBF12F07F4393F07F4F4E
:1002E00081F06051704732F07F4208BF704793F051
:1002F0007F4F04BF41F40021704730B54FF4607464
:1003000001F0004521F000411CE700BF50EA010266
:1003100008BF704730B54FF000050AE050EA01020F
:1003200008BF704730B511F0004502D5404261EB7F
:1003300041014FF4806404F132045FEA915C3FF4C0
:10034000D8AE4FF003025FEADC0C18BF03325FEA5D
:10035000DC0C18BF033202EBDC02C2F1200300FA0E
:1003600003FC20FA02F001FA03FE40EA0E0021FA33
:1003700002F11444BDE600BF53B94AB9002908BFD1
:1003800000281CBF4FF0FF314FF0FF3000F00CB8D9
:10039000ADF1080C6DE904CE22F07EFFDDF804E03B
:1003A000DDE9022304B07047704700BF10F8012B4D
:1003B00011F8013B012A28BF9A42F7D0D01A7047A2
:1003C00001F0FF01102A2BDB10F0070F08D010F806
:1003D000013B013A8B422DD010F0070F42B3F6D10A
:1003E000F0B441EA012141EA014122F007047FF023
:1003F00000070023F0E80256083C85EA010586EA7A
:10040000010685FA47F5A3FA87F586FA47F6A5FAB5
:1004100087F68EB9EED1F0BC01F0FF0102F00702C1
:1004200032B110F8013B013A83EA010313B1F8D16C
:100430000020704701387047002D06BF354603384D
:10044000073815F0010F07D1013015F4807F02BF86
:10045000013015F4C03F0130F0BC0138704700BFD7
:10046000034613F8012B002AFBD1181A01387047F4
:100470000348044B834202D0034B03B11847704733
:100480007403002074030020000000000548064BA0
:100490001B1AD90F01EBA301491002D0034B03B182
:1004A0001847704774030020740300200000000008
:1004B00010B5064C237843B9FFF7DAFF044B13B1AC
:1004C0000448AFF300800123237010BD780300209F
:1004D000000000000485030808B5054B1BB1054961
:1004E0000548AFF30080BDE80840FFF7CFBF00BF6D
:1004F000000000007C0300200485030880B400AFE6
:10050000064BD3F88830054A43F47003C2F88830AC
:1005100000BFBD465DF8047B704700BF00ED00E002
:1005200080B582B000AF78607B68002B01D10123D9
:1005300049E07B6893F83D30DBB2002B06D17B6845
:10054000002283F83C20786810F032FF7B6802229A
:1005500083F83D207B681A687B680433194610468F
:1005600001F07AF97B68012283F848207B68012238
:1005700083F83E207B68012283F83F207B680122BC
:1005800083F840207B68012283F841207B680122A8
:1005900083F842207B68012283F843207B68012294
:1005A00083F844207B68012283F845207B68012280
:1005B00083F846207B68012283F847207B6801226C
:1005C00083F83D20002318460837BD4680BD000053
:1005D00080B485B000AF78607B6893F83D30DBB2C3
:1005E000012B01D0012354E07B68022283F83D20D7
:1005F0007B681B68DA687B681B6842F00102DA607E
:100600007B681B68264A934222D07B681B68B3F143
:10061000804F1DD07B681B68224A934218D07B68AC
:100620001B68214A934213D07B681B681F4A934280
:100630000ED07B681B681E4A934209D07B681B68FA
:100640001C4A934204D07B681B681B4A934215D115
:100650007B681B689A68194B1340FB60FB68062B8C
:1006600015D0FB68B3F5803F11D07B681B681A6812
:100670007B681B6842F001021A6008E07B681B6817
:100680001A687B681B6842F001021A6000E000BF34
:10069000002318461437BD465DF8047B704700BF41
:1006A000000001400004004000080040000C004031
:1006B0000004014000400140001800400700010014
:1006C00080B582B000AF78607B68002B01D1012338
:1006D00049E07B6893F83D30DBB2002B06D17B68A4
:1006E000002283F83C20786810F02EFE7B680222FE
:1006F00083F83D207B681A687B68043319461046EE
:1007000001F0AAF87B68012283F848207B68012267
:1007100083F83E207B68012283F83F207B6801221A
:1007200083F840207B68012283F841207B68012206
:1007300083F842207B68012283F843207B680122F2
:1007400083F844207B68012283F845207B680122DE
:1007500083F846207B68012283F847207B680122CA
:1007600083F83D20002318460837BD4680BD0000B1
:1007700080B584B000AF786039603B68002B09D148
:100780007B6893F83E30DBB2012B14BF01230023BA
:10079000DBB23CE03B68042B09D17B6893F83F3027
:1007A000DBB2012B14BF01230023DBB22FE03B6837
:1007B000082B09D17B6893F84030DBB2012B14BFC2
:1007C00001230023DBB222E03B680C2B09D17B68BC
:1007D00093F84130DBB2012B14BF01230023DBB2BD
:1007E00015E03B68102B09D17B6893F84230DBB2EF
:1007F000012B14BF01230023DBB208E07B6893F8D0
:100800004330DBB2012B14BF01230023DBB2002BEA
:1008100001D0012392E03B68002B04D17B680222C7
:1008200083F83E2023E03B68042B04D17B6802223E
:1008300083F83F201BE03B68082B04D17B68022231
:1008400083F8402013E03B680C2B04D17B68022224
:1008500083F841200BE03B68102B04D17B68022217
:1008600083F8422003E07B68022283F843207B6800
:100870001B6801223968184601F02FFD7B681B6850
:10088000304A934204D07B681B682F4A934201D1BF
:10089000012300E00023002B07D07B681B685A6C03
:1008A0007B681B6842F400425A647B681B68254AD7
:1008B000934222D07B681B68B3F1804F1DD07B68C8
:1008C0001B68224A934218D07B681B68204A9342D7
:1008D00013D07B681B681F4A93420ED07B681B684D
:1008E000194A934209D07B681B681B4A934204D083
:1008F0007B681B68194A934215D17B681B689A680C
:10090000174B1340FB60FB68062B15D0FB68B3F553
:10091000803F11D07B681B681A687B681B6842F0B7
:1009200001021A6008E07B681B681A687B681B6814
:1009300042F001021A6000E000BF002318461037A1
:10094000BD4680BD0000014000040140000400409D
:1009500000080040000C004000400140001800402A
:100960000700010080B582B000AF78607B68002B83
:1009700001D1012349E07B6893F83D30DBB2002BC5
:1009800006D17B68002283F83C20786810F044FD93
:100990007B68022283F83D207B681A687B680433F9
:1009A0001946104600F058FF7B68012283F8482062
:1009B0007B68012283F83E207B68012283F83F2078
:1009C0007B68012283F840207B68012283F8412064
:1009D0007B68012283F842207B68012283F8432050
:1009E0007B68012283F844207B68012283F845203C
:1009F0007B68012283F846207B68012283F8472028
:100A00007B68012283F83D20002318460837BD4645
:100A100080BD000080B582B000AF78607B680222A4
:100A200083F83D207B681B681A6A284B1340002B13
:100A30000FD17B681B681A6A40F244431340002BB5
:100A400007D17B681B681A687B681B6822F001026B
:100A50001A60786800F03CF87B68002283F8482030
:100A60007B68002283F83E207B68002283F83F20C9
:100A70007B68002283F840207B68002283F84120B5
:100A80007B68002283F842207B68002283F84320A1
:100A90007B68002283F844207B68002283F845208D
:100AA0007B68002283F846207B68002283F8472079
:100AB0007B68002283F83D207B68002283F83C207D
:100AC000002318460837BD4680BD00BF1111110034
:100AD00080B483B000AF786000BF0C37BD465DF8CE
:100AE000047B704780B584B000AF786039603B68A4
:100AF000002B04D17B6893F83E30DBB223E03B68E7
:100B0000042B04D17B6893F83F30DBB21BE03B68D9
:100B1000082B04D17B6893F84030DBB213E03B68CC
:100B20000C2B04D17B6893F84130DBB20BE03B68BF
:100B3000102B04D17B6893F84230DBB203E07B6872
:100B400093F84330DBB2FB733B68002B04D17B6826
:100B500093F84430DBB213E03B68042B04D17B688C
:100B600093F84530DBB20BE03B68082B04D17B687F
:100B700093F84630DBB203E07B6893F84730DBB292
:100B8000BB73FB7B012B02D1BB7B012B01D001236B
:100B900097E03B68002B04D17B68022283F83E205B
:100BA00023E03B68042B04D17B68022283F83F20BA
:100BB0001BE03B68082B04D17B68022283F84020AD
:100BC00013E03B680C2B04D17B68022283F84120A0
:100BD0000BE03B68102B04D17B68022283F8422093
:100BE00003E07B68022283F843203B68002B04D19A
:100BF0007B68022283F8442013E03B68042B04D175
:100C00007B68022283F845200BE03B68082B04D167
:100C10007B68022283F8462003E07B68022283F887
:100C200047207B681B6801223968184601F055FB94
:100C30007B681B68254A934222D07B681B68B3F10E
:100C4000804F1DD07B681B68214A934218D07B6877
:100C50001B68204A934213D07B681B681E4A93424C
:100C60000ED07B681B681D4A934209D07B681B68C5
:100C70001B4A934204D07B681B681A4A934215D1E1
:100C80007B681B689A68184B1340BB60BB68062BD7
:100C900015D0BB68B3F5803F11D07B681B681A681C
:100CA0007B681B6842F001021A6008E07B681B68E1
:100CB0001A687B681B6842F001021A6000E000BFFE
:100CC000002318461037BD4680BD00BF000001401C
:100CD0000004004000080040000C004000040140F7
:100CE00000400140001800400700010080B582B0BC
:100CF00000AF786039607B681B680022396818464D
:100D000001F0EBFA7B681B681A6A304B1340002B2A
:100D10000FD17B681B681A6A40F244431340002BD2
:100D200007D17B681B681A687B681B6822F0010288
:100D30001A603B68002B04D17B68012283F83E20B7
:100D400023E03B68042B04D17B68012283F83F2019
:100D50001BE03B68082B04D17B68012283F840200C
:100D600013E03B680C2B04D17B68012283F84120FF
:100D70000BE03B68102B04D17B68012283F84220F2
:100D800003E07B68012283F843203B68002B04D1F9
:100D90007B68012283F8442013E03B68042B04D1D4
:100DA0007B68012283F845200BE03B68082B04D1C7
:100DB0007B68012283F8462003E07B68012283F8E8
:100DC0004720002318460837BD4680BD1111110089
:100DD00080B586B000AF786039607B68002B01D1A8
:100DE00001238FE07B6893F83D30DBB2002B06D106
:100DF0007B68002283F83C20786810F093F97B68C8
:100E0000022283F83D207B681B6899687B681A681A
:100E10003E4B0B4093607B681A687B68043319462D
:100E2000104600F019FD7B681B689B687B617B683E
:100E30001B689B693B617B681B681B6AFB603B68A6
:100E40001B687A6913437B613A69314B13403B61FC
:100E50003B689A683B689B691B0213433A691343DA
:100E60003B613A692B4B13403B613A692A4B134073
:100E70003B613B68DA683B68DB691B0213433A69F4
:100E800013433B613B681B691A013B681B6A1B03E8
:100E900013433A6913433B61FB6823F02203FB6071
:100EA000FB6823F08803FB603B685A683B685B691A
:100EB0001B011343FA681343FB607B681B687A6964
:100EC0009A607B681B683A699A617B681B68FA685C
:100ED0001A627B68012283F848207B68012283F82C
:100EE0003E207B68012283F83F207B68012283F843
:100EF00044207B68012283F845207B68012283F827
:100F00003D20002318461837BD4680BDF8BFFEFFC0
:100F1000FCFCFFFFF3F3FFFF0F0FFFFF80B582B074
:100F200000AF78607B68022283F83D207B681B68F5
:100F30001A6A1C4B1340002B0FD17B681B681A6A7E
:100F400040F244431340002B07D17B681B681A68AA
:100F50007B681B6822F001021A60786810F00AFCB6
:100F60007B68002283F848207B68002283F83E20BB
:100F70007B68002283F83F207B68002283F84420AE
:100F80007B68002283F845207B68002283F83D209F
:100F90007B68002283F83C20002318460837BD46B2
:100FA00080BD00BF1111110080B584B000AF786022
:100FB00039607B6893F83E30FB737B6893F83F3071
:100FC000BB737B6893F844307B737B6893F8453040
:100FD0003B733B68002B10D1FB7B012B02D17B7B49
:100FE000012B01D0012369E07B68022283F83E20B7
:100FF0007B68022283F8442031E03B68042B10D147
:10100000BB7B012B02D13B7B012B01D0012355E09F
:101010007B68022283F83F207B68022283F8452008
:101020001DE0FB7B012B08D1BB7B012B05D17B7B1A
:10103000012B02D13B7B012B01D001233EE07B68D9
:10104000022283F83E207B68022283F83F207B68DF
:10105000022283F844207B68022283F845203B6803
:10106000002B03D03B68042B08D00FE07B681B6883
:1010700001220021184601F030F916E07B681B6858
:1010800001220421184601F028F90EE07B681B6854
:1010900001220021184601F020F97B681B6801221B
:1010A0000421184601F019F900BF7B681B681A6813
:1010B0007B681B6842F001021A6000231846103753
:1010C000BD4680BD80B582B000AF786039603B68B6
:1010D000002B03D03B68042B08D00FE07B681B6813
:1010E00000220021184601F0F8F816E07B681B6822
:1010F00000220421184601F0F0F80EE07B681B681E
:1011000000220021184601F0E8F87B681B680022E5
:101110000421184601F0E1F800BF7B681B681A6AD9
:101120003B4B1340002B0FD17B681B681A6A40F2BF
:1011300044431340002B07D17B681B681A687B6807
:101140001B6822F001021A603B68002B02D03B684A
:10115000042B48D13B68002B04D17B68012283F823
:101160003E2023E03B68042B04D17B68012283F8F6
:101170003F201BE03B68082B04D17B68012283F8E9
:10118000402013E03B680C2B04D17B68012283F8DC
:1011900041200BE03B68102B04D17B68012283F8CF
:1011A000422003E07B68012283F843203B68002B48
:1011B00004D17B68012283F8442024E03B68042B9F
:1011C00004D17B68012283F845201CE03B68082B92
:1011D00004D17B68012283F8462014E07B68012259
:1011E00083F847200FE07B68012283F83E207B686C
:1011F000012283F83F207B68012283F844207B682A
:10120000012283F84520002318460837BD4680BDDB
:101210001111110080B584B000AF78607B681B6845
:10122000DB68FB607B681B681B69BB60BB6803F005
:101230000203002B20D0FB6803F00203002B1BD01D
:101240007B681B686FF002021A617B6801221A77C3
:101250007B681B689B6903F00303002B03D078684D
:1012600000F0DCFA05E0786800F0CEFA786800F06B
:10127000DFFA7B6800221A77BB6803F00403002BB7
:1012800020D0FB6803F00403002B1BD07B681B6895
:101290006FF004021A617B6802221A777B681B6870
:1012A0009B6903F44073002B03D0786800F0B6FA12
:1012B00005E0786800F0A8FA786800F0B9FA7B6871
:1012C00000221A77BB6803F00803002B20D0FB68CC
:1012D00003F00803002B1BD07B681B686FF008022B
:1012E0001A617B6804221A777B681B68DB6903F04C
:1012F0000303002B03D0786800F090FA05E07868CB
:1013000000F082FA786800F093FA7B6800221A777E
:10131000BB6803F01003002B20D0FB6803F0100320
:10132000002B1BD07B681B686FF010021A617B6872
:1013300008221A777B681B68DB6903F44073002B73
:1013400003D0786800F06AFA05E0786800F05CFA8B
:10135000786800F06DFA7B6800221A77BB6803F0AA
:101360000103002B0CD0FB6803F00103002B07D016
:101370007B681B686FF001021A6178680EF048FF05
:10138000BB6803F08003002B04D1BB6803F4005357
:10139000002B0CD0FB6803F08003002B07D07B6888
:1013A0001B686FF402521A61786801F053F8BB6849
:1013B00003F48073002B0CD0FB6803F08003002B38
:1013C00007D07B681B686FF480721A61786801F03F
:1013D0004BF8BB6803F04003002B0CD0FB6803F014
:1013E0004003002B07D07B681B686FF040021A6136
:1013F000786800F027FABB6803F02003002B0CD0BC
:10140000FB6803F02003002B07D07B681B686FF09C
:1014100020021A61786801F013F800BF1037BD464A
:1014200080BD80B586B000AFF860B9607A600023F7
:10143000FB75FB6893F83C30012B01D1022388E057
:10144000FB68012283F83C207B68002B1BD1FB68E2
:101450001868BB681968BB685A68BB68DB6800F02D
:1014600093FDFB681B689A69FB681B6822F00C02FD
:101470009A61FB681B689969BB689A68FB681B687E
:101480000A439A6160E07B68042B1CD1FB681868F2
:10149000BB681968BB685A68BB68DB6800F017FE58
:1014A000FB681B689A69FB681B6822F440629A61BA
:1014B000FB681B689969BB689B681A02FB681B681C
:1014C0000A439A6140E07B68082B1BD1FB681868CF
:1014D000BB681968BB685A68BB68DB6800F064FECB
:1014E000FB681B68DA69FB681B6822F00C02DA6192
:1014F000FB681B68D969BB689A68FB681B680A436C
:10150000DA6121E07B680C2B1CD1FB681868BB6892
:101510001968BB685A68BB68DB6800F081FEFB682D
:101520001B68DA69FB681B6822F44062DA61FB68B9
:101530001B68D969BB689B681A02FB681B680A4371
:10154000DA6101E00123FB75FB68002283F83C208F
:10155000FB7D18461837BD4680BD000080B586B0BB
:1015600000AFF860B9607A600023FB75FB6893F800
:101570003C30012B01D10223FFE0FB68012283F8FC
:101580003C207B68142B00F2F08001A252F823F07B
:10159000E51501086B1701086B1701086B170108A7
:1015A000251601086B1701086B1701086B17010856
:1015B000671601086B1701086B1701086B17010804
:1015C000A71601086B1701086B1701086B170108B4
:1015D000E91601086B1701086B1701086B17010862
:1015E00029170108FB681B68B968184600F0DAF98A
:1015F000FB681B689A69FB681B6842F008029A61E5
:10160000FB681B689A69FB681B6822F004029A61F8
:10161000FB681B689969BB681A69FB681B680A4309
:101620009A61A5E0FB681B68B968184600F02CFABF
:10163000FB681B689A69FB681B6842F400629A6148
:10164000FB681B689A69FB681B6822F480629A61D8
:10165000FB681B689969BB681B691A02FB681B68F9
:101660000A439A6184E0FB681B68B968184600F079
:1016700083FAFB681B68DA69FB681B6842F00802A2
:10168000DA61FB681B68DA69FB681B6822F00402F8
:10169000DA61FB681B68D969BB681A69FB681B685B
:1016A0000A43DA6164E0FB681B68B968184600F019
:1016B000D9FAFB681B68DA69FB681B6842F40062B0
:1016C000DA61FB681B68DA69FB681B6822F48062D8
:1016D000DA61FB681B68D969BB681B691A02FB6881
:1016E0001B680A43DA6143E0FB681B68B968184667
:1016F00000F010FBFB681B685A6DFB681B6842F02A
:1017000008025A65FB681B685A6DFB681B6822F06B
:1017100004025A65FB681B68596DBB681A69FB684F
:101720001B680A435A6523E0FB681B68B9681846C2
:1017300000F042FBFB681B685A6DFB681B6842F4B3
:1017400000625A65FB681B685A6DFB681B6822F4CF
:1017500080625A65FB681B68596DBB681B691A0279
:10176000FB681B680A435A6502E00123FB7500BF52
:10177000FB68002283F83C20FB7D18461837BD46E5
:1017800080BD00BF80B582B000AF786039607B68F3
:1017900093F83C30012B01D1022331E07B68012218
:1017A00083F83C207B68022283F83D203968786802
:1017B00000F056FB0346002B09D07B68012283F81A
:1017C0003D207B68002283F83C20012318E07B68E1
:1017D0001B68DA687B681B6822F04002DA607B686D
:1017E0001B68DA687B681B6822F48042DA607B68D9
:1017F000012283F83D207B68002283F83C200023EF
:1018000018460837BD4680BD80B483B000AF78600D
:1018100000BF0C37BD465DF8047B704780B483B0D1
:1018200000AF786000BF0C37BD465DF8047B7047A1
:1018300080B483B000AF786000BF0C37BD465DF860
:10184000047B704780B483B000AF786000BF0C3772
:10185000BD465DF8047B704780B485B000AF78600A
:1018600039607B681B68FB607B68434A934213D0F6
:101870007B68B3F1804F0FD07B68404A93420BD016
:101880007B683F4A934207D07B683E4A934203D02D
:101890007B683D4A934208D1FB6823F07003FB60EC
:1018A0003B685B68FA681343FB607B68324A93428B
:1018B0002BD07B68B3F1804F27D07B682F4A9342AF
:1018C00023D07B682E4A93421FD07B682D4A9342D7
:1018D0001BD07B682C4A934217D07B682B4A9342DB
:1018E00013D07B682A4A93420FD07B68294A9342DF
:1018F0000BD07B68284A934207D07B68274A9342E3
:1019000003D07B68264A934208D1FB6823F44073D6
:10191000FB603B68DB68FA681343FB60FB6823F0FD
:1019200080023B685B691343FB603B689A687B6895
:10193000DA623B681A687B689A627B680E4A934257
:1019400003D07B68104A934203D13B681A697B68D5
:101950001A637B681B6843F004027B681A607B682B
:1019600001225A617B68FA681A6000BF1437BD46CD
:101970005DF8047B704700BF000001400004004098
:1019800000080040000C00400004014000400140FD
:10199000004401400048014000180040001C004085
:1019A0000020004080B487B000AF786039607B6869
:1019B0001B6A7B617B681B6A23F001027B681A62E9
:1019C0007B685B683B617B689B69FB60FA682B4BBB
:1019D0001340FB60FB6823F00303FB603B681B685C
:1019E000FA681343FB607B6923F002037B613B6869
:1019F0009B687A6913437B617B68214A934203D0D9
:101A00007B68204A93420CD17B6923F008037B61F9
:101A10003B68DB687A6913437B617B6923F00403CD
:101A20007B617B68164A934203D07B68154A9342D8
:101A300011D13B6923F480733B613B6923F400734C
:101A40003B613B685B693A6913433B613B689B6957
:101A50003A6913433B617B683A695A607B68FA686C
:101A60009A613B685A687B685A637B687A691A6234
:101A700000BF1C37BD465DF8047B70478FFFFEFF3B
:101A8000000001400004014080B487B000AF7860DE
:101A900039607B681B6A7B617B681B6A23F01002DC
:101AA0007B681A627B685B683B617B689B69FB6053
:101AB000FA682E4B1340FB60FB6823F44073FB6015
:101AC0003B681B681B02FA681343FB607B6923F0C9
:101AD00020037B613B689B681B017A6913437B6130
:101AE0007B68234A934203D07B68224A93420DD1FC
:101AF0007B6923F080037B613B68DB681B017A69AB
:101B000013437B617B6923F040037B617B68184A48
:101B1000934203D07B68174A934213D13B6923F465
:101B200080633B613B6923F400633B613B685B6915
:101B30009B003A6913433B613B689B699B003A6990
:101B400013433B617B683A695A607B68FA689A6123
:101B50003B685A687B689A637B687A691A6200BF3F
:101B60001C37BD465DF8047B704700BFFF8FFFFE4A
:101B7000000001400004014080B487B000AF7860ED
:101B800039607B681B6A7B617B681B6A23F4807207
:101B90007B681A627B685B683B617B68DB69FB6022
:101BA000FA682D4B1340FB60FB6823F00303FB60D6
:101BB0003B681B68FA681343FB607B6923F400737E
:101BC0007B613B689B681B027A6913437B617B687E
:101BD000224A934203D07B68214A93420DD17B690C
:101BE00023F400637B613B68DB681B027A69134363
:101BF0007B617B6923F480637B617B68174A934236
:101C000003D07B68164A934213D13B6923F4805377
:101C10003B613B6923F400533B613B685B691B01FB
:101C20003A6913433B613B689B691B013A69134363
:101C30003B617B683A695A607B68FA68DA613B68A5
:101C40005A687B68DA637B687A691A6200BF1C375E
:101C5000BD465DF8047B70478FFFFEFF000001402A
:101C60000004014080B487B000AF786039607B68C1
:101C70001B6A3B617B681B6A23F480527B681A6293
:101C80007B685B687B617B68DB69FB60FA681E4B85
:101C90001340FB60FB6823F44073FB603B681B68E8
:101CA0001B02FA681343FB603B6923F400533B615A
:101CB0003B689B681B033A6913433B617B68134A8B
:101CC000934203D07B68124A934209D17B6923F483
:101CD00080437B613B685B699B017A6913437B614D
:101CE0007B687A695A607B68FA68DA613B685A688F
:101CF0007B681A647B683A691A6200BF1C37BD466C
:101D00005DF8047B704700BFFF8FFFFE00000140BD
:101D10000004014080B487B000AF786039607B6810
:101D20001B6A3B617B681B6A23F480327B681A6202
:101D30007B685B687B617B685B6DFB60FA681B4B53
:101D40001340FB603B681B68FA681343FB603B6908
:101D500023F400333B613B689B681B043A691343DF
:101D60003B617B68124A934203D07B68114A9342DD
:101D700009D17B6923F480337B613B685B691B027B
:101D80007A6913437B617B687A695A607B68FA6879
:101D90005A653B685A687B689A657B683A691A623B
:101DA00000BF1C37BD465DF8047B70478FFFFEFF08
:101DB000000001400004014080B487B000AF7860AB
:101DC00039607B681B6A3B617B681B6A23F4801265
:101DD0007B681A627B685B687B617B685B6DFB601C
:101DE000FA681C4B1340FB603B681B681B02FA68D7
:101DF0001343FB603B6923F400133B613B689B6822
:101E00001B053A6913433B617B68134A934203D035
:101E10007B68124A934209D17B6923F480237B615A
:101E20003B685B699B027A6913437B617B687A69D3
:101E30005A607B68FA685A653B685A687B68DA655D
:101E40007B683A691A6200BF1C37BD465DF8047BA7
:101E5000704700BFFF8FFFFE0000014000040140FB
:101E600080B586B000AF786039600023FB757B6871
:101E70001B689B683B613B6923F070033B613B68D7
:101E80005B683A6913433B613A693E4B13403B61DF
:101E90003B681B683A6913433B617B681B683A697E
:101EA0009A603B685B68702B1AD0702B60D8602BEF
:101EB00054D0602B5CD8502B46D0502B58D8402B98
:101EC00019D0402B54D8302B55D0302B50D8202B44
:101ED00051D0202B4CD8002B4DD0102B4BD047E0AD
:101EE0007B6818683B68D9683B689A683B681B69DF
:101EF00000F0D3F940E03B681B68052B01D10123BA
:101F00003BE07B681B681B6AFB607B681B681A6A86
:101F10007B681B6822F001021A627B681B689B6960
:101F2000BB60BB6823F0F003BB603B681B691B010F
:101F3000BA681343BB607B681B68BA689A617B68A8
:101F40001B68FA681A6217E07B6818683B68996832
:101F50003B681B691A4600F08BF80DE07B68186837
:101F60003B6899683B681B691A4600F0EDF803E08E
:101F70000123FB7500E000BFFB7D18461837BD4606
:101F800080BD00BFF8FFFEFF80B487B000AFF860EF
:101F9000B9607A603B60FB681B6A3B61FB681B6A47
:101FA00023F00102FB681A62FB689B697B61FB6896
:101FB000284A93421BD0FB68B3F1804F17D0FB68CF
:101FC000254A934213D0FB68244A93420FD0FB6802
:101FD000234A93420BD0FB68224A934207D0FB6806
:101FE000214A934203D0FB68204A934201D1012346
:101FF00000E00023002B08D07B6923F003037B6102
:102000007A697B6813437B6103E07B6943F00103DA
:102010007B617B6923F0F0037B613B681B01DBB2D2
:102020007A6913437B613B6923F00A033B61BB6818
:1020300003F00A033A6913433B61FB687A699A61CA
:10204000FB683A691A6200BF1C37BD465DF8047B25
:10205000704700BF0000014000040040000800403D
:10206000000C004000040140004001400018004006
:1020700080B487B000AFF860B9607A60FB681B6A13
:102080007B61FB681B6A23F00102FB681A62FB6834
:102090009B693B613B6923F0F0033B617B681B015B
:1020A0003A6913433B617B6923F00A037B617A69D8
:1020B000BB6813437B61FB683A699A61FB687A6984
:1020C0001A6200BF1C37BD465DF8047B704780B4C0
:1020D00087B000AFF860B9607A603B60FB681B6A4C
:1020E0007B61FB681B6A23F01002FB681A62FB68C5
:1020F0009B693B613B6923F440733B617B681B0236
:102100003A6913433B613B6923F470433B613B688D
:102110001B039BB23A6913433B617B6923F0A00325
:102120007B61BB681B0103F0A0037A6913437B61E9
:10213000FB683A699A61FB687A691A6200BF1C37CA
:10214000BD465DF8047B704780B487B000AFF8608F
:10215000B9607A60FB681B6A7B61FB681B6A23F0CD
:102160001002FB681A62FB689B693B613B6923F4C0
:1021700070433B617B681B033A6913433B617B6996
:1021800023F0A0037B61BB681B017A6913437B6169
:10219000FB683A699A61FB687A691A6200BF1C376A
:1021A000BD465DF8047B704780B487B000AFF8602F
:1021B000B9607A603B60FB681B6A7B61FB681B6AE5
:1021C00023F48072FB681A62FB68DB693B613B6940
:1021D00023F003033B613A697B6813433B613B692E
:1021E00023F0F0033B613B681B01DBB23A69134308
:1021F0003B617B6923F420637B61BB681B0203F4B2
:1022000020637A6913437B61FB683A69DA61FB6892
:102210007A691A6200BF1C37BD465DF8047B7047BF
:1022200080B487B000AFF860B9607A603B60FB684B
:102230001B6A7B61FB681B6A23F48052FB681A628D
:10224000FB68DB693B613B6923F440733B617B685E
:102250001B023A6913433B613B6923F470433B61C2
:102260003B681B039BB23A6913433B617B6923F4D0
:1022700020437B61BB681B0303F420437A6913434B
:102280007B61FB683A69DA61FB687A691A6200BFB0
:102290001C37BD465DF8047B704780B487B000AF43
:1022A000F860B9607A603B60FB689B687B617B6922
:1022B00023F47F437B613B681A027B681A43BB6847
:1022C00013437A6913437B61FB687A699A6000BFA4
:1022D0001C37BD465DF8047B704780B487B000AF03
:1022E000F860B9607A60BB6803F01F03012202FA4C
:1022F00003F37B61FB681A6A7B69DB431A40FB6866
:102300001A62FB681A6ABB6803F01F03796801FA56
:1023100003F31A43FB681A6200BF1C37BD465DF821
:10232000047B704780B485B000AF786039607B680B
:1023300093F83C30012B01D102236DE07B68012230
:1023400083F83C207B68022283F83D207B681B6871
:102350005B68FB607B681B689B68BB607B681B6875
:10236000304A934204D07B681B682F4A934208D1BD
:10237000FB6823F47003FB603B685B68FA681343F7
:10238000FB60FB6823F07003FB603B681B68FA6826
:102390001343FB607B681B68FA685A607B681B68A4
:1023A000204A934222D07B681B68B3F1804F1DD036
:1023B0007B681B681D4A934218D07B681B681C4AC7
:1023C000934213D07B681B681A4A93420ED07B68F5
:1023D0001B68154A934209D07B681B68164A9342D2
:1023E00004D07B681B68154A93420CD1BB6823F06C
:1023F0008003BB603B689B68BA681343BB607B6823
:102400001B68BA689A607B68012283F83D207B686C
:10241000002283F83C20002318461437BD465DF89F
:10242000047B7047000001400004014000040040AC
:1024300000080040000C004000400140001800402F
:1024400080B483B000AF786000BF0C37BD465DF844
:10245000047B704780B483B000AF786000BF0C3756
:10246000BD465DF8047B704780B483B000AF7860F0
:1024700000BF0C37BD465DF8047B704780B586B061
:1024800002AF78607B68002B01D1012308E17B68F3
:102490001B68BB607B6893F89534DBB2002B06D1D8
:1024A0007B68002283F8942478680BF06DFE7B68CB
:1024B000032283F89524BB68B3F1A04F02D17B6857
:1024C00000229A717B681B68184601F070FB7B68DC
:1024D00018687B681A7C8DF8002004330ECB01F05D
:1024E00059FA0346002B05D07B68022283F8952415
:1024F0000123D5E07B681B680021184601F068FBCA
:102500000346002B05D07B68022283F89524012323
:10251000C6E00023FB734AE0FA7B79681346DB00D0
:1025200013449B000B44153301221A70FA7B79681F
:102530001346DB0013449B000B441433FA7B1A70E0
:10254000FA7BFB7B98B279681346DB0013449B004F
:102550000B442E3302461A80FA7B79681346DB005F
:1025600013449B000B44183300221A70FA7B7968DD
:102570001346DB0013449B000B441C3300221A60FB
:10258000FA7B79681346DB0013449B000B4420332D
:1025900000221A60FA7B79681346DB0013449B0023
:1025A0000B44243300221A60FB7B0133FB737B68EE
:1025B0001B79FA7B9A42AFD30023FB7344E0FA7B8A
:1025C00079681346DB0013449B000B4403F2552348
:1025D00000221A70FA7B79681346DB0013449B00D3
:1025E0000B4403F51573FA7B1A70FA7B796813466E
:1025F000DB0013449B000B4403F5167300221A7092
:10260000FA7B79681346DB0013449B000B4403F507
:10261000177300221A60FA7B79681346DB001344B3
:102620009B000B4403F5187300221A60FA7B79684B
:102630001346DB0013449B000B4403F5197300227F
:102640001A60FB7B0133FB737B681B79FA7B9A4230
:10265000B5D37B6818687B681A7C8DF8002004333A
:102660000ECB01F001FB0346002B05D07B68022254
:1026700083F89524012313E07B6800225A747B6859
:10268000012283F895247B681B7B012B02D178689B
:1026900001F05CF97B681B68184602F044FB0023DC
:1026A00018461037BD4680BD80B582B000AF786057
:1026B0007B6893F89434012B01D1022312E07B68EC
:1026C000012283F894247B681B68184601F05EFAA7
:1026D0007B681B68184602F005FB7B68002283F8C4
:1026E0009424002318460837BD4680BD90B58DB0B0
:1026F00000AF78607B681B683B623B6AFB617B686C
:102700001B68184602F0C3FB0346002B40F0B98457
:102710007B681B68184602F027FB0346002B00F07D
:10272000AF84FB6903F500639B681B0AC3F30D02CA
:102730007B68C3F8D4247B681B68184602F014FB3E
:10274000034603F00203022B07D17B681B685A691A
:102750007B681B6802F002025A617B681B6818469E
:1027600002F002FB034603F01003102B61D17B68DB
:102770001B689A697B681B6822F010029A613B6AA9
:102780001B6ABB61BB6903F00F021346DB001344F5
:102790009B0003F514737A68134404337B61BB69AF
:1027A00003F4F013B3F5802F24D1BA6947F6F07320
:1027B0001340002B35D07B69D968BB691B099BB2DC
:1027C000C3F30A039BB21A46386A02F039F97B69EF
:1027D000DA68BB691B09C3F30A031A447B69DA6030
:1027E0007B695A69BB691B09C3F30A031A447B69F5
:1027F0005A6116E0BB6903F4F013B3F5402F10D112
:102800007B6803F29C4308221946386A02F018F9E3
:102810007B695A69BB691B09C3F30A031A447B69C4
:102820005A617B681B689A697B681B6842F01002DA
:102830009A617B681B68184602F096FA034603F417
:102840000023B3F5002F40F0A78000237B627B6854
:102850001B68184602F09BFAB86299E0BB6A03F065
:102860000103002B00F08E807B681B687A6AD2B26D
:102870001146184602F0BFFA38613B6903F00103C4
:10288000002B0CD07B6A5A01FB69134403F53063BB
:102890001A4601239360796A786800F0D1FE3B699B
:1028A00003F00803002B0CD07B6A5A01FB69134428
:1028B00003F530631A4608239360796A786800F05C
:1028C000A7FF3B6903F01003002B08D07B6A5A0175
:1028D000FB69134403F530631A46102393603B6988
:1028E00003F00203002B30D03B6A5B6903F08003E6
:1028F000802B09D1FB6903F500635B68FA6902F577
:10290000006243F4806353607A6A1346DB00134429
:102910009B0003F514737A68134404337B617B696D
:10292000DB78012B08D17B690022DA707B6ADBB28D
:10293000194678680BF04CFD7B6A5A01FB69134419
:1029400003F530631A46022393603B6903F02003CA
:10295000002B08D07B6A5A01FB69134403F53063EE
:102960001A46202393603B6903F40053002B09D0DF
:102970007B6A5A01FB69134403F530631A464FF42E
:10298000005393607B6A01337B62BB6A5B08BB6266
:10299000BB6A002B7FF462AF7B681B68184602F0AD
:1029A000E3F9034603F48023B3F5802F40F0DB8086
:1029B0007B681B68184602F004FAB86200237B6249
:1029C000CDE0BB6A03F00103002B00F0C2807B68FE
:1029D0001B687A6AD2B21146184602F02AFA3861A8
:1029E0003B6903F00103002B57D07B6A03F00F0310
:1029F000012202FA03F3FB60FB6903F500635A6BE3
:102A0000FB68DB43F96901F5006113404B637B6AA6
:102A10005A01FB69134403F510631A4601239360BE
:102A20007B689B79012B32D179687A6A1346DB0087
:102A300013449B000B442033196878687A6A134664
:102A4000DB0013449B0003441C331B681944786863
:102A50007A6A1346DB0013449B0003442033196059
:102A60007B6A002B13D179687A6A1346DB00134422
:102A70009B000B4424331B68002B08D17B6818682B
:102A80007B6803F29C431A46012102F033FA7B6A09
:102A9000DBB2194678680BF016FC3B6903F00803BB
:102AA000002B08D07B6A5A01FB69134403F51063BD
:102AB0001A46082393603B6903F01003002B08D0EB
:102AC0007B6A5A01FB69134403F510631A4610230D
:102AD00093603B6903F04003002B08D07B6A5A01E6
:102AE000FB69134403F510631A46402393603B6966
:102AF00003F00203002B23D0796A386A01F012FA3E
:102B00007A6A1346DB0013449B0010337A6813443F
:102B100004337B617B69DB78012B08D17B69002260
:102B2000DA707B6ADBB2194678680BF063FC7B6A6B
:102B30005A01FB69134403F510631A46022393609C
:102B40003B6903F08003002B03D0796A786800F0BA
:102B5000EAFC7B6A01337B62BB6A5B08BB62BB6ACF
:102B6000002B7FF42EAF7B681B68184602F0FCF840
:102B7000034603F00043B3F1004F22D1FB6903F594
:102B800000635B68FA6902F5006223F00103536099
:102B90007B6893F8CC34012B08D17B68002283F842
:102BA000CC24002178680BF0DDFD02E078680BF0A2
:102BB00001FC7B681B685A697B681B6802F0004255
:102BC0005A617B681B68184602F0CEF8034603F48E
:102BD0000063B3F5006F12D1FB6903F500639B68D6
:102BE00003F00103012B02D178680BF0BDFB7B6879
:102BF0001B685A697B681B6802F400625A617B6833
:102C00001B68184602F0B0F8034603F00063B3F106
:102C1000006F21D17B681B685A697B681B6802F0D2
:102C200000625A617B6893F8CC34002B11D17B6829
:102C3000012283F8CC247B681B685B6D9B0803F042
:102C40000F027B68C3F8D024012178680BF08AFD5D
:102C500002E078680BF088FB7B681B68184602F07E
:102C600083F8034603F48053B3F5805F40F0B780E8
:102C7000FB6903F500635B68FA6902F5006223F003
:102C8000010353607B681B681021184601F04AF964
:102C90000023FB6246E0FB6A5A01FB69134403F51B
:102CA00010631A464FF67F339360FB6A5A01FB6943
:102CB000134403F510631B68FA6A5101FA690A4468
:102CC00002F5106223F400131360FB6A5A01FB69DA
:102CD000134403F530631A464FF67F339360FB6A63
:102CE0005A01FB69134403F530631B68FA6A51010A
:102CF000FA690A4402F5306223F400131360FB6A98
:102D00005A01FB69134403F530631B68FA6A5101E9
:102D1000FA690A4402F5306243F000631360FB6A0B
:102D20000133FB627B681B791A46FB6A9342B2D37C
:102D3000FB6903F50063DB69FA6902F5006243F0A1
:102D40000113D3617B68DB7B002B16D0FB6903F595
:102D50000063D3F88430FA6902F5006243F00B0394
:102D6000C2F88430FB6903F500635B6CFA6902F515
:102D7000006243F00B03536415E0FB6903F5006345
:102D80005A69FB6903F50063194642F22B031343AA
:102D90004B61FB6903F500631B69FA6902F5006288
:102DA00043F00B031361FB6903F500631B68FA69C9
:102DB00002F5006223F4FE6313607B6818687B6889
:102DC00099797B6803F29C431A4602F093F87B687A
:102DD0001B685A697B681B6802F480525A617B68E1
:102DE0001B68184601F0C0FF034603F40053B3F517
:102DF000005F23D17B681B68184602F057F87B6898
:102E00001B68184601F007F903461A467B68DA7119
:102E10007B681C6802F042FE01467B68DB791A463B
:102E2000204600F011FE78680BF075FA7B681B688D
:102E30005A697B681B6802F400525A617B681B6800
:102E4000184601F091FF034603F00803082B0AD14E
:102E500078680BF052FA7B681B685A697B681B68BC
:102E600002F008025A617B681B68184601F07CFF7B
:102E7000034603F08003802B23D13B6A9B6923F038
:102E800080023B6A9A6101237B6214E079687A6A66
:102E90001346DB0013449B000B4403F257231B78BB
:102EA000012B05D17B6ADBB21946786800F00AFB7A
:102EB0007B6A01337B627B681B791A467B6A93428B
:102EC000E4D37B681B68184601F04EFF034603F409
:102ED0008013B3F5801F3CD101237B622BE07B6A1A
:102EE0005A01FB69134403F510631B68BB617968E1
:102EF0007A6A1346DB0013449B000B4418331B789B
:102F0000012B15D1BB69002B12DA79687A6A134656
:102F1000DB0013449B000B44173301221A707B6AB9
:102F2000DBB263F07F03DBB21946786800F0CAFABF
:102F30007B6A01337B627B681B791A467B6A93420A
:102F4000CDD37B681B685A697B681B6802F48012CA
:102F50005A617B681B68184601F006FF034603F4BC
:102F60000013B3F5001F56D101237B6245E07B6A55
:102F70005A01FB69134403F530631B68BB61796830
:102F80007A6A1346DB0013449B000B4403F5167367
:102F90001B78012B2ED1BB69002B2BDABB691A0CD5
:102FA0007B68D3F8D434534003F00103002B21D1C4
:102FB00079687A6A1346DB0013449B000B4403F2E2
:102FC000572301221A703B6A9B6943F080023B6AD7
:102FD0009A613B6A5B6903F08003002B0AD1FB69AD
:102FE00003F500635B68FA6902F5006243F400735D
:102FF000536008E07B6A01337B627B681B791A4669
:103000007B6A9342B3D37B681B685A697B681B68F1
:1030100002F400125A617B681B68184601F0A4FE96
:10302000034603F08043B3F1804F0AD178680BF078
:10303000F3F97B681B685A697B681B6802F0804261
:103040005A617B681B68184601F08EFE034603F048
:103050000403042B15D17B681B685B68BB61BB69EB
:1030600003F00403002B02D078680BF0E3F97B68CF
:103070001B6859687B681B68BA690A435A6000E09C
:1030800000BF3437BD4690BD80B582B000AF7860D8
:103090000B46FB707B6893F89434012B01D102231B
:1030A00012E07B68012283F894247B68FA785A74D2
:1030B0007B681B68FA781146184601F0EDFD7B68C5
:1030C000002283F89424002318460837BD4680BDAB
:1030D00080B584B000AF7860084611461A460346B2
:1030E000FB700B463B801346BB700023FB7297F9C5
:1030F0000330002B0FDAFB7803F00F021346DB00DE
:1031000013449B0010337A6813440433FB60FB685C
:1031100001225A700FE0FB7803F00F021346DB0028
:1031200013449B0003F514737A6813440433FB6063
:10313000FB6800225A70FB7803F00F03DAB2FB68D9
:103140001A703B88C3F30A02FB689A60FB68BA787E
:103150001A71FB685B78002B04D0FB681B781A4659
:10316000FB685A83BB78022B02D1FB6800225A719C
:103170007B6893F89434012B01D102230EE07B6825
:10318000012283F894247B681B68F968184600F0D4
:1031900067FF7B68002283F89424FB7A1846103777
:1031A000BD4680BD80B584B000AF78600B46FB7033
:1031B00097F90330002B0FDAFB7803F00F02134668
:1031C000DB0013449B0010337A6813440433FB6024
:1031D000FB6801225A700FE0FB7803F00F021346E0
:1031E000DB0013449B0003F514737A681344043323
:1031F000FB60FB6800225A70FB7803F00F03DAB221
:10320000FB681A707B6893F89434012B01D1022378
:103210000EE07B68012283F894247B681B68F968C0
:10322000184600F0A5FF7B68002283F89424002351
:1032300018461037BD4680BD80B586B000AFF86037
:103240007A603B600B46FB72FB7A03F00F02134679
:10325000DB0013449B0003F51473FA681344043332
:103260007B617B697A68DA607B693A681A617B699D
:1032700000225A617B6900225A70FB7A03F00F0327
:10328000DAB27B691A70FB689B79012B02D17A68EC
:103290007B69DA61FB681868FB689B791A46796973
:1032A00001F042F8002318461837BD4680BD80B4AF
:1032B00083B000AF78600B46FB70FB7803F00F0221
:1032C00079681346DB0013449B000B4403F51A7323
:1032D0001B6818460C37BD465DF8047B704780B507
:1032E00086B000AFF8607A603B600B46FB72FB7AF9
:1032F00003F00F021346DB0013449B001033FA68FF
:10330000134404337B617B697A68DA607B693A68CD
:103310001A617B6900225A617B6901225A70FB7A2B
:1033200003F00F03DAB27B691A70FB689B79012BFB
:1033300002D17A687B69DA61FB681868FB689B795F
:103340001A46796900F0F0FF002318461837BD4689
:1033500080BD80B584B000AF78600B46FB70FB7811
:1033600003F00F037A681279934201D901234FE0E9
:1033700097F90330002B0FDAFB7803F00F021346A6
:10338000DB0013449B0010337A6813440433FB6062
:10339000FB6801225A700DE0FA781346DB001344F3
:1033A0009B0003F514737A6813440433FB60FB68D5
:1033B00000225A70FB6801229A70FB7803F00F0319
:1033C000DAB2FB681A707B6893F89434012B01D150
:1033D00002231DE07B68012283F894247B681B682C
:1033E000F968184601F084FBFB7803F00F03002B0B
:1033F00009D17B6818687B6899797B6803F29C43E4
:103400001A4601F077FD7B68002283F8942400239C
:1034100018461037BD4680BD80B584B000AF7860D7
:103420000B46FB70FB7803F00F037A681279934226
:1034300001D9012342E097F90330002B0FDAFB7822
:1034400003F00F021346DB0013449B0010337A682D
:1034500013440433FB60FB6801225A700FE0FB78D1
:1034600003F00F021346DB0013449B0003F51473B3
:103470007A6813440433FB60FB6800225A70FB68CF
:1034800000229A70FB7803F00F03DAB2FB681A701F
:103490007B6893F89434012B01D102230EE07B6802
:1034A000012283F894247B681B68F968184601F0B0
:1034B0008DFB7B68002283F8942400231846103784
:1034C000BD4680BD80B584B000AF78600B46FB7010
:1034D00097F90330002B0CDAFB7803F00F02134648
:1034E000DB0013449B0010337A6813440433FB6001
:1034F0000CE0FB7803F00F021346DB0013449B0043
:1035000003F514737A6813440433FB607B681B680B
:10351000F968184601F0ACF90346FB72FB7A1846CD
:103520001037BD4680BD80B58AB002AF7860396083
:103530007B681B687B617B693B613A681346DB00F3
:1035400013449B0010337A6813440433FB60FB6818
:103550005A69FB681B699A4201D901236BE0FB6839
:103560001A69FB685B69D31AFB61FB689B68FA699F
:103570009A4202D9FB689B68FB61FB6903339B0895
:10358000BB612AE0FB681A69FB685B69D31AFB61BF
:10359000FB689B68FA699A4202D9FB689B68FB61E9
:1035A000FB6903339B08BB61FB68D9683B68DAB2EF
:1035B000FB6998B27B689B7900930346786901F0B8
:1035C00001FAFB68DA68FB691A44FB68DA60FB6899
:1035D0005A69FB691A44FB685A613B685A013B69A6
:1035E000134403F510639B699BB2BA699A4209D8E8
:1035F000FB685A69FB681B699A4203D2FB681B6926
:10360000002BBFD1FB681A69FB685B699A4211D82D
:103610003B6803F00F03012202FA03F3BB603B692E
:1036200003F500635A6BBB68DB43396901F5006140
:1036300013404B63002318462037BD4680BD000071
:1036400080B588B000AF786039607B681B68FB612B
:10365000FB69BB61FB693C3304331B687B613B68DE
:103660005A01BB69134403F530639B683B617B6877
:103670009B79012B7BD13B6903F00803002B15D00C
:103680007B69614A934240F2B9803B6903F400438D
:10369000002B00F0B3803B685A01BB69134403F56B
:1036A00030631A464FF400439360A7E03B6903F090
:1036B0002003002B09D03B685A01BB69134403F572
:1036C00030631A462023936098E03B6903F0280397
:1036D000002B40F093807B694B4A93420FD93B69A2
:1036E00003F40043002B0AD03B685A01BB69134422
:1036F00003F530631A464FF4004393607EE03A6866
:103700001346DB0013449B0003F514737A681344DB
:103710000433FB60FB681A6A3B685901BB690B44C0
:1037200003F530631B69C3F31203D21AFB685A61B5
:103730003B68002B14D1FB681B69002B09D17B6807
:1037400018687B6803F29C431A46012101F0D2FB02
:1037500006E0FB68DA68FB685B691A44FB68DA60BC
:103760003B68DBB2194678680AF092FD46E07B6957
:10377000264A934224D13B6903F40043002B0AD02C
:103780003B685A01BB69134403F530631A464FF492
:103790000043936032E03B6903F02003002B08D024
:1037A0003B685A01BB69134403F530631A46202372
:1037B00093603B68DBB2194678680AF069FD1DE04A
:1037C0003B68002B14D179683A681346DB00134438
:1037D0009B000B4403F519731B68002B08D17B6811
:1037E00018687B6803F29C431A46002101F082FBB3
:1037F0003B68DBB2194678680AF04AFD0023184698
:103800002037BD4680BD00BF0A30544F0A31544FA7
:1038100080B586B000AF786039607B681B687B61DB
:103820007B693B617B693C3304331B68FB603B680D
:103830005A013B69134403F530639B68BB60FB6826
:10384000154A93420ED9BB6803F40043002B09D0FC
:103850003B685A013B69134403F530631A464FF441
:103860000043936078680AF001FDFB680A4A9342BE
:103870000CD97B689B79012B08D17B6818687B6821
:1038800003F29C431A46012101F034FB0023184641
:103890001837BD4680BD00BF0A30544F80B485B094
:1038A00000AF78600B46FB7013463B807B681B685B
:1038B0005B6ABB60FB78002B07D13B8819047B68EF
:1038C0001B68BA680A439A6228E07B681B689B6A97
:1038D0001B0CBA681344BB600023FB730DE07B68CC
:1038E0001A68FB7B40339B0013445B681B0CBA686F
:1038F0001344BB60FB7B0133FB73FA7BFB78013B1A
:103900009A42ECD33B8818047B681968FB78013B2A
:10391000BA68024340339B000B445A6000231846A8
:103920001437BD465DF8047B704780B483B000AFA8
:1039300078600B467B807B681B687A885A6200231C
:1039400018460C37BD465DF8047B704780B485B0DF
:1039500000AF78607B681B68FB607B680122C3F85E
:10396000D8247B68002283F8CC24FB689B6943F051
:103970000062FB689A61FB685A6D054B1343FA6855
:103980005365002318461437BD465DF8047B704725
:103990000300001084B080B584B000AF786007F1F8
:1039A0001C0080E80E0097F82130012B21D17B68A4
:1039B0009B6B23F480327B689A637B68DA68214BC7
:1039C00013407A68D3607B68DB6823F440127B681D
:1039D000DA6097F82830012B05D17B68DB6843F467
:1039E00080127B68DA60786801F0E2FA0346FB73C4
:1039F00010E07B68DB6843F040027B68DA6078683F
:103A000001F0D6FA0346FB737B689B6B43F480326C
:103A10007B689A63BB7F012B0BD17B689B6843F06B
:103A200006027B689A607B689B6843F020027B6893
:103A30009A60FB7B18461037BD46BDE8804004B055
:103A4000704700BFBFFFBDFF80B487B000AFF86014
:103A5000B9601346FB71FB79022B65D1BB68414A03
:103A6000934206D9BB68404A934202D20F237B613E
:103A700062E0BB683C4A934206D3BB683B4A934230
:103A800002D20E237B6157E0BB68384A934206D3CB
:103A9000BB68374A934202D20D237B614CE0BB687E
:103AA000334A934206D3BB68324A934202D80C236E
:103AB0007B6141E0BB682F4A934206D9BB682E4A1E
:103AC000934202D80B237B6136E0BB682A4A9342BB
:103AD00006D9BB68294A934202D80A237B612BE0AE
:103AE000BB68264A934206D9BB68254A934202D254
:103AF00009237B6120E0BB68214A934206D3BB685F
:103B0000204A934202D808237B6115E0BB681D4A16
:103B1000934206D9BB681C4A934202D207237B61B9
:103B20000AE006237B6107E0FB79002B02D1092321
:103B30007B6101E009237B61FB68DB6823F4705241
:103B4000FB68DA60FB68DA687B699B0203F47053F8
:103B50001A43FB68DA60002318461C37BD465DF83F
:103B6000047B7047BFACD800C0E1E4000024F4003F
:103B7000807306019F491A01FF2C31013FA44C01BB
:103B800000366E011FABA6010048E80180B483B087
:103B900000AF78607B689B6843F001027B689A60A5
:103BA000002318460C37BD465DF8047B704780B48F
:103BB00083B000AF78607B689B6823F001027B686C
:103BC0009A60002318460C37BD465DF8047B7047A9
:103BD00080B584B000AF78600B46FB700023FB60BB
:103BE0007B68DB6823F0C0427B68DA60FB78012BDE
:103BF00015D17B68DB6843F000527B68DA600A20ED
:103C000003F0E4FAFB680A33FB60786801F03FF9DF
:103C10000346012B1ED0FB68C72BF0D91AE0FB78B6
:103C2000002B15D17B68DB6843F080427B68DA604B
:103C30000A2003F0CBFAFB680A33FB60786801F0D6
:103C400026F90346002B05D0FB68C72BF0D901E00D
:103C5000012305E0FB68C82B01D1012300E000230C
:103C600018461037BD4680BD84B080B586B000AF21
:103C7000786007F1240080E80E000023FB757B6864
:103C8000FB6000233B6109E07A683B6940339B009D
:103C9000134400225A603B6901333B613B690E2BA0
:103CA000F2D997F82E30002B1CD1FB6803F5006386
:103CB0005B68FA6802F5006243F0020353607B68B8
:103CC0009B6B23F400127B689A637B681B6843F04C
:103CD00040027B681A607B681B6843F080027B6847
:103CE0001A6005E07B689B6B43F400127B689A6363
:103CF000FB6803F560631A460023136097F82930C8
:103D0000012B0DD197F82730002B04D100217868C2
:103D100000F068F908E00121786800F063F903E039
:103D20000321786800F05EF91021786800F0FAF855
:103D30000346002B01D00123FB75786800F024F9BD
:103D40000346002B01D00123FB75FB6803F50063DC
:103D50001A4600231361FB6803F500631A4600232B
:103D60005361FB6803F500631A460023D361002307
:103D70003B6143E03B695A01FB68134403F5106360
:103D80001B6803F00043B3F1004F18D13B69002BCF
:103D90000AD13B695A01FB68134403F510631A46C4
:103DA0004FF00063136013E03B695A01FB68134452
:103DB00003F510631A464FF09043136008E03B6927
:103DC0005A01FB68134403F510631A46002313607D
:103DD0003B695A01FB68134403F510631A4600233C
:103DE00013613B695A01FB68134403F510631A46DB
:103DF0004FF67F3393603B6901333B6197F8243082
:103E00001A463B699342B5D300233B6143E03B69CB
:103E10005A01FB68134403F530631B6803F0004349
:103E2000B3F1004F18D13B69002B0AD13B695A010D
:103E3000FB68134403F530631A464FF000631360C8
:103E400013E03B695A01FB68134403F530631A46DB
:103E50004FF09043136008E03B695A01FB6813443C
:103E600003F530631A46002313603B695A01FB686F
:103E7000134403F530631A46002313613B695A016A
:103E8000FB68134403F530631A464FF67F339360A3
:103E90003B6901333B6197F824301A463B699342F2
:103EA000B5D3FB6803F500631B69FA6802F500628D
:103EB00023F4807313617B6800229A617B686FF042
:103EC00080425A6197F82630002B05D17B689B69A8
:103ED00043F010027B689A617B689A690F4B134329
:103EE0007A68936197F82A30002B05D07B689B692C
:103EF00043F008027B689A6197F82E30012B05D1B8
:103F00007B689A69064B13437A689361FB7D184678
:103F10001837BD46BDE8804004B0704700383C808B
:103F20000400004080B485B000AF786039600023A1
:103F3000FB60FB680133FB60FB68B3F1706F01D974
:103F400003231BE07B681B69002BF2DA0023FB6074
:103F50003B689B0143F020027B681A61FB680133D8
:103F6000FB60FB68B3F1706F01D9032306E07B6847
:103F70001B6903F02003202BF0D0002318461437D0
:103F8000BD465DF8047B704780B485B000AF7860B3
:103F90000023FB60FB680133FB60FB68B3F1706FCB
:103FA00001D9032318E07B681B69002BF2DA002398
:103FB000FB607B6810221A61FB680133FB60FB68C1
:103FC000B3F1706F01D9032306E07B681B6903F02E
:103FD0001003102BF0D0002318461437BD465DF8AF
:103FE000047B704780B485B000AF78600B46FB70EF
:103FF0007B68FB60FB6803F500631A68FB78F9686F
:1040000001F5006113430B60002318461437BD46C9
:104010005DF8047B704780B487B000AF78607B6840
:104020003B613B6903F500639B6803F00603FB609B
:10403000FB68002B02D10023FB750AE0FB68022B12
:1040400002D0FB68062B02D10223FB7501E00F238F
:10405000FB75FB7D18461C37BD465DF8047B704739
:1040600080B485B000AF786039607B68FB603B68E6
:104070001B78BB603B685B78012B39D1FB6803F58B
:104080000063DA693B681B7803F00F03012101FA32
:1040900003F39BB2F96801F500611343CB61BB6880
:1040A0005A01FB68134403F510631B6803F40043D3
:1040B000002B53D1BB685A01FB68134403F510630E
:1040C0001A683B689B68C3F30A013B681B799B0431
:1040D0001943BB689B050B431A43BB685901FB6836
:1040E0000B4403F510631946204B13430B6035E076
:1040F000FB6803F50063DA693B681B7803F00F0384
:10410000012101FA03F31B04F96801F5006113436F
:10411000CB61BB685A01FB68134403F530631B682D
:1041200003F40043002B19D1BB685A01FB68134408
:1041300003F530631A683B689B68C3F30A013B6868
:104140001B799B040B431A43BB685901FB680B4462
:1041500003F530631946054B13430B6000231846E3
:104160001437BD465DF8047B704700BF0080001027
:1041700080B485B000AF786039607B68FB603B68D5
:104180001B78BB603B685B78012B61D1BB685A012F
:10419000FB68134403F510631B6803F00043B3F19D
:1041A000004F1FD1BB685A01FB68134403F510632D
:1041B0001B68BA685101FA680A4402F5106243F0BC
:1041C00000631360BB685A01FB68134403F5106376
:1041D0001B68BA685101FA680A4402F5106243F09C
:1041E00080431360FB6803F50063DA6B3B681B7860
:1041F00003F00F03012101FA03F39BB2DB43F968DB
:1042000001F500611340CB63FB6803F50063DA69D5
:104210003B681B7803F00F03012101FA03F39BB203
:10422000DB43F96801F500611340CB61BB685A01BB
:10423000FB68134403F510631A68BB685901FB68F7
:104240000B4403F510631946354B13400B6060E0D7
:10425000BB685A01FB68134403F530631B6803F025
:104260000043B3F1004F1FD1BB685A01FB681344F0
:1042700003F530631B68BA685101FA680A4402F515
:10428000306243F000631360BB685A01FB6813445B
:1042900003F530631B68BA685101FA680A4402F5F5
:1042A000306243F080431360FB6803F50063DA6B10
:1042B0003B681B7803F00F03012101FA03F31B0491
:1042C000DB43F96801F500611340CB63FB6803F53C
:1042D0000063DA693B681B7803F00F03012101FAE0
:1042E00003F31B04DB43F96801F500611340CB6164
:1042F000BB685A01FB68134403F530631A68BB6856
:104300005901FB680B4403F530631946054B134014
:104310000B60002318461437BD465DF8047B7047D8
:10432000007833EC0078F3EF80B58AB002AFF86024
:10433000B9601346FB71FB68FB61BB681B78BB610E
:10434000BB685B78012B40F08581BB681B69002B43
:1043500032D1BB695A01FB69134403F510631A6932
:10436000BB695901FB690B4403F510631946A74B60
:1043700013400B61BB695A01FB69134403F51063D9
:104380001B69BA695101FA690A4402F5106243F4E3
:1043900000231361BB695A01FB69134403F51063E1
:1043A0001A69BB695901FB690B4403F5106319468F
:1043B000974B13400B6197E0BB695A01FB691344AB
:1043C00003F510631A69BB695901FB690B4403F5D6
:1043D000106319468E4B13400B61BB695A01FB6990
:1043E000134403F510631A69BB695901FB690B4457
:1043F00003F510631946854B13400B61BB69002B15
:104400001AD1BB681A69BB689B689A4203D9BB681A
:104410009A68BB681A61BB695A01FB69134403F5CA
:1044200010631B69BA695101FA690A4402F5106206
:1044300043F40023136144E0BB681A69BB689B68BE
:1044400013445A1EBB689B68B2FBF3F3FB82BB6943
:104450005A01FB69134403F510631A69FB8AD904F6
:104460006C4B0B40B9694801F969014401F51061D1
:1044700013430B61BB681B79012B22D1BB695A0125
:10448000FB69134403F510631B69BA695101FA69AA
:104490000A4402F5106223F0C0431361BB695A015C
:1044A000FB69134403F510631A69FB8A5B0703F089
:1044B000C043B9694801F969014401F5106113432A
:1044C0000B61BB695A01FB69134403F510631A6958
:1044D000BB681B69C3F31203B9694801F969014458
:1044E00001F5106113430B61FB79012B4BD1BB68C4
:1044F000DB69002B09D0BB695A01FB69134403F542
:1045000010631A46BB68DB695361BB681B79012BDA
:1045100028D1FB6903F500639B6803F48073002BCB
:1045200010D1BB695A01FB69134403F510631B6882
:10453000BA695101FA690A4402F5106243F0005366
:1045400013600FE0BB695A01FB69134403F5106364
:104550001B68BA695101FA690A4402F5106243F016
:1045600080531360BB695A01FB69134403F5106360
:104570001B68BA695101FA690A4402F5106243F0F6
:104580000443136069E1BB695A01FB69134403F5F5
:1045900010631B68BA695101FA690A4402F5106296
:1045A00043F004431360BB681B79012B15D0BB6833
:1045B0001B69002B00F05181FB6903F500635A6B06
:1045C000BB681B7803F00F03012101FA03F3F969BB
:1045D00001F5006113434B633FE1FB6903F50063A1
:1045E0009B6803F48073002B16D1BB695A01FB69E9
:1045F000134403F510631B68BA695101FA690A4450
:1046000002F5106243F00053136015E0FFFF07E06E
:104610000000F8FF0000F81FBB695A01FB69134452
:1046200003F510631B68BA695101FA690A4402F57F
:10463000106243F080531360BB68D968BB681A7876
:10464000BB681B6998B2FB7900930346F86800F0D9
:10465000B9F902E1BB695A01FB69134403F5306300
:104660001A69BB695901FB690B4403F530631946AC
:104670007C4B13400B61BB695A01FB69134403F582
:1046800030631A69BB695901FB690B4403F5306358
:104690001946754B13400B61BB69002B2FD1BB68CA
:1046A0001B69002B03D0BB689A68BB681A61BB68A2
:1046B0009A68BB681A62BB695A01FB69134403F527
:1046C00030631A69BB681B6AC3F31203B9694801F6
:1046D000F969014401F5306113430B61BB695A016B
:1046E000FB69134403F530631B69BA695101FA6928
:1046F0000A4402F5306243F4002313615FE0BB68B3
:104700001B69002B23D1BB695A01FB69134403F5D4
:1047100030631A69BB689B68C3F31203B969480127
:10472000F969014401F5306113430B61BB695A011A
:10473000FB69134403F530631B69BA695101FA69D7
:104740000A4402F5306243F40023136137E0BB688A
:104750001A69BB689B6813445A1EBB689B68B2FB0E
:10476000F3F3FB82BB689B68FA8A03FB02F2BB6827
:104770001A62BB695A01FB69134403F530631A6975
:10478000FB8AD904394B0B40B9694801F9690144E6
:1047900001F5306113430B61BB695A01FB69134496
:1047A00003F530631A69BB681B6AC3F31203B96966
:1047B0004801F969014401F5306113430B61FB794C
:1047C000012B0DD1BB68DB68002B09D0BB68D96811
:1047D000BB695A01FB69134403F530630A465A6109
:1047E000BB681B79012B28D1FB6903F500639B682B
:1047F00003F48073002B10D1BB695A01FB69134489
:1048000003F530631B68BA695101FA690A4402F57D
:10481000306243F0005313600FE0BB695A01FB693B
:10482000134403F530631B68BA695101FA690A44FD
:1048300002F5306243F080531360BB695A01FB6993
:10484000134403F530631B68BA695101FA690A44DD
:1048500002F5306243F0044313600023184620370A
:10486000BD4680BD0000F8FFFFFF07E00000F81F15
:1048700080B487B000AF786039600023FB6000230C
:10488000FB757B683B613B685B78012B4AD13B68D9
:104890001B785A013B69134403F510631B6803F04E
:1048A0000043B3F1004F40F086803B681B785A010B
:1048B0003B69134403F510631B683A681278510191
:1048C0003A690A4402F5106243F0006313603B68E2
:1048D0001B785A013B69134403F510631B683A685F
:1048E000127851013A690A4402F5106243F080439C
:1048F0001360FB680133FB60FB6842F21072934265
:1049000002D90123FB7556E03B681B785A013B69CD
:10491000134403F510631B6803F00043B3F1004F29
:10492000E7D048E03B681B785A013B69134403F524
:1049300030631B6803F00043B3F1004F3BD13B6889
:104940001B785A013B69134403F530631B683A68CE
:10495000127851013A690A4402F5306243F000636B
:1049600013603B681B785A013B69134403F53063BD
:104970001B683A68127851013A690A4402F53062BC
:1049800043F080431360FB680133FB60FB6842F235
:104990001072934202D90123FB750CE03B681B782F
:1049A0005A013B69134403F530631B6803F000436D
:1049B000B3F1004FE7D0FB7D18461C37BD465DF8CC
:1049C000047B704780B489B000AFF860B9601146CD
:1049D0001A460B46FB711346BB80FB687B61BB68C4
:1049E000FB6197F82830002B23D1BB8803339B0849
:1049F0003B610023BB6118E0FB791A037B69134418
:104A000003F580531A46FB691B681360FB69013389
:104A1000FB61FB690133FB61FB690133FB61FB69EE
:104A20000133FB61BB690133BB61BA693B699A42DF
:104A3000E2D3002318462437BD465DF8047B704757
:104A400080B48BB000AFF860B9601346FB80FB68A0
:104A5000BB61BB687B62FB889B089BB27B61FB8868
:104A600003F00303FB8300233B6214E0BB6903F5FF
:104A700080531A687B6A1A607B6A01337B627B6AA7
:104A800001337B627B6A01337B627B6A01337B6229
:104A90003B6A01333B623A6A7B699A42E6D3FB8BFD
:104AA000002B1ED000233B62BB6903F580531A46DE
:104AB00007F1100312681A603A693B6ADBB2DB0047
:104AC00022FA03F3DAB27B6A1A703B6A01333B6263
:104AD0007B6A01337B62FB8B013BFB83FB8B002BEF
:104AE000EAD17B6A18462C37BD465DF8047B7047D7
:104AF00080B485B000AF786039607B68FB603B684C
:104B00001B78BB603B685B78012B2CD1BB685A01DA
:104B1000FB68134403F510631B68002B12DBBB68B2
:104B2000002B0FD0BB685A01FB68134403F51063D8
:104B30001B68BA685101FA680A4402F5106223F052
:104B400080431360BB685A01FB68134403F510638C
:104B50001B68BA685101FA680A4402F5106243F40E
:104B6000001313602BE0BB685A01FB68134403F584
:104B700030631B68002B12DBBB68002B0FD0BB68B7
:104B80005A01FB68134403F530631B68BA6851018E
:104B9000FA680A4402F5306223F080431360BB6870
:104BA0005A01FB68134403F530631B68BA6851016E
:104BB000FA680A4402F5306243F4001313600023DC
:104BC00018461437BD465DF8047B704780B485B045
:104BD00000AF786039607B68FB603B681B78BB6026
:104BE0003B685B78012B28D1BB685A01FB681344F2
:104BF00003F510631B68BA685101FA680A4402F5AC
:104C0000106223F4001313603B681B79032B03D05D
:104C10003B681B79022B38D1BB685A01FB681344EF
:104C200003F510631B68BA685101FA680A4402F57B
:104C3000106243F08053136027E0BB685A01FB68A1
:104C4000134403F530631B68BA685101FA680A44DB
:104C500002F5306223F4001313603B681B79032BC9
:104C600003D03B681B79022B0FD1BB685A01FB684C
:104C7000134403F530631B68BA685101FA680A44AB
:104C800002F5306243F08053136000231846143756
:104C9000BD465DF8047B704780B485B000AF786096
:104CA0000B46FB707B68FB60FB6803F500631B68C9
:104CB000FA6802F5006223F4FE631360FB6803F5F3
:104CC00000631A68FB781B0103F4FE63F96801F5C1
:104CD000006113430B60002318461437BD465DF88E
:104CE000047B704780B485B000AF78607B68FB6060
:104CF000FB6803F560631B68FA6802F5606223F0E5
:104D000003031360FB6803F500635B68FA6802F550
:104D1000006223F002035360002318461437BD4697
:104D20005DF8047B704780B485B000AF78607B6825
:104D3000FB60FB6803F560631B68FA6802F560625C
:104D400023F003031360FB6803F500635B68FA68F4
:104D500002F5006243F00203536000231846143743
:104D6000BD465DF8047B704780B485B000AF7860C5
:104D70007B685B69FB607B689B69FA681340FB603A
:104D8000FB6818461437BD465DF8047B704780B455
:104D900085B000AF78607B68FB60FB6803F500635B
:104DA0009B69BB60FB6803F50063DB69BA6813406D
:104DB000BB60BB681B0C18461437BD465DF8047B0E
:104DC000704780B485B000AF78607B68FB60FB689B
:104DD00003F500639B69BB60FB6803F50063DB6957
:104DE000BA681340BB60BB689BB218461437BD4617
:104DF0005DF8047B704780B485B000AF78600B46E7
:104E0000FB707B68FB60FB785A01FB68134403F579
:104E100030639B68BB60FB6803F500635B69BA683D
:104E20001340BB60BB6818461437BD465DF8047B71
:104E3000704780B487B000AF78600B46FB707B682A
:104E40007B617B6903F500631B693B617B6903F54B
:104E500000635B6BFB60FB7803F00F03FA6822FAD8
:104E600003F3DB01DBB23A6913433B61FB785A0180
:104E70007B69134403F510639B683A691340BB6078
:104E8000BB6818461C37BD465DF8047B704780B48C
:104E900083B000AF78607B685B6903F0010318465C
:104EA0000C37BD465DF8047B7047000080B485B0C8
:104EB00000AF78607B68FB60FB6803F510631A68DD
:104EC000FB6803F510631946094B13400B60FB6840
:104ED00003F500635B68FA6802F5006243F48073CF
:104EE0005360002318461437BD465DF8047B7047B5
:104EF00000F8FFFF80B487B000AFF8600B467A601F
:104F0000FB72FB687B61FB683C3304331B683B61CD
:104F10003B69264A93420AD97B6903F530631B68D3
:104F200003F00043B3F1004F01D1002337E07B6968
:104F300003F530631A46002313617B6903F5306380
:104F40001B697A6902F5306243F4002313617B69BF
:104F500003F530631B697A6902F5306243F0180388
:104F600013617B6903F530631B697A6902F530626E
:104F700043F0C0431361FB7A012B0FD17B6903F52A
:104F800030631A467B6853617B6903F530631B68A5
:104F90007A6902F5306243F08023136000231846DB
:104FA0001C37BD465DF8047B704700BF0A30544F84
:104FB00080B485B000AF78600023FB60FB680133EC
:104FC000FB60FB68B3F1706F01D9032322E07B68BB
:104FD0001B69002BF2DA0A23FB6002E0FB68013B4D
:104FE000FB60FB68002BF9D17B681B6943F0010271
:104FF0007B681A61FB680133FB60FB68B3F1706F7B
:1050000001D9032306E07B681B6903F00103012B30
:10501000F0D0002318461437BD465DF8047B704776
:1050200080B582B000AF02F0C5F87860664B1B68AF
:10503000654A43F00103136008E002F0BBF8024642
:105040007B68D31A022B01D90323B8E05E4B1B689F
:1050500003F00203002BF0D05B4B1B685A4A43F06D
:105060008003136002F0A6F87860574B00229A6024
:105070000AE002F09FF802467B68D31A41F28832B8
:10508000934201D903239AE04F4B9B6803F00C0332
:10509000002BEED102F08EF878604B4B1B684A4A29
:1050A00023F45023136008E002F084F802467B6882
:1050B000D31A642B01D9032381E0434B1B6803F40B
:1050C0000033002BF0D102F075F878603E4B1B687E
:1050D0003D4A23F08073136008E002F06BF802464B
:1050E0007B68D31A022B01D9032368E0364B1B6877
:1050F00003F00073002BF0D102F05CF87860324BC3
:105100001B68314A23F08063136008E002F052F814
:1051100002467B68D31A642B01D903234FE02A4B44
:105120001B6803F00063002BF0D102F043F87860B5
:10513000254B1B68244A23F08053136008E002F0DB
:1051400039F802467B68D31A642B01D9032336E071
:105150001D4B1B6803F00053002BF0D11A4B1B4A68
:105160005A60194B1A4AC3F88420174B184AC3F8DF
:105170008820154BDB68144A23F4FE43D360124B9E
:10518000DB68114A43F47F03D3600F4B5B6F0E4A19
:1051900023F0010353670C4B5B6F0B4A43F08073A2
:1051A00053670C4B0C4A1A600C4B1B6818460CF0EA
:1051B00043FB0346002B01D0012300E000231846E7
:1051C0000837BD4680BD00BF0038024010300024C3
:1051D00000300024000000200024F400040000201F
:1051E00080B586B000AF78600023FB757B68002B2C
:1051F00001D101239BE27B681B6803F00103002BB4
:1052000000F08780964B9B6803F00C03042B0CD0B6
:10521000934B9B6803F00C03082B12D1904B5B68F7
:1052200003F48003B3F5800F0BD18D4B1B6803F49F
:105230000033002B6CD07B685B68002B68D10123A6
:1052400075E27B685B68B3F5803F06D1844B1B68D1
:10525000834A43F4803313602EE07B685B68002B45
:105260000CD17F4B1B687E4A23F4803313607C4B48
:105270001B687B4A23F4802313601DE07B685B6816
:10528000B3F5A02F0CD1764B1B68754A43F48023ED
:105290001360734B1B68724A43F4803313600BE056
:1052A0006F4B1B686E4A23F4803313606C4B1B6892
:1052B0006B4A23F4802313607B685B68002B13D058
:1052C00001F078FF386108E001F074FF02463B69A5
:1052D000D31A642B01D9032329E2614B1B6803F421
:1052E0000033002BF0D014E001F064FF386108E0D7
:1052F00001F060FF02463B69D31A642B01D90323F6
:1053000015E2574B1B6803F40033002BF0D100E08B
:1053100000BF7B681B6803F00203002B69D0504B71
:105320009B6803F00C03002B0BD04D4B9B6803F0E4
:105330000C03082B1CD14A4B5B6803F48003002B41
:1053400016D1474B1B6803F00203002B05D07B6886
:10535000DB68012B01D00123E9E1414B1B6823F0FD
:10536000F8027B681B69DB003D4913430B6040E09A
:105370007B68DB68002B23D0394B1B68384A43F02D
:105380000103136001F016FF386108E001F012FF1D
:1053900002463B69D31A022B01D90323C7E1304BE4
:1053A0001B6803F00203002BF0D02D4B1B6823F089
:1053B000F8027B681B69DB00294913430B6018E086
:1053C000274B1B68264A23F00103136001F0F2FE0D
:1053D000386108E001F0EEFE02463B69D31A022B69
:1053E00001D90323A3E11E4B1B6803F00203002B2A
:1053F000F0D17B681B6803F00803002B38D07B6872
:105400005B69002B19D0164B5B6F154A43F0010303
:10541000536701F0CFFE386108E001F0CBFE024691
:105420003B69D31A022B01D9032380E10C4B5B6F3C
:1054300003F00203002BF0D01AE0094B5B6F084A1F
:1054400023F00103536701F0B5FE38610AE001F073
:10545000B1FE02463B69D31A022B03D9032366E14E
:1054600000380240924B5B6F03F00203002BEED139
:105470007B681B6803F00403002B00F0A4808C4BB6
:105480001B6C03F08053002B0DD1894B1B6C884A99
:1054900043F080531364864B1B6C03F08053BB6056
:1054A000BB680123FB75834B1B6803F48073002BDF
:1054B00018D1804B1B687F4A43F48073136001F05E
:1054C00079FE386108E001F075FE02463B69D31AA7
:1054D000642B01D903232AE1764B1B6803F4807304
:1054E000002BF0D07B689B68012B06D1704B1B6FA3
:1054F0006F4A43F0010313672DE07B689B68002B24
:105500000CD16B4B1B6F6A4A23F001031367684B86
:105510001B6F674A23F0040313671CE07B689B68DA
:10552000052B0CD1624B1B6F614A43F004031367D8
:105530005F4B1B6F5E4A43F0010313670BE05C4B4C
:105540001B6F5B4A23F001031367594B1B6F584ACB
:1055500023F0040313677B689B68002B15D001F0D0
:1055600029FE38610AE001F025FE02463B69D31AA4
:1055700041F28832934201D90323D8E04C4B1B6F90
:1055800003F00203002BEED014E001F013FE3861AB
:105590000AE001F00FFE02463B69D31A41F288325D
:1055A000934201D90323C2E0414B1B6F03F0020376
:1055B000002BEED1FB7D012B05D13D4B1B6C3C4AF2
:1055C00023F0805313647B689B69002B00F0AE804E
:1055D000374B9B6803F00C03082B6DD07B689B69ED
:1055E000022B4BD1324B1B68314A23F0807313607E
:1055F00001F0E0FD386108E001F0DCFD02463B69A6
:10560000D31A022B01D9032391E0294B1B6803F025
:105610000073002BF0D17B68DA697B681B6A1A4340
:105620007B685B6A9B011A437B689B6A5B08013B52
:105630001B041A437B68DB6A1B061A437B681B6BDF
:105640001B071B4913434B60194B1B68184A43F057
:105650008073136001F0AEFD386108E001F0AAFD2F
:1056600002463B69D31A022B01D903235FE0104B9A
:105670001B6803F00073002BF0D057E00C4B1B6845
:105680000B4A23F08073136001F094FD386108E049
:1056900001F090FD02463B69D31A022B01D9032386
:1056A00045E0034B1B6803F00073002BF0D13DE095
:1056B00000380240007000401F4B5B68FB607B6855
:1056C0009B69012B30D0FB6803F480027B68DB69A7
:1056D0009A4229D1FB6803F03F027B681B6A9A4219
:1056E00022D1FA6847F6C07313407A68526A920171
:1056F000934219D1FB6803F440327B689B6A5B08D4
:10570000013B1B049A420FD1FB6803F070627B6877
:10571000DB6A1B069A4207D1FB6803F0E0427B6814
:105720001B6B1B079A4201D0012300E0002318469F
:105730001837BD4680BD00BF0038024080B584B038
:1057400000AF786039600023FB607B68002B01D1DB
:105750000123D0E06A4B1B6803F00F033A689A42BA
:1057600010D9674B1B6823F00F0265493B68134350
:105770000B60634B1B6803F00F033A689A4201D039
:105780000123B8E07B681B6803F00203002B20D0E4
:105790007B681B6803F00403002B05D0594B9B6802
:1057A000584A43F4E05393607B681B6803F0080396
:1057B000002B05D0534B9B68524A43F460439360DF
:1057C000504B9B6823F0F0027B689B684D49134364
:1057D0008B607B681B6803F00103002B40D07B6863
:1057E0005B68012B07D1474B1B6803F40033002B88
:1057F00015D101237FE07B685B68022B07D1414B09
:105800001B6803F00073002B09D1012373E03D4BAB
:105810001B6803F00203002B01D101236BE0394B1D
:105820009B6823F003027B685B68364913438B60F7
:1058300001F0C0FCF8600AE001F0BCFC0246FB6825
:10584000D31A41F28832934201D9032353E02D4BFE
:105850009B6803F00C027B685B689B009A42EBD16B
:10586000274B1B6803F00F033A689A4210D2244B6F
:105870001B6823F00F0222493B6813430B60204B47
:105880001B6803F00F033A689A4201D0012332E00B
:105890007B681B6803F00403002B08D0194B9B683E
:1058A00023F4E0527B68DB68164913438B607B6806
:1058B0001B6803F00803002B09D0124B9B6823F4EC
:1058C00060427B681B69DB000E4913438B6000F06C
:1058D00021F802460B4B9B681B0903F00F030A4992
:1058E000CB5C22FA03F3094A1360094B1B68184684
:1058F0000BF0A2FF002318461037BD4680BD00BF45
:10590000003C024000380240C4B4030800000020FC
:10591000040000202DE9B04F90B000AF00237B635E
:105920000023FB6300233B630023BB63584B9B684E
:1059300003F00C03082B0DD0082B00F2A080002BE5
:1059400002D0042B03D09AE0524BBB639AE0524B37
:10595000BB6397E04E4B5B6803F03F037B634C4BAC
:105960005B6803F48003002B27D0494B5B689B09DD
:1059700000223B627A623B6AC3F308000021464B77
:1059800003FB01F2002300FB03F31344424AA0FB94
:105990000221F962BA62FA6A1344FB627B6B00224D
:1059A000BB61FA61D7E90623D7E90A01FAF7E4FCFB
:1059B00002460B461346FB6353E0354B5B689B097D
:1059C00000223B617A613B69C3F3080A4FF0000B88
:1059D00052465B464FF000004FF00001590141EA8A
:1059E000D261500102460B46B2EB0A0863EB0B0989
:1059F0004FF000024FF000034FEA891343EA986327
:105A00004FEA8812B2EB080463EB09054FF000027D
:105A10004FF00003EB0043EA5473E20014461D46C6
:105A200014EB0A033B6045EB0B037B604FF0000275
:105A30004FF00003D7E9004529468B02214643EA8F
:105A4000915321468A02104619467B6B0022BB60A7
:105A5000FA60D7E90223FAF78FFC02460B46134699
:105A6000FB630B4B5B681B0C03F0030301335B0010
:105A70003B63FA6B3B6BB2FBF3F3BB6302E0054B9A
:105A8000BB6300BFBB6B18464037BD46BDE8B08F57
:105A9000003802400024F40040787D0180B400AF5B
:105AA000034B1B681846BD465DF8047B704700BF7A
:105AB0000000002080B500AFFFF7F0FF0246054B65
:105AC0009B689B0A03F007030349CB5C22FA03F3AC
:105AD000184680BD00380240D4B4030880B483B0B7
:105AE00000AF786039607B680F221A60124B9B68A8
:105AF00003F003027B685A600F4B9B6803F0F002CF
:105B00007B689A600C4B9B6803F4E0527B68DA6018
:105B1000094B9B68DB0803F4E0527B681A61074B72
:105B20001B6803F00F023B681A6000BF0C37BD46CC
:105B30005DF8047B704700BF00380240003C024023
:105B400080B588B000AF786000237B6100233B61A3
:105B50000023FB600023FB610023BB617B681B68A3
:105B600003F00103002B12D0694B9B68684A23F4B1
:105B700000039360664B9A687B685B6B64491343D0
:105B80008B607B685B6B002B01D10123FB617B6821
:105B90001B6803F40023002B17D05D4BD3F88C3027
:105BA00023F440127B68DB6B59491343C1F88C30F6
:105BB0007B68DB6BB3F5801F01D10123FB617B6840
:105BC000DB6B002B01D10123BB617B681B6803F4F5
:105BD0008013002B17D04E4BD3F88C3023F44002A7
:105BE0007B681B6C4A491343C1F88C307B681B6C83
:105BF000B3F5800F01D10123FB617B681B6C002B87
:105C000001D10123BB617B681B6803F08073002B0B
:105C100001D00123FB617B681B6803F02003002B8C
:105C200000F08B803A4B1B6C394A43F0805313646D
:105C3000374B1B6C03F08053BB60BB68354B1B6854
:105C4000344A43F48073136001F0B4FA786108E0D9
:105C500001F0B0FA02467B69D31A642B01D9032301
:105C60008FE32C4B1B6803F48073002BF0D0284B80
:105C70001B6F03F440733B613B69002B35D07B689D
:105C80001B6B03F440733A699A422ED0204B1B6F72
:105C900023F440733B611E4B1B6F1D4A43F480335A
:105CA00013671B4B1B6F1A4A23F480331367184A80
:105CB0003B691367164B1B6F03F00103012B14D1D3
:105CC00001F078FA78610AE001F074FA02467B6923
:105CD000D31A41F28832934201D9032351E30C4B8A
:105CE0001B6F03F00203002BEED07B681B6B03F4E9
:105CF0004073B3F5407F11D1054B9B6823F4F81234
:105D00007B68196B044B0B40014913438B600BE01C
:105D10000038024000700040FFFCFF0FAC4B9B6856
:105D2000AB4A23F4F8139360A94B1A6F7B681B6B83
:105D3000C3F30B03A64913430B677B681B6803F08F
:105D40001003002B10D0A24BD3F88C30A04A23F0C4
:105D50008073C2F88C309E4BD3F88C207B689B6B91
:105D60009B491343C1F88C307B681B6803F4804364
:105D7000002B0AD0964BD3F8903023F440327B6846
:105D80005B6E93491343C1F890307B681B6803F442
:105D90000043002B0AD08E4BD3F8903023F44022DE
:105DA0007B689B6E8A491343C1F890307B681B68FF
:105DB00003F48033002B0AD0854BD3F8903023F4C2
:105DC00040127B68DB6E82491343C1F890307B68D8
:105DD0001B6803F40033002B0AD07D4BD3F89030BE
:105DE00023F440027B681B6F79491343C1F890305C
:105DF0007B681B6803F04003002B0AD0744BD3F878
:105E0000903023F003027B685B6C71491343C1F847
:105E100090307B681B6803F08003002B0AD06C4B2A
:105E2000D3F8903023F00C027B689B6C68491343D5
:105E3000C1F890307B681B6803F48073002B0AD094
:105E4000634BD3F8903023F030027B68DB6C604901
:105E50001343C1F890307B681B6803F40073002B78
:105E60000AD05B4BD3F8903023F0C0027B681B6DE7
:105E700057491343C1F890307B681B6803F4806373
:105E8000002B0AD0524BD3F8903023F440727B6839
:105E90005B6D4F491343C1F890307B681B6803F476
:105EA0000063002B0AD04A4BD3F8903023F44062B1
:105EB0007B689B6D46491343C1F890307B681B6833
:105EC00003F48053002B0AD0414BD3F8903023F4D5
:105ED00040527B68DB6D3E491343C1F890307B68CC
:105EE0001B6803F40053002B0AD0394BD3F89030D1
:105EF00023F440427B681B6E35491343C1F8903050
:105F00007B681B6803F48003002B0AD0304BD3F866
:105F1000903023F080627B689B6F2D491343C1F85A
:105F200090307B681B6803F40013002B11D0284BC2
:105F3000D3F8903023F000627B68DB6F2449134371
:105F4000C1F890307B68DB6FB3F1006F01D10123A2
:105F5000BB617B681B6803F00803002B01D00123A1
:105F6000BB617B681B6803F48023002B0AD0184BAD
:105F7000D3F8903023F040727B685B6F1449134371
:105F8000C1F890307B681B6803F40003002B0BD032
:105F90000F4BD3F8903023F080527B68D3F88030D9
:105FA0000B491343C1F890307B681B6803F0806392
:105FB000002B0FD0064BD3F8903023F000527B68B3
:105FC000D3F8843002491343C1F8903002E000BF97
:105FD000003802407B681B6803F00063002B0BD085
:105FE0008A4BD3F88C3023F000727B68D3F888306A
:105FF00086491343C1F88C307B681B6803F08053DB
:10600000002B0BD0814BD3F88C3023F080627B685F
:10601000D3F88C307D491343C1F88C30FB69012BD8
:1060200006D07B681B6803F00073002B00F0D6805D
:10603000764B1B68754A23F08063136001F0BAF851
:10604000786108E001F0B6F802467B69D31A642B48
:1060500001D9032395E16D4B1B6803F00063002B0E
:10606000F0D17B681B6803F00103002B21D07B6813
:106070005B6B002B1DD1654BD3F884301B0C03F0F8
:1060800003033B61614BD3F884301B0E03F00F0315
:10609000FB607B685B689A013B691B041A43FB68E1
:1060A0001B061A437B689B681B0758491343C1F8BA
:1060B00084307B681B6803F40023002B04D07B68CA
:1060C000DB6BB3F5801F0AD07B681B6803F4801379
:1060D000002B2ED07B681B6CB3F5800F29D14B4B66
:1060E000D3F884301B0C03F003033B61474BD3F818
:1060F00084301B0F03F00703FB607B685B689A0129
:106100003B691B041A437B68DB681B061A43FB6868
:106110001B073E491343C1F884303C4BD3F88C3005
:1061200023F01F027B685B6A013B38491343C1F8C7
:106130008C307B681B6803F08073002B1DD0334BC1
:10614000D3F884301B0E03F00F033B612F4BD3F8C1
:1061500084301B0F03F00703FB607B685B689A01C8
:106160007B681B691B041A433B691B061A43FB68C7
:106170001B0726491343C1F884307B681B6803F072
:106180000073002B11D07B685B689A017B681B69E8
:106190001B041A437B68DB681B061A437B689B68F9
:1061A0001B071A491343C1F88430184B1B68174A60
:1061B00043F08063136000F0FDFF786108E000F0B9
:1061C000F9FF02467B69D31A642B01D90323D8E077
:1061D0000E4B1B6803F00063002BF0D0BB69012B52
:1061E00040F0CE80094B1B68084A23F080531360AF
:1061F00000F0E0FF78610BE000F0DCFF02467B6915
:10620000D31A642B04D90323BBE000BF003802403B
:106210005E4B1B6803F00053B3F1005FECD07B686A
:106220001B6803F40023002B03D07B68DB6B002B7F
:1062300009D07B681B6803F48013002B2ED07B6889
:106240001B6C002B2AD1514BD3F888301B0C03F068
:1062500003033B614D4BD3F888301B0F03F007035A
:10626000FB607B685B699A013B691B041A437B688E
:106270009B691B061A43FB681B0744491343C1F87B
:106280008830424BD3F88C3023F4F8527B689B6AF9
:10629000013B1B023D491343C1F88C307B681B68EE
:1062A00003F40013002B22D07B68DB6FB3F1006F87
:1062B0001DD1364BD3F888301B0E03F00F033B6122
:1062C000324BD3F888301B0F03F00703FB607B6869
:1062D0005B699A017B681B6A1B041A433B691B06B6
:1062E0001A43FB681B0729491343C1F888307B68B0
:1062F0001B6803F00803002B28D0244BD3F8883008
:106300001B0E03F00F033B61204BD3F888301B0CAE
:1063100003F00303FB607B685B699A01FB681B0465
:106320001A433B691B061A437B68DB691B07174945
:106330001343C1F88830154BD3F88C3023F4403226
:106340007B68DB6A11491343C1F88C300F4B1B6823
:106350000E4A43F08053136000F02CFF786108E090
:1063600000F028FF02467B69D31A642B01D903236E
:1063700007E0064B1B6803F00053B3F1005FEFD159
:10638000002318462037BD4680BD00BF00380240BC
:1063900080B586B000AFF860B960C7E90023274B2D
:1063A0001B7D012B01D1022343E0244B01221A75EE
:1063B0004CF2503000F084F80346FB75FB7D002B57
:1063C00033D1FB68032B23D801A252F823F000BF7E
:1063D000E1630108ED630108F96301080564010840
:1063E0003B781946B86800F02DF912E03B88194651
:1063F000B86800F001F90CE03B681946B86800F095
:10640000D5F806E0D7E90023B86800F099F800E075
:1064100000BF4CF2503000F053F80346FB75084BB8
:106420001B69074A23F001031361044B00221A750C
:10643000FB7D18461837BD4680BD00BF9403002081
:10644000003C024080B483B000AF0023FB710B4BD3
:106450001B69002B0BDA094B094A5A60074B094AA2
:106460005A60064B1B69002B01DA0123FB71FB7993
:1064700018460C37BD465DF8047B7047003C02406F
:1064800023016745AB89EFCD80B400AF054B1B6995
:10649000044A43F00043136100231846BD465DF8EB
:1064A000047B7047003C024080B400AF034B9B6903
:1064B0001846BD465DF8047B704700BF940300207A
:1064C00080B584B000AF78600023FB601A4B0022D7
:1064D0009A6100F06FFEF86010E07B68B3F1FF3F57
:1064E0000CD07B68002B07D000F064FE0246FB68EE
:1064F000D31A7A689A4201D2032319E00F4BDB6862
:1065000003F48033002BE8D10C4BDB6803F0F2037B
:10651000002B03D000F0BAF8012309E0074BDB6839
:1065200003F00103002B02D0044B0122DA600023A8
:1065300018461037BD4680BD94030020003C024041
:1065400080B485B000AFF860C7E90023164B1B6923
:10655000154A23F440731361134B1B69124A43F429
:1065600040731361104B1B690F4A43F00103136121
:10657000FB683A681A60BFF36F8F00BFD7E900016C
:106580004FF000024FF000030A000023F9680431C5
:1065900013460B60BFF34F8F00BF00BF1437BD46DB
:1065A0005DF8047B704700BF003C024080B483B0BC
:1065B00000AF786039600F4B1B690E4A23F44073BB
:1065C00013610C4B1B690B4A43F400731361094BB5
:1065D0001B69084A43F0010313617B683A681A603B
:1065E000BFF34F8F00BF00BF0C37BD465DF8047B83
:1065F000704700BF003C024080B483B000AF7860B9
:106600000B467B800E4B1B690D4A23F440731361CC
:106610000B4B1B690A4A43F480731361084B1B69D7
:10662000074A43F0010313617B687A881A80BFF33D
:106630004F8F00BF00BF0C37BD465DF8047B70472D
:10664000003C024080B483B000AF78600B46FB7022
:106650000D4B1B690C4A23F4407313610A4B0A4A21
:106660001B691361084B1B69074A43F0010313615F
:106670007B68FA781A70BFF34F8F00BF00BF0C37EA
:10668000BD465DF8047B7047003C024080B400AF1B
:10669000214BDB6803F00203002B05D01F4B9B69E5
:1066A00043F020031D4A93611B4BDB6803F010038A
:1066B000002B05D0194B9B6943F01003174A9361D7
:1066C000154BDB6803F02003002B05D0134B9B69AF
:1066D00043F00803114A93610F4BDB6803F040035A
:1066E000002B05D00D4B9B6943F004030B4A9361CB
:1066F000094BDB6803F08003002B05D0074B9B6937
:1067000043F00203054A9361034BF222DA6000BFB3
:10671000BD465DF8047B7047003C024094030020B6
:1067200080B584B000AF786039600023BB60304B27
:106730001B7D012B01D1022356E02D4B01221A753E
:106740004CF25030FFF7BCFE0346FB73FB7B002B83
:1067500046D13B684FF0FF321A607B681B68012B03
:1067600015D17B681B69DAB27B685B6819461046F5
:1067700000F044F84CF25030FFF7A2FE0346FB73E2
:106780001C4B1A691B491C4B13400B6128E07B68AA
:106790009B68BB601CE07B681B69DBB21946B8686C
:1067A00000F068F84CF25030FFF78AFE0346FB73A6
:1067B000104B1B690F4A23F0FA031361FB7B002B7C
:1067C00003D03B68BA681A600AE0BB680133BB605B
:1067D0007B68DA687B689B681344BA689A42DAD3AC
:1067E000034B00221A75FB7B18461037BD4680BD4F
:1067F00094030020003C0240FB7FFFFF80B483B085
:1068000000AF03463960FB71194B1B69184A23F42A
:10681000407313613B68032B07D1154B1A69144968
:1068200048F2040313430B610FE03B68022B06D1CF
:106830000F4B1B690E4A43F40043136105E00C4BF8
:106840001B690B4A43F004031361094B1A69FB7976
:106850001B021343064A43F480331361BFF34F8F87
:1068600000BF00BF0C37BD465DF8047B704700BF1A
:10687000003C024080B485B000AF78600B46FB70EE
:106880000023FB60FB78002B02D10023FB6010E0AB
:10689000FB78012B03D14FF48073FB6009E0FB7898
:1068A000022B03D14FF40073FB6002E04FF44073FE
:1068B000FB607B680B2B02D97B6804337B60154B34
:1068C0001B69144A23F440731361124B1A6911496E
:1068D000FB6813430B610F4B1B690E4A23F0F8034F
:1068E00013610C4B1A697B68DB001343094A43F0C0
:1068F00002031361074B1B69064A43F4803313619B
:10690000BFF34F8F00BF00BF1437BD465DF8047B57
:10691000704700BF003C024080B489B000AF78608F
:1069200039600023FB6100237B6100233B6100236E
:10693000BB610023FB6175E10122FB6902FA03F3ED
:106940007B613B681B687A6913403B613A697B69EC
:106950009A4240F064813B685B6803F00303012BBB
:1069600005D03B685B6803F00303022B30D17B68E2
:106970009B68BB61FB695B00032202FA03F3DB4304
:10698000BA691340BB613B68DA68FB695B0002FAD5
:1069900003F3BA691343BB617B68BA699A607B6889
:1069A0005B68BB610122FB6902FA03F3DB43BA694E
:1069B0001340BB613B685B681B0903F00102FB6984
:1069C00002FA03F3BA691343BB617B68BA695A6080
:1069D0003B685B6803F00303032B17D07B68DB681D
:1069E000BB61FB695B00032202FA03F3DB43BA6974
:1069F0001340BB613B689A68FB695B0002FA03F3D2
:106A0000BA691343BB617B68BA69DA603B685B684B
:106A100003F00303022B23D1FB69DA087B680832F9
:106A200053F82230BB61FB6903F007039B000F2280
:106A300002FA03F3DB43BA691340BB613B681A698E
:106A4000FB6903F007039B0002FA03F3BA691343DF
:106A5000BB61FB69DA087B680832B96943F8221028
:106A60007B681B68BB61FB695B00032202FA03F3CE
:106A7000DB43BA691340BB613B685B6803F0030208
:106A8000FB695B0002FA03F3BA691343BB617B68DD
:106A9000BA691A603B685B6803F44033002B00F06E
:106AA000BE80664B5B6C654A43F480435364634B22
:106AB0005B6C03F48043FB60FB68614AFB699B08E5
:106AC000023352F82330BB61FB6903F003039B00E0
:106AD0000F2202FA03F3DB43BA691340BB617B6800
:106AE000584A934237D07B68574A934231D07B68EB
:106AF000564A93422BD07B68554A934225D07B68F7
:106B0000544A93421FD07B68534A934219D07B6802
:106B1000524A934213D07B68514A93420DD07B680E
:106B2000504A934207D07B684F4A934201D10923D0
:106B300012E00A2310E008230EE007230CE00623EE
:106B40000AE0052308E0042306E0032304E002230F
:106B500002E0012300E00023FA6902F00302920040
:106B60009340BA691343BB613549FB699B08023303
:106B7000BA6941F823203D4B9B68BB613B69DB430D
:106B8000BA691340BB613B685B6803F48013002B58
:106B900003D0BA693B691343BB61344ABB69936054
:106BA000324BDB68BB613B69DB43BA691340BB61B5
:106BB0003B685B6803F40013002B03D0BA693B69A0
:106BC0001343BB61294ABB69D360284B5B68BB6137
:106BD0003B69DB43BA691340BB613B685B6803F404
:106BE0000033002B03D0BA693B691343BB611F4AD2
:106BF000BB6953601D4B1B68BB613B69DB43BA69D2
:106C00001340BB613B685B6803F48033002B03D007
:106C1000BA693B691343BB61144ABB691360FB69E2
:106C20000133FB61FB690F2B7FF686AE00BF00BF0F
:106C30002437BD465DF8047B704700BF0038024032
:106C400000380140000002400004024000080240F9
:106C5000000C0240001002400014024000180240E4
:106C6000001C02400020024000240240003C014081
:106C700080B487B000AF7860396000233B610023A7
:106C8000FB600023BB6000237B61D9E001227B69AC
:106C900002FA03F33B613A683B691340FB60FA6810
:106CA0003B699A4240F0C9806B4A7B699B0802337A
:106CB00052F82330BB607B6903F003039B000F2273
:106CC00002FA03F3BA681340BB607B68634A9342DD
:106CD00037D07B68624A934231D07B68614A9342E5
:106CE0002BD07B68604A934225D07B685F4A9342F1
:106CF0001FD07B685E4A934219D07B685D4A9342FD
:106D000013D07B685C4A93420DD07B685B4A934208
:106D100007D07B685A4A934201D1092312E00A2323
:106D200010E008230EE007230CE006230AE0052309
:106D300008E0042306E0032304E0022302E0012329
:106D400000E000237A6902F0030292009340BA68DF
:106D50009A4232D14B4B1A68FB68DB4349491340D6
:106D60000B60484B5A68FB68DB43464913404B6055
:106D7000444BDA68FB68DB4342491340CB60414B2C
:106D80009A68FB68DB433F4913408B607B6903F0E3
:106D900003039B000F2202FA03F3BB602E4A7B69B8
:106DA0009B08023352F82310BB68DA432A487B69F8
:106DB0009B080A40023340F823207B681A687B69ED
:106DC0005B00032101FA03F3DB431A407B681A607E
:106DD0007B69DA087B68083253F822107B6903F07C
:106DE00007039B000F2202FA03F3DB437A69D20800
:106DF00019407B68083243F822107B68DA687B69A7
:106E00005B00032101FA03F3DB431A407B68DA607D
:106E10007B685A6801217B6901FA03F3DB431A405E
:106E20007B685A607B689A687B695B00032101FA82
:106E300003F3DB431A407B689A607B6901337B6113
:106E40007B690F2B7FF622AF00BF00BF1C37BD460A
:106E50005DF8047B704700BF00380140000002402D
:106E60000004024000080240000C024000100240F2
:106E70000014024000180240001C024000200240A2
:106E800000240240003C014080B485B000AF78602F
:106E90000B467B807B681A697B881340002B02D0ED
:106EA0000123FB7301E00023FB73FB7B18461437BF
:106EB000BD465DF8047B704780B483B000AF786056
:106EC0000B467B8013467B707B78002B03D07A883F
:106ED0007B689A6103E07B881A047B689A6100BF33
:106EE0000C37BD465DF8047B7047000080B400AFEE
:106EF000054B1B68044A43F48073136000BFBD4612
:106F00005DF8047B704700BF0070004080B582B020
:106F100000AF00237B60234B1B6C224A43F080535D
:106F20001364204B1B6C03F080533B603B681E4B8B
:106F30001B681D4A43F48033136000F03BF978600E
:106F400009E000F037F902467B68D31AB3F57A7F7F
:106F500001D9032322E0144B5B6803F48033B3F5BB
:106F6000803FEED1104B1B680F4A43F4003313608F
:106F700000F020F9786009E000F01CF902467B6817
:106F8000D31AB3F57A7F01D9032307E0064B5B6878
:106F900003F40033B3F5003FEED100231846083761
:106FA000BD4680BD003802400070004080B485B00E
:106FB00000AF78607B6803F00703FB600B4BDB6876
:106FC000BB60BA684FF6FF031340BB60FB681A0250
:106FD000BB681A43064B1343BB60044ABB68D360CB
:106FE00000BF1437BD465DF8047B704700ED00E03C
:106FF0000000FA0580B400AF044BDB681B0A03F005
:1070000007031846BD465DF8047B704700ED00E0BD
:1070100080B483B000AF0346FB7197F90730002BB3
:107020000BDBFB7903F01F02074997F907305B0977
:10703000012000FA02F241F8232000BF0C37BD46C0
:107040005DF8047B704700BF00E100E080B483B0CE
:1070500000AF03463960FB7197F90730002B0ADB5C
:107060003B68DAB20C4997F907301201D2B20B44EF
:1070700083F800230AE03B68DAB20849FB7903F0A1
:107080000F03043B1201D2B20B441A7600BF0C3737
:10709000BD465DF8047B704700E100E000ED00E0D4
:1070A00080B489B000AFF860B9607A60FB6803F023
:1070B0000703FB61FB69C3F10703042B28BF04230B
:1070C000BB61FB690433062B02D9FB69033B00E07B
:1070D00000237B614FF0FF32BB6902FA03F3DA430E
:1070E000BB681A407B699A404FF0FF317B6901FA17
:1070F00003F3D9437B680B40134318462437BD463E
:107100005DF8047B704780B582B000AF7860786826
:10711000FFF74CFF00BF0837BD4680BD80B586B085
:1071200000AF0346B9607A60FB7300237B61FFF711
:1071300061FF78617A68B9687869FFF7B1FF024644
:1071400097F90F3011461846FFF780FF00BF183738
:10715000BD4680BD80B582B000AF0346FB7197F994
:1071600007301846FFF754FF00BF0837BD4680BD03
:1071700080B500AF0320FFF7C6FF05200AF05CFBD7
:1071800009F08AFE0023184680BD000080B400AFDD
:10719000064B1B781A46064B1B681344044A1360BF
:1071A00000BFBD465DF8047B704700BF08000020AB
:1071B000B003002080B400AF034B1B681846BD46E7
:1071C0005DF8047B704700BFB003002080B584B039
:1071D00000AF7860FFF7EEFFB8607B68FB60FB688C
:1071E000B3F1FF3F05D00A4B1B781A46FB681344E6
:1071F000FB6000BFFFF7DEFF0246BB68D31AFA68E8
:107200009A42F7D800BF00BF1037BD4680BD00BF0F
:107210000800002080B400AF034B1B681846BD4631
:107220005DF8047B704700BF20F4F01F80B400AF0E
:10723000034B1B681846BD465DF8047B704700BFD2
:1072400024F4F01F80B400AF034B1B681846BD4602
:107250005DF8047B704700BF28F4F01F80B584B050
:1072600000AF78600023FB737B68002B01D1012302
:1072700031E07B681B6C002B09D1786809F034FE83
:107280007B6800225A647B68002283F83C207B687C
:107290001B6C03F01003002B16D17B681A6C104B8B
:1072A000134043F002027B681A64786800F00EFB1A
:1072B0007B6800225A647B681B6C23F0030343F055
:1072C00001027B681A6401E00123FB737B680022E2
:1072D00083F83C20FB7B18461037BD4680BD00BFBD
:1072E000FDEEFFFF80B485B000AF78600023FB6047
:1072F0007B6893F83C30012B01D10223ADE07B6821
:10730000012283F83C207B681B689B6803F0010323
:10731000012B18D07B681B689A687B681B6842F059
:1073200001029A60504B1B68504AA2FB03239A0C3F
:1073300013465B001344FB6002E0FB68013BFB600B
:10734000FB68002BF9D17B681B689B6803F0010385
:10735000012B75D17B681A6C454B134043F4807246
:107360007B681A647B681B685B6803F48063002B8E
:1073700007D07B681B6C23F4405343F480527B6836
:107380001A647B681B6C03F48053B3F5805F06D1ED
:107390007B685B6C23F006027B685A6402E07B68C2
:1073A00000225A647B68002283F83C207B681B68BB
:1073B0006FF022021A602F4B5B6803F01F03002B53
:1073C0000FD17B681B689B6803F04053002B43D1AF
:1073D0007B681B689A687B681B6842F080429A60F1
:1073E0003AE07B681B68244A93420ED17B681B6895
:1073F0009B6803F04053002B07D17B681B689A6899
:107400007B681B6842F080429A601A4B5B6803F00D
:107410001003002B20D17B681B68184A93421BD1B4
:107420007B681B689B6803F04053002B14D17B687A
:107430001B689A687B681B6842F080429A600BE088
:107440007B681B6C43F010027B681A647B685B6C82
:1074500043F001027B685A64002318461437BD4686
:107460005DF8047B704700BF0000002083DE1B43F3
:10747000FEF8FFFF002301400020014000220140F0
:1074800080B483B000AF78607B6893F83C30012B08
:1074900001D102231FE07B68012283F83C207B6836
:1074A0001B689A687B681B6822F001029A607B68FF
:1074B0001B689B6803F00103002B07D17B681A6CE3
:1074C000084B134043F001027B681A647B6800227A
:1074D00083F83C20002318460C37BD465DF8047B3A
:1074E000704700BFFEEEFFFF80B584B000AF78604C
:1074F00039600023FB607B681B689B6803F4806332
:10750000B3F5806F13D17B681B689B6803F48073AD
:10751000B3F5807F0BD17B681B6C43F020027B6846
:107520001A647B68002283F83C20012363E0FFF7A4
:1075300041FEF86021E03B68B3F1FF3F1DD03B689E
:10754000002B07D0FFF736FE0246FB68D31A3A68D5
:107550009A4212D27B681B681B6803F00203022B5D
:107560000BD07B681B6C43F004027B681A647B6859
:10757000002283F83C2003233DE07B681B681B68E6
:1075800003F00203022BD6D17B681B686FF0120256
:107590001A607B681B6C43F400727B681A647B681A
:1075A0001B689B6803F04053002B23D17B689B69C9
:1075B000002B1FD17B681B68DB6A03F47003002B70
:1075C00006D07B681B689B6803F48063002B11D195
:1075D0007B681B6C23F480727B681A647B681B6C6D
:1075E00003F48053002B05D17B681B6C43F0010230
:1075F0007B681A64002318461037BD4680BD80B4EE
:1076000083B000AF78607B681B68DB6C18460C3772
:10761000BD465DF8047B704780B485B000AF7860EC
:1076200039600023FB607B6893F83C30012B01D16B
:1076300002233AE17B68012283F83C203B681B6807
:10764000092B3AD93B681B68B3F1004F35D07B68F2
:107650001B68D9683B681B689BB21A4613465B00DF
:1076600013441E3B072202FA03F3DA437B681B68CC
:107670000A40DA603B681B688F4A93420AD17B68F4
:107680001B68D9683B689B681A067B681B680A43BD
:10769000DA6039E07B681B68D9683B689A683B68A8
:1076A0001B689BB2184603465B0003441E3B9A408E
:1076B0007B681B680A43DA6026E07B681B681969EF
:1076C0003B681B689BB21A4613465B00134403F0E9
:1076D0001F03072202FA03F3DA437B681B680A40A0
:1076E0001A617B681B6819693B689A683B681B686C
:1076F0009BB2184603465B00034403F01F039A4005
:107700007B681B680A431A613B685B68062B24D8B8
:107710007B681B68596B3B685A6813469B0013448F
:10772000053B1F2202FA03F3DA437B681B680A4019
:107730005A637B681B68596B3B681B689BB2184691
:107740003B685A6813469B001344053B00FA03F25A
:107750007B681B680A435A634CE03B685B680C2BF0
:1077600024D87B681B68196B3B685A6813469B00DA
:107770001344233B1F2202FA03F3DA437B681B689E
:107780000A401A637B681B68196B3B681B689BB2D5
:1077900018463B685A6813469B001344233B00FA83
:1077A00003F27B681B680A431A6323E07B681B684B
:1077B000D96A3B685A6813469B001344413B1F2219
:1077C00002FA03F3DA437B681B680A40DA627B68DB
:1077D0001B68D96A3B681B689BB218463B685A68AD
:1077E00013469B001344413B00FA03F27B681B687D
:1077F0000A43DA627B681B68304A93420AD13B68CD
:107800001B68B3F1004F05D12D4B5B682C4A23F464
:10781000400353607B681B68284A93420FD13B6842
:107820001B68122B0BD1264B5B68254A23F40003FF
:107830005360234B5B68224A43F4800353607B68A8
:107840001B681E4A93422BD13B681B681A4A93421D
:1078500003D03B681B68112B22D1194B5B68184A77
:1078600023F480035360164B5B68154A43F400030E
:1078700053603B681B68104A934211D1114B1B683F
:10788000114AA2FB03239A0C13469B0013445B008E
:10789000FB6002E0FB68013BFB60FB68002BF9D159
:1078A0007B68002283F83C20002318461437BD462D
:1078B0005DF8047B704700BF1200001000200140FB
:1078C000002301400000002083DE1B4380B483B00E
:1078D00000AF7860784B5B68774A23F4403353609D
:1078E000754B5A687B685B68734913434B607B68D0
:1078F0001B685A687B681B6822F480725A607B6838
:107900001B6859687B681B691A027B681B680A43FD
:107910005A607B681B685A687B681B6822F040725B
:107920005A607B681B6859687B689A687B681B682B
:107930000A435A607B681B689A687B681B6822F45C
:1079400000629A607B681B6899687B68DA687B686C
:107950001B680A439A607B689B6A584A934222D00C
:107960007B681B689A687B681B6822F070629A606B
:107970007B681B6899687B689A6A7B681B680A4306
:107980009A607B681B689A687B681B6822F040528B
:107990009A607B681B6899687B68DA6A7B681B68F9
:1079A0000A439A600FE07B681B689A687B681B68D3
:1079B00022F070629A607B681B689A687B681B681B
:1079C00022F040529A607B681B689A687B681B684B
:1079D00022F002029A607B681B6899687B689B6949
:1079E0005A007B681B680A439A607B6893F82030D2
:1079F000002B1BD07B681B685A687B681B6842F4AD
:107A000000625A607B681B685A687B681B6822F4B6
:107A100060425A607B681B6859687B685B6A013BFF
:107A20005A037B681B680A435A6007E07B681B683F
:107A30005A687B681B6822F400625A607B681B6886
:107A4000DA6A7B681B6822F47002DA627B681B6862
:107A5000D96A7B68DB69013B1A057B681B680A43AE
:107A6000DA627B681B689A687B681B6822F4007284
:107A70009A607B681B6899687B6893F830305A027B
:107A80007B681B680A439A607B681B689A687B68FE
:107A90001B6822F480629A607B681B6899687B6827
:107AA0005B699A027B681B680A439A6000BF0C37C7
:107AB000BD465DF8047B7047002301400100000FC4
:107AC00080B584B000AF78607B68002B01D10123C2
:107AD000EDE07B6893F82030DBB2002B02D17868B0
:107AE00009F088FA7B681B681A687B681B6842F09B
:107AF00001021A60FFF75EFBF86012E0FFF75AFB25
:107B00000246FB68D31A0A2B0BD97B685B6A43F4E5
:107B100000327B685A627B68052283F820200123AB
:107B2000C5E07B681B685B6803F00103002BE5D0B0
:107B30007B681B681A687B681B6822F002021A6067
:107B4000FFF738FBF86012E0FFF734FB0246FB68F2
:107B5000D31A0A2B0BD97B685B6A43F400327B682B
:107B60005A627B68052283F8202001239FE07B680E
:107B70001B685B6803F00203002BE5D17B681B7E6A
:107B8000012B08D17B681B681A687B681B6842F070
:107B900080021A6007E07B681B681A687B681B68B4
:107BA00022F080021A607B685B7E012B08D17B6823
:107BB0001B681A687B681B6842F040021A6007E085
:107BC0007B681B681A687B681B6822F040021A6099
:107BD0007B689B7E012B08D17B681B681A687B68D9
:107BE0001B6842F020021A6007E07B681B681A6875
:107BF0007B681B6822F020021A607B68DB7E012B09
:107C000008D17B681B681A687B681B6822F0100229
:107C10001A6007E07B681B681A687B681B6842F083
:107C200010021A607B681B7F012B08D17B681B68E0
:107C30001A687B681B6842F008021A6007E07B68DC
:107C40001B681A687B681B6822F008021A607B6850
:107C50005B7F012B08D17B681B681A687B681B68F7
:107C600042F004021A6007E07B681B681A687B68B0
:107C70001B6822F004021A607B689A687B68DB68E4
:107C80001A437B681B691A437B685B6942EA0301FC
:107C90007B685B685A1E7B681B680A43DA617B68F5
:107CA00000225A627B68012283F8202000231846B4
:107CB0001037BD4680BD000080B487B000AF78604B
:107CC00039607B6893F82030FB74FB7C012B03D078
:107CD000FB7C022B40F0CB807B681B686A4A934296
:107CE00003D17B681B687B6101E0684B7B617B692A
:107CF000D3F8003243F001027B69C3F800227B69AC
:107D0000624A934211D17B69D3F8003223F47C524A
:107D10007B69C3F800227B69D3F800223B685B6A69
:107D20001B021A437B69C3F800223B685B6903F0BE
:107D30001F03012202FA03F3FB607B69D3F81C22C4
:107D4000FB68DB431A407B69C3F81C223B68DB6994
:107D5000002B23D17B69D3F80C22FB68DB431A404C
:107D60007B69C3F80C223B68DB6819043B685B68DD
:107D70009BB23A68526919437B69483243F8321022
:107D80003B689B6819043B681B689AB23B685B6957
:107D90000A4379694833DB000B445A603B68DB696E
:107DA000012B22D17B69D3F80C22FB681A437B6933
:107DB000C3F80C223B681B6819043B685B689BB2E4
:107DC0003A68526919437B69483243F832103B687C
:107DD0009B6819043B68DB689AB23B685B690A439D
:107DE00079694833DB000B445A603B689B69002B80
:107DF00009D17B69D3F80422FB68DB431A407B6915
:107E0000C3F8042207E07B69D3F80422FB681A4315
:107E10007B69C3F804223B681B69002B09D17B698D
:107E2000D3F81422FB68DB431A407B69C3F81422A1
:107E300007E07B69D3F81422FB681A437B69C3F817
:107E400014223B681B6A012B07D17B69D3F81C22E3
:107E5000FB681A437B69C3F81C227B69D3F80032A4
:107E600023F001027B69C3F80022002306E07B684F
:107E70005B6A43F480227B685A62012318461C37F0
:107E8000BD465DF8047B704700340040006400404C
:107E900080B584B000AF78607B6893F82030DBB2A7
:107EA000012B2ED17B68022283F820207B681B687F
:107EB0001A687B681B6822F001021A60FFF77AF9E2
:107EC000F86012E0FFF776F90246FB68D31A0A2B36
:107ED0000BD97B685B6A43F400327B685A627B682B
:107EE000052283F82020012312E07B681B685B6871
:107EF00003F00103002BE5D17B6800225A620023C6
:107F000006E07B685B6A43F400227B685A620123C7
:107F100018461037BD4680BD80B489B000AFF86008
:107F2000B9607A603B60FB6893F82030FB77FB68B0
:107F30001B689B68BB61FB7F012B03D0FB7F022B7F
:107F400040F0AD80BB6903F08063002B0AD1BB69B0
:107F500003F00063002B05D1BB6903F08053002BB5
:107F600000F09580BB691B0E03F003037B610122C7
:107F70007B699A403B681A60BB689B68002B0DD1F7
:107F8000BB681B685A05BB68DB68F96809681A4357
:107F90007B6918331B010B441A600FE0BB685B68F8
:107FA000DA00BB689B681A43BB68DB68F96809683C
:107FB0001A437B6918331B010B441A60FB6819686C
:107FC000BB681A697B6918331B010B4404331A60C0
:107FD000BB681B7D012B11D1FB681A687B691833C4
:107FE0001B01134404331B68FA68116843F4807260
:107FF0007B6918331B010B4404331A607B68073319
:108000001B781A067B6806331B781B041A437B68AF
:1080100005331B781B0213437A680432127810462A
:10802000FA68116843EA00027B691B010B4403F5FF
:10803000C6731A607B6803331B781A067B680233A9
:108040001B781B041A437B6801331B781B02134304
:108050007A6812781046FA68116843EA00027B6970
:108060001B010B4403F5C4731A60FB681A687B6933
:1080700018331B0113441B68FA68116843F00102AE
:108080007B6918331B010B441A6000230EE0FB6868
:108090005B6A43F40012FB685A62012306E0FB6846
:1080A0005B6A43F48022FB685A6201231846243736
:1080B000BD465DF8047B704780B485B000AF786042
:1080C0000023FB607B6893F82030FB72FB7A012B66
:1080D00002D0FB7A022B1DD17B681B689B6803F0E2
:1080E0008063002B02D0FB680133FB607B681B6858
:1080F0009B6803F00063002B02D0FB680133FB6038
:108100007B681B689B6803F08053002B02D0FB68E0
:108110000133FB60FB6818461437BD465DF8047BED
:10812000704780B487B000AFF860B9607A603B6098
:10813000FB6893F82030FB75FB7D012B03D0FB7DA2
:10814000022B40F00381BB68002B0ED1FB681B683B
:10815000DB6803F00303002B16D1FB685B6A43F472
:108160000012FB685A620123F7E0FB681B681B6979
:1081700003F00303002B07D1FB685B6A43F4001292
:10818000FB685A620123E8E0FB681A68BB681B338E
:108190001B0113441B6803F004027B689A607B6830
:1081A0009B68002B0CD1FB681A68BB681B331B0152
:1081B00013441B685B0DC3F30A027B681A600BE073
:1081C000FB681A68BB681B331B0113441B68DB0880
:1081D00023F060427B685A60FB681A68BB681B33F7
:1081E0001B0113441B6803F002027B68DA60FB6822
:1081F0001A68BB681B331B01134404331B6803F06C
:108200000803002B03D07B6808221A610BE0FB688F
:108210001A68BB681B331B01134404331B6803F04B
:108220000F027B681A61FB681A68BB681B331B016D
:10823000134404331B681B0ADAB27B689A61FB683B
:108240001A68BB681B331B01134404331B681B0CE7
:108250009AB27B685A61FB681A68BB681B011344B9
:1082600003F5DC731B68DAB23B681A70FB681A68A6
:10827000BB681B01134403F5DC731B681A0A3B68D7
:108280000133D2B21A70FB681A68BB681B01134431
:1082900003F5DC731B681A0C3B680233D2B21A7008
:1082A000FB681A68BB681B01134403F5DC731B6889
:1082B0001A0E3B680333D2B21A70FB681A68BB68A7
:1082C0001B01134403F5DE731A683B680433D2B212
:1082D0001A70FB681A68BB681B01134403F5DE7350
:1082E0001B681A0A3B680533D2B21A70FB681A6819
:1082F000BB681B01134403F5DE731B681A0C3B6853
:108300000633D2B21A70FB681A68BB681B011344AB
:1083100003F5DE731B681A0E3B680733D2B21A707E
:10832000BB68002B08D1FB681B68DA68FB681B6818
:1083300042F02002DA6007E0FB681B681A69FB68FC
:108340001B6842F020021A61002306E0FB685B6AAA
:1083500043F48022FB685A62012318461C37BD464D
:108360005DF8047B704780B485B000AF78603960F9
:108370007B6893F82030FB73FB7B012B02D0FB7BE7
:10838000022B09D17B681B6859697B681B683A68B6
:108390000A435A61002306E07B685B6A43F480224B
:1083A0007B685A62012318461437BD465DF8047B8A
:1083B000704780B58AB000AF786000237B627B682D
:1083C0001B685B693B627B681B685B68FB617B6861
:1083D0001B689B68BB617B681B68DB687B617B6893
:1083E0001B681B693B617B681B689B69FB603B6A80
:1083F00003F00103002B7CD0BB6903F00103002BC9
:1084000023D07B681B6801229A60BB6903F00203DA
:10841000002B03D0786800F083F916E0BB6903F005
:108420000403002B04D07B6A43F400637B620CE0FE
:10843000BB6903F00803002B04D07B6A43F480532C
:108440007B6202E0786800F089F9BB6903F480730D
:10845000002B24D07B681B684FF480729A60BB6944
:1084600003F40073002B03D0786800F063F916E082
:10847000BB6903F48063002B04D07B6A43F4005390
:108480007B620CE0BB6903F40063002B04D07B6AC1
:1084900043F480437B6202E0786800F069F9BB69CD
:1084A00003F48033002B24D07B681B684FF48032A8
:1084B0009A60BB6903F40033002B03D0786800F0A6
:1084C00043F916E0BB6903F48023002B04D07B6AD8
:1084D00043F400437B620CE0BB6903F40023002BF0
:1084E00004D07B6A43F480337B6202E0786800F05A
:1084F00049F93B6A03F00803002B0CD07B6903F0B9
:108500001003002B07D07B6A43F400737B627B6807
:108510001B681022DA603B6A03F00403002B0BD0C7
:108520007B6903F00803002B06D07B681B680822D8
:10853000DA60786800F030F93B6A03F00203002B40
:1085400009D07B681B68DB6803F00303002B02D0B3
:10855000786808F08BFC3B6A03F04003002B0CD0DA
:108560003B6903F01003002B07D07B6A43F4806360
:108570007B627B681B6810221A613B6A03F0200350
:10858000002B0BD03B6903F00803002B06D07B685F
:108590001B6808221A61786800F012F93B6A03F040
:1085A0001003002B09D07B681B681B6903F00303D1
:1085B000002B02D0786800F0F9F83B6A03F400332E
:1085C000002B0BD0FB6903F01003002B06D07B6857
:1085D0001B6810225A60786800F0FCF83B6A03F4CC
:1085E0008033002B0BD0FB6903F00803002B06D06F
:1085F0007B681B6808225A60786800F0F5F83B6ACF
:1086000003F40043002B7BD0FB6903F00403002B31
:1086100072D03B6A03F48073002B08D0FB6803F030
:108620000103002B03D07B6A43F001037B623B6AAA
:1086300003F40073002B08D0FB6803F00203002B47
:1086400003D07B6A43F002037B623B6A03F48063DE
:10865000002B08D0FB6803F00403002B03D07B6AD7
:1086600043F004037B623B6A03F40063002B43D0B6
:10867000FB6803F07003002B3ED0FB6803F070032F
:10868000602B2BD0602B2ED8502B22D0502B2AD8E9
:10869000402B19D0402B26D8302B10D0302B22D88D
:1086A000102B02D0202B05D01DE07B6A43F008037D
:1086B0007B6219E07B6A43F010037B6214E07B6A03
:1086C00043F020037B620FE07B6A43F040037B6250
:1086D0000AE07B6A43F080037B6205E07B6A43F437
:1086E00080737B6200E000BF7B681B689A697B68CF
:1086F0001B6822F070029A617B681B6804225A6032
:108700007B6A002B08D07B685A6A7B6A1A437B68B5
:108710005A62786808F0B5FB00BF2837BD4680BDB7
:1087200080B483B000AF786000BF0C37BD465DF801
:10873000047B704780B483B000AF786000BF0C3713
:10874000BD465DF8047B704780B483B000AF7860AD
:1087500000BF0C37BD465DF8047B704780B483B022
:1087600000AF786000BF0C37BD465DF8047B7047F2
:1087700080B483B000AF786000BF0C37BD465DF8B1
:10878000047B704780B483B000AF786000BF0C37C3
:10879000BD465DF8047B704780B483B000AF78605D
:1087A00000BF0C37BD465DF8047B704780B483B0D2
:1087B00000AF786000BF0C37BD465DF8047B7047A2
:1087C00080B483B000AF786000BF0C37BD465DF861
:1087D000047B704780B483B000AF786000BF0C3773
:1087E000BD465DF8047B704780B483B000AF78600D
:1087F00000BF0C37BD465DF8047B704780B483B082
:1088000000AF78607B685B6A18460C37BD465DF840
:10881000047B704780B584B000AF78607B68002B24
:1088200001D1012371E07B685B7FDBB2002B05D1B6
:108830007B6800221A77786808F046FC7B68022281
:108840005A777B681B68DB6803F01003102B53D04A
:108850007B681B68CA225A627B681B6853225A6273
:10886000786800F07FF80346FB73FB7B002B2AD16E
:108870007B681B6899687B681A68264B0B4093607D
:108880007B681B6899687B685A687B681B691A4318
:108890007B685B691A437B681B680A439A607B6844
:1088A0001B687A68D2681A617B681B6819697B68E3
:1088B0009B681A047B681B680A431A61786800F099
:1088C00088F80346FB73FB7B002B10D17B681B6889
:1088D000DA6C7B681B6822F00802DA647B681B682C
:1088E000D96C7B689A697B681B680A43DA647B6889
:1088F0001B68FF225A6201E00023FB73FB7B002B05
:1089000002D17B6801225A77FB7B18461037BD469F
:1089100080BD00BFBFFF8FFF80B584B000AF78601F
:108920000023FB607B681B680D4ADA60FEF742FC9F
:10893000F86009E0FEF73EFC0246FB68D31AB3F587
:108940007A7F01D9032307E07B681B68DB6803F0AB
:108950002003002BEED0002318461037BD4680BD03
:108960005FFF010080B584B000AF78600023BB607A
:108970000023FB737B681B68DB6803F04003002B5C
:1089800022D17B681B68DA687B681B6842F0800232
:10899000DA60FEF70FFCB8600CE0FEF70BFC024655
:1089A000BB68D31AB3F57A7F04D97B6804225A775F
:1089B0000123FB737B681B68DB6803F04003002B1B
:1089C00002D1FB7B012BE8D1FB7B18461037BD465B
:1089D00080BD80B584B000AF78600023FB737B68F6
:1089E0001B68DA687B681B6822F08002DA607B68AB
:1089F0001B689B6803F02003002B0AD17868FFF7FF
:108A00008BFF0346002B04D07B6804225A77012396
:108A1000FB73FB7B18461037BD4680BD80B586B022
:108A200000AFF860B9601346FB71FB68002B01D101
:108A300003231FE0FB680022C3F8B822FB68002272
:108A4000C3F8C422FB680022C3F8D022BB68002B05
:108A500003D0FB68BA68C3F8B422FB68012283F82C
:108A60009C22FB68FA791A70F86805F0F1FC03465D
:108A7000FB75FB7D18461837BD4680BD80B584B0B8
:108A800000AF786039600023FB813B68002B01D187
:108A9000032325E07B683A68C3F8B8227B68D3F8E3
:108AA000D4227B68AE3253F82230DB6A002B0FD021
:108AB0007B68D3F8D4227B68AE3253F82230DB6A6D
:108AC00007F10E021046984702467B68C3F8D02291
:108AD0007B68D3F8D8325A1C7B68C3F8D8220023AD
:108AE00018461037BD4680BD80B582B000AF7860B3
:108AF000786805F0F9FC034618460837BD4680BD86
:108B000080B483B000AF7860002318460C37BD46B0
:108B10005DF8047B704780B584B000AF78600B4689
:108B2000FB700023FB737B68D3F8B832002B09D0AD
:108B30007B68D3F8B8321B68FA7811467868984792
:108B40000346FB73FB7B18461037BD4680BD80B5DE
:108B500084B000AF78600B46FB700023FB737B682A
:108B6000D3F8B8325B68FA781146786898470346BC
:108B7000002B01D00323FB73FB7B18461037BD4647
:108B800080BD80B584B000AF786039607B6803F247
:108B9000AA233968184601F04CF97B680122C3F812
:108BA00094227B68B3F8B0321A467B68C3F89822E7
:108BB0007B6893F8AA3203F01F03022B1AD0022B12
:108BC00022D8002B02D0012B0AD01DE07B6803F2D3
:108BD000AA231946786800F077FB0346FB7320E070
:108BE0007B6803F2AA231946786800F0DFFB03468E
:108BF000FB7316E07B6803F2AA231946786800F03D
:108C000041FC0346FB730CE07B6893F8AA3223F027
:108C10007F03DBB21946786805F0C6FC0346FB7398
:108C200000BFFB7B18461037BD4680BD80B586B0BF
:108C300000AFF8600B467A60FB720023FB75FB7A8D
:108C4000002B77D1FB6803F5AA733B61FB68D3F86F
:108C50009432032B40F0A1803B695B683A699289AA
:108C600093421CD93B695B683A6992899A1A3B69BD
:108C70005A603B691B693A6992891A443B691A61D7
:108C80003B6919693B699B891A463B695B6893425A
:108C900038BF13461A46F86801F0D2F97DE0FB6848
:108CA00093F8AA3203F01F03022B14D0022B1DD815
:108CB000002B02D0012B03D018E00023BB7518E075
:108CC000FB68B3F8AE32DBB21946F86800F06EFA12
:108CD0000346BB750DE0FB68B3F8AE32DBB2194654
:108CE000F86800F070FA0346BB7502E00023BB751C
:108CF00000BFBB7D002B19D1FB6893F89C32DBB21F
:108D0000032B13D1BA7DFB68AE3253F822301B69B6
:108D1000002B0BD0BA7DFB68C3F8D422BA7DFB6868
:108D2000AE3253F822301B69F8689847F86801F0B2
:108D300098F932E0FB7A03F07F03DBB21946F8685A
:108D400000F041FA0346BB75BB7DFF2B25D0BB7DF0
:108D5000002B22D1FB6893F89C32DBB2032B17D196
:108D6000BA7DFB68AE3253F822309B69002B0FD0DE
:108D7000BA7DFB68C3F8D422BA7DFB68AE3253F8E3
:108D800022309B69FA7A1146F86898470346FB75CA
:108D9000FB7D002B01D0FB7D00E000231846183737
:108DA000BD4680BD80B586B000AFF8600B467A60E6
:108DB000FB72FB7A002B78D1FB6814333B61FB68B4
:108DC000D3F89432022B63D13B695B683A6992898C
:108DD00093421CD93B695B683A6992899A1A3B694C
:108DE0005A603B691B693A6992891A443B691A6166
:108DF0003B6919693B695B681A46F86801F0EEF84F
:108E0000002300220021F86805F078FC40E03B696F
:108E10009B891A463B695B689A421CD13B691B6877
:108E20003A699289934216D33B691A68FB68D3F872
:108E300098329A420FD200220021F86801F0CEF851
:108E4000FB680022C3F89822002300220021F86862
:108E500005F054FC1CE0FB6893F89C32DBB2032B5A
:108E60000FD1FB68D3F8B832DB68002B09D0FB6860
:108E70000022C3F8D422FB68D3F8B832DB68F86864
:108E800098478021F86805F08FFBF86801F0FCF83E
:108E9000FB6893F8A032002B3AD0F868FFF730FE59
:108EA000FB68002283F8A02232E0FB7A63F07F03A4
:108EB000DBB21946F86800F086F90346FB75FB7DC6
:108EC000FF2B25D0FB7D002B22D1FB6893F89C3231
:108ED000DBB2032B1CD1FA7DFB68AE3253F8223093
:108EE0005B69002B14D0FA7DFB68C3F8D422FA7DAD
:108EF000FB68AE3253F822305B69FA7A1146F868A3
:108F000098470346BB75BB7D002B01D0BB7D00E0BD
:108F1000002318461837BD4680BD80B584B000AF29
:108F200078600023FB737B68012283F89C227B68B6
:108F30000022C3F894227B6800225A607B680022DA
:108F4000C3F8A4227B68002283F8A0227B68D3F8B0
:108F5000B832002B14D07B68D3F8B8325B68002B92
:108F60000ED07B68D3F8B8325B687A685268D2B2A8
:108F70001146786898470346002B01D00323FB7302
:108F8000402300220021786805F0C9FA7B6801229D
:108F900083F863217B684022A3F8602140230022EC
:108FA0008021786805F0BBFA7B68012283F82320D2
:108FB0007B6840221A84FB7B18461037BD4680BD73
:108FC00080B483B000AF78600B46FB707B68FA78A2
:108FD0001A74002318460C37BD465DF8047B7047B1
:108FE00080B483B000AF78607B6893F89C32DBB2CA
:108FF000042B06D07B6893F89C32DAB27B6883F846
:109000009D227B68042283F89C22002318460C379B
:10901000BD465DF8047B704780B483B000AF7860D4
:109020007B6893F89C32DBB2042B06D17B6893F803
:109030009D32DAB27B6883F89C22002318460C37F5
:10904000BD465DF8047B704780B582B000AF7860A4
:109050007B6893F89C32DBB2032B10D17B68D3F88A
:10906000B832002B0BD07B68D3F8B832DB69002B09
:1090700005D07B68D3F8B832DB697868984700235D
:1090800018460837BD4680BD80B582B000AF786015
:109090000B46FB707B68D3F8D4227B68AE3253F862
:1090A0002230002B01D103231CE07B6893F89C3213
:1090B000DBB2032B15D17B68D3F8D4227B68AE32A8
:1090C00053F822301B6A002B0BD07B68D3F8D422D4
:1090D0007B68AE3253F822301B6AFA781146786802
:1090E0009847002318460837BD4680BD80B582B03A
:1090F00000AF78600B46FB707B68D3F8D4227B68A6
:10910000AE3253F82230002B01D103231CE07B68E0
:1091100093F89C32DBB2032B15D17B68D3F8D422B1
:109120007B68AE3253F822305B6A002B0BD07B6831
:10913000D3F8D4227B68AE3253F822305B6AFA78D7
:10914000114678689847002318460837BD4680BD09
:1091500080B483B000AF7860002318460C37BD465A
:109160005DF8047B704780B584B000AF7860002361
:10917000FB737B68012283F89C227B68D3F8B832AA
:10918000002B0ED07B68D3F8B8325B687A685268DF
:10919000D2B21146786898470346002B01D00323CA
:1091A000FB73FB7B18461037BD4680BD80B483B08F
:1091B00000AF78600B46FB70002318460C37BD46A5
:1091C0005DF8047B704780B483B000AF78600B46D5
:1091D000FB70002318460C37BD465DF8047B7047D2
:1091E00080B586B000AF78600B46FB707B687B6112
:1091F0007B68FB6000233B61FB685B889BB2FA687D
:10920000127893421FD9FB681B787B8113E007F12A
:109210000A031946786900F01BF878617B695B786E
:10922000052B08D17B693B613B699B78FA789A42B0
:1092300008D000233B61FB685B889AB27B899A4225
:10924000E5D800E000BF3B6918461837BD4680BD31
:1092500080B485B000AF786039607B68FB603B68A4
:109260001B88FA68127813449AB23B681A80FB682C
:109270001B781A467B681344FB60FB68184614375A
:10928000BD465DF8047B704780B487B000AF78605E
:109290007B687B617B691B787B827B6901337B61A7
:1092A0007B691B783B82B7F910301B021AB2B7F901
:1092B000123013431BB2FB81FB8918461C37BD4695
:1092C0005DF8047B7047000080B584B000AF786023
:1092D00039600023FB733B681B7803F06003402B6D
:1092E00005D0402B57D8002B0FD0202B53D17B68B3
:1092F000D3F8D4227B68AE3253F822309B683968A9
:10930000786898470346FB734AE03B685B78092B13
:109310003BD801A252F823F06D9301088193010814
:109320008B930108779301088B9301084B930108F5
:10933000419301088B930108639301085593010839
:109340003968786800F03EFA24E03968786800F0FF
:10935000CDFB1FE03968786800F00CFC0346FB7316
:1093600018E03968786800F0AFFC13E03968786875
:1093700000F0E0FC0EE03968786800F00FFD09E0CD
:109380003968786800F033FD04E03968786800F0E7
:109390008AFD00BF04E03968786800F084FD00BFF2
:1093A000FB7B18461037BD4680BD00BF80B584B03A
:1093B00000AF786039600023FB733B681B7803F0D3
:1093C0006003402B05D0402B52D8002B01D0202B1E
:1093D0004ED17B6893F89C32DBB2013B022B40D824
:1093E0003B689B88DBB2012B36D83B689B88DBB29D
:1093F00019467868FFF7DAFE0346BB73BB7BFF2B89
:109400001DD0BB7B002B1AD1BA7B7B68AE3253F8E0
:1094100022309B68002B0FD0BA7B7B68C3F8D42224
:10942000BA7B7B68AE3253F822309B683968786823
:1094300098470346FB7304E00323FB7301E0032317
:10944000FB733B68DB88002B10D1FB7B002B0DD11D
:10945000786800F006FE09E03968786800F023FDBE
:1094600004E03968786800F01EFD00E000BF04E009
:109470003968786800F017FD00BFFB7B184610378D
:10948000BD4680BD80B584B000AF786039600023F0
:10949000FB733B689B88BB733B681B7803F06003DE
:1094A000402B07D0402B00F28181002B2AD0202BAB
:1094B00040F07C81BB7B19467868FFF784FE034649
:1094C0007B737B7BFF2B00F076817B7B002B40F056
:1094D00072817A7B7B68C3F8D4227A7B7B68AE3258
:1094E00053F822309B68002B00F065817A7B7B6803
:1094F000AE3253F822309B68396878689847034643
:10950000FB7358E13B685B78032B08D0032B00F317
:109510004781002B00F09B80012B3CD040E17B6811
:1095200093F89C32DBB2022B02D0032B16D02CE036
:10953000BB7B002B0DD0BB7B802B0AD0BB7B19469D
:10954000786805F031F88021786805F02DF800BFC3
:1095500020E03968786800F0A6FC1BE03B685B8877
:10956000002B0ED1BB7B002B0BD0BB7B802B08D0FC
:109570003B68DB88002B04D1BB7B1946786805F07B
:1095800013F8786800F06DFD04E03968786800F041
:109590008AFC00BF09E17B6893F89C32DBB2022BA6
:1095A00002D0032B16D04BE0BB7B002B0DD0BB7B36
:1095B000802B0AD0BB7B1946786804F0F5FF802128
:1095C000786804F0F1FF00BF40E03968786800F087
:1095D0006AFC3BE03B685B88002B36D1BB7B03F029
:1095E0007F03002B04D0BB7B1946786804F0FBFF97
:1095F000786800F036FDBB7B19467868FFF7E3FD1D
:1096000003467B737B7BFF2B1FD07B7B002B1CD106
:109610007A7B7B68C3F8D4227A7B7B68AE3253F8BE
:1096200022309B68002B10D07A7B7B68AE3253F8D7
:1096300022309B683968786898470346FB7304E0DA
:109640003968786800F02FFC00E000BFADE07B686F
:1096500093F89C32DBB2022B02D0032B33D099E07B
:10966000BB7B002B07D0BB7B802B04D0396878688C
:1096700000F019FC93E097F90E30002B0BDABB7B5E
:1096800003F07F0213469B0013449B0010337A685B
:10969000134404330BE0BB7B03F07F0213469B00B3
:1096A00013449B0003F5A8737A6813440433BB602A
:1096B000BB6800229A73BB680E3302221946786891
:1096C00000F06EFC6BE097F90E30002B11DABB7BDB
:1096D00003F00F02796813469B0013449B000B4470
:1096E00023331B78002B17D13968786800F0DBFB37
:1096F00055E0BB7B03F00F02796813469B001344CF
:109700009B000B4403F263131B78002B04D13968D0
:10971000786800F0C8FB42E097F90E30002B0BDAB6
:10972000BB7B03F07F0213469B0013449B00103366
:109730007A68134404330BE0BB7B03F07F021346CB
:109740009B0013449B0003F5A8737A681344043309
:10975000BB60BB7B002B02D0BB7B802B03D1BB68E3
:1097600000229A730EE0BB7B1946786804F05AFF1A
:109770000346002B03D0BB6801229A7302E0BB684A
:1097800000229A73BB680E3302221946786800F0F3
:1097900007FC04E03968786800F085FB00BF04E04E
:1097A0003968786800F07FFB00BF05E039687868A9
:1097B00000F079FB00E000BFFB7B18461037BD4688
:1097C00080BD000080B584B000AF786039600023B0
:1097D0003B810023FB600023FB723B685B881B0A14
:1097E0009BB2013B0E2B00F2528101A252F823F0F2
:1097F0006198010879980108B99801088F9A0108C1
:109800008F9A01082F9A01085B9A01088F9A010824
:109810008F9A01088F9A01088F9A01088F9A010880
:109820008F9A01088F9A01082D9801087B68D3F858
:10983000B432DB69002B0BD07B68D3F8B432DB6920
:109840007A68127C07F1080110469847F86026E113
:109850003968786800F027FBFB7A0133FB721EE160
:109860007B68D3F8B4321B687A68127C07F1080170
:1098700010469847F86012E17B681B7C002B0DD1E5
:109880007B68D3F8B8329B6A07F108021046984704
:10989000F860FB68013302221A7000E17B68D3F89C
:1098A000B832DB6A07F1080210469847F860FB6897
:1098B000013302221A70F2E03B685B88DBB2052BB1
:1098C00000F2AC8001A252F823F000BFE598010835
:1098D000199901084D99010881990108B599010864
:1098E000E99901087B68D3F8B4325B68002B0BD090
:1098F0007B68D3F8B4325B687A68127C07F10801A0
:1099000010469847F86091E03968786800F0CBFA23
:10991000FB7A0133FB7289E07B68D3F8B4329B6831
:10992000002B0BD07B68D3F8B4329B687A68127C2A
:1099300007F1080110469847F86077E039687868C1
:1099400000F0B1FAFB7A0133FB726FE07B68D3F869
:10995000B432DB68002B0BD07B68D3F8B432DB6801
:109960007A68127C07F1080110469847F8605DE0BC
:109970003968786800F097FAFB7A0133FB7255E09A
:109980007B68D3F8B4321B69002B0BD07B68D3F80B
:10999000B4321B697A68127C07F1080110469847B7
:1099A000F86043E03968786800F07DFAFB7A0133AB
:1099B000FB723BE07B68D3F8B4325B69002B0BD0C1
:1099C0007B68D3F8B4325B697A68127C07F10801CE
:1099D00010469847F86029E03968786800F063FA23
:1099E000FB7A0133FB7221E07B68D3F8B4329B69C8
:1099F000002B0BD07B68D3F8B4329B697A68127C59
:109A000007F1080110469847F8600FE03968786858
:109A100000F049FAFB7A0133FB7207E03968786895
:109A200000F041FAFB7A0133FB7200BF37E07B683C
:109A30001B7C002B09D17B68D3F8B8325B6B07F134
:109A4000080210469847F86029E03968786800F005
:109A50002AFAFB7A0133FB7221E07B681B7C002B26
:109A60000DD17B68D3F8B8321B6B07F108021046A2
:109A70009847F860FB68013307221A700FE03968D5
:109A8000786800F010FAFB7A0133FB7207E039685E
:109A9000786800F008FAFB7A0133FB7200BFFB7AAA
:109AA000002B1ED13B68DB88002B16D03B89002B96
:109AB0000ED03B68DA883B89934228BF13469BB29D
:109AC0003B813B891A46F968786800F069FA09E039
:109AD0003968786800F0E7F904E0786800F0C1FAC6
:109AE00000E000BF1037BD4680BD00BF80B584B028
:109AF00000AF786039603B689B88002B31D13B68B0
:109B0000DB88002B2DD13B685B887F2B29D83B68F5
:109B10005B88DBB203F07F03FB737B6893F89C32B6
:109B2000DBB2032B04D13968786800F0BCF91DE082
:109B30007B68FA7B83F89E22FB7B1946786804F0E9
:109B40009DFD786800F08DFAFB7B002B04D07B68CC
:109B5000022283F89C2209E07B68012283F89C2280
:109B600004E03968786800F09EF900BF00BF103744
:109B7000BD4680BD80B584B000AF786039600023F9
:109B8000FB733B685B88DAB24E4B1A704D4B1B7807
:109B9000012B05D93968786800F085F903238CE03A
:109BA0007B6893F89C32DBB2022B02D0032B29D0C6
:109BB00075E0444B1B78002B20D0424B1B781A4693
:109BC0007B685A603F4B1B7819467868FEF7A3FF05
:109BD0000346FB73FB7B002B08D03968786800F0E4
:109BE00062F97B68022283F89C2265E0786800F0C5
:109BF00038FA7B68032283F89C225DE0786800F0E5
:109C000030FA59E02F4B1B78002B12D17B680222CF
:109C100083F89C222B4B1B781A467B685A60294B91
:109C20001B7819467868FEF792FF786800F019FAF9
:109C300042E0244B1B781A467B685B689A422AD024
:109C40007B685B68DBB219467868FEF780FF1D4BC6
:109C50001B781A467B685A601A4B1B78194678683D
:109C6000FEF759FF0346FB73FB7B002B0FD03968CF
:109C7000786800F018F97B685B68DBB21946786891
:109C8000FEF765FF7B68022283F89C2214E0786867
:109C900000F0E7F910E0786800F0E3F90CE03968CB
:109CA000786800F000F9074B1B7819467868FEF7D2
:109CB0004EFF0323FB7300BFFB7B18461037BD46E6
:109CC00080BD00BFB403002080B582B000AF7860D3
:109CD00039603B68DB88012B04D03968786800F074
:109CE000E2F823E07B6893F89C32DBB2022B02DCC3
:109CF000002B03DC15E0032B0BD012E07B68002265
:109D00009A607B68083301221946786800F048F9A8
:109D10000CE07B68043301221946786800F040F9B2
:109D200004E03968786800F0BEF800BF00BF08376B
:109D3000BD4680BD80B582B000AF786039607B6879
:109D400093F89C32DBB2013B022B1ED83B68DB88C8
:109D5000022B04D03968786800F0A5F81AE07B6817
:109D60000122DA607B68D3F8A432002B05D07B682F
:109D7000DB6843F002027B68DA607B680C33022206
:109D80001946786800F00CF904E03968786800F04A
:109D90008AF800BF00BF0837BD4680BD80B582B0DD
:109DA00000AF786039603B685B88012B07D17B6826
:109DB0000122C3F8A422786800F053F913E03B684D
:109DC0005B88022B0BD13B689B881B0A9BB2DAB2E3
:109DD0007B6883F8A022786800F043F903E03968D3
:109DE000786800F060F800BF0837BD4680BD80B5D8
:109DF00082B000AF786039607B6893F89C32DBB248
:109E0000013B022B0BD83B685B88012B0CD17B6894
:109E10000022C3F8A422786800F023F904E039682E
:109E2000786800F040F800E000BF00BF0837BD468A
:109E300080BD80B584B000AF786039603B68FB605E
:109E4000FB681A787B681A70FB680133FB60FB685B
:109E50001A787B685A70FB680133FB60F868FFF77B
:109E600013FA03461A467B685A80FB680133FB608D
:109E7000FB680133FB60F868FFF706FA03461A46F1
:109E80007B689A80FB680133FB60FB680133FB60F1
:109E9000F868FFF7F9F903461A467B68DA8000BFD5
:109EA0001037BD4680BD80B582B000AF78603960A4
:109EB0008021786804F078FB0021786804F074FB56
:109EC00000BF0837BD4680BD80B586B000AFF860E2
:109ED000B9607A600023FB75FB68002B42D0FB68F9
:109EE0003B61386900F042F8034601335B00B3F58B
:109EF000007F08D8386900F039F8034601339BB277
:109F00005B009AB201E04FF400727B681A80FB7D1F
:109F1000BA6813447A6812781A70FB7D0133FB75B6
:109F2000FB7DBA68134403221A70FB7D0133FB7575
:109F300013E0FB7DBA6813443A6912781A703B69E2
:109F400001333B61FB7D0133FB75FB7DBA68134434
:109F500000221A70FB7D0133FB753B691B78002BD7
:109F6000E7D100E000BF1837BD4680BD80B485B0A2
:109F700000AF78600023FB737B68BB6005E0FB7B70
:109F80000133FB73BB680133BB60BB681B78002BDC
:109F9000F5D1FB7B18461437BD465DF8047B70474E
:109FA00080B584B000AFF860B9607A60FB680222C7
:109FB000C3F89422FB687A685A61FB68BA685A62EF
:109FC000FB687A689A617B68BA680021F86804F0D7
:109FD00074FB002318461037BD4680BD80B584B0A1
:109FE00000AFF860B9607A607B68BA680021F868F1
:109FF00004F063FB002318461037BD4680BD80B5D2
:10A0000084B000AFF860B9607A60FB680322C3F8DF
:10A010009422FB687A68C3F85421FB68BA68C3F8D5
:10A020006421FB687A68C3F858217B68BA6800210C
:10A03000F86804F063FB002318461037BD4680BD66
:10A0400080B584B000AFF860B9607A607B68BA68A8
:10A050000021F86804F052FB002318461037BD4673
:10A0600080BD80B582B000AF78607B680422C3F801
:10A070009422002300220021786804F01EFB0023B4
:10A0800018460837BD4680BD80B582B000AF786005
:10A090007B680522C3F894220023002200217868FF
:10A0A00004F02CFB002318460837BD4680BD000095
:10A0B00080B584B000AF78600B46FB704FF407703A
:10A0C00019F06AFA0346FB60FB68002B09D17B6834
:10A0D000D3F8D4227B68B032002143F82210022347
:10A0E000D4E04FF407720021F8681BF065F97B6833
:10A0F000D3F8D4227B68B032F96843F822107B6829
:10A10000D3F8D4227B68B03253F822207B68C3F89E
:10A11000BC227B681B7C002B38D15E4B19784FF436
:10A1200000730222786804F0FAF95A4B1B7803F0A6
:10A130000F02796813469B0013449B000B442333A2
:10A1400001221A70544B19784FF400730222786878
:10A1500004F0E5F9504B1B7803F00F0279681346C1
:10A160009B0013449B000B4403F2631301221A70FB
:10A170004A4B1B7803F00F02796813469B00134487
:10A180009B000B441C3310221A6035E0414B1978B8
:10A1900040230222786804F0C2F93E4B1B7803F09A
:10A1A0000F02796813469B0013449B000B44233332
:10A1B00001221A70384B197840230222786804F083
:10A1C000AEF9354B1B7803F00F02796813469B00FC
:10A1D00013449B000B4403F2631301221A702F4BAC
:10A1E0001B7803F00F02796813469B0013449B0011
:10A1F0000B441C3310221A60284B197808230322C1
:10A20000786804F08CF9254B1B7803F00F0279680D
:10A2100013469B0013449B000B44233301221A7006
:10A22000FB680022C3F804227B68D3F8D4327A6832
:10A23000B0339B0013445B681B689847FB6800229F
:10A24000C3F81422FB680022C3F81822FB68D3F875
:10A250000432002B01D1022318E07B681B7C002B09
:10A260000AD10D4B1978FB68D3F804224FF4007320
:10A27000786804F043FA08E0074B1978FB68D3F8D4
:10A2800004224023786804F039FA00231846103776
:10A29000BD4680BD93000020940000209500002062
:10A2A00080B582B000AF78600B46FB703A4B1B78EC
:10A2B0001946786804F059F9374B1B7803F00F0200
:10A2C000796813469B0013449B000B442333002200
:10A2D0001A70324B1B781946786804F046F92F4BF8
:10A2E0001B7803F00F02796813469B0013449B0010
:10A2F0000B4403F2631300221A70294B1B78194692
:10A30000786804F032F9264B1B7803F00F02796865
:10A3100013469B0013449B000B44233300221A7006
:10A320001F4B1B7803F00F02796813469B00134400
:10A330009B000B441C3300221A607B68D3F8D422A4
:10A340007B68B03253F82230002B1FD07B68D3F8E3
:10A35000D4327A68B0339B0013445B685B689847DB
:10A360007B68D3F8D4227B68B03253F82230184689
:10A3700019F01AF97B68D3F8D4227B68B032002137
:10A3800043F822107B680022C3F8BC220023184641
:10A390000837BD4680BD00BF930000209400002018
:10A3A0009500002080B586B000AF786039607B688A
:10A3B000D3F8D4227B68B03253F822303B610023BB
:10A3C0007B7300237B810023FB753B69002B01D14C
:10A3D0000323BFE03B681B7803F06003002B50D0E1
:10A3E000202B40F0AF803B68DB88002B3AD03B68E5
:10A3F0001B785BB2002B1BDA7B68D3F8D4327A6807
:10A40000B0339B0013445B689B683A6850783969A5
:10A410003A68D28898473B68DB88072B28BF072318
:10A42000FB813B69FA8919467868FFF7B9FD90E02E
:10A430003B685A783B6983F800223B68DB883F2BF6
:10A4400003D83B68DB88DAB200E040223B6983F83E
:10A45000012239693B6993F801321A467868FFF79F
:10A46000CEFD76E07B68D3F8D4327A68B0339B00B7
:10A4700013445B689B683A685078002239689847B3
:10A4800067E03B685B780B2B51D801A252F823F0B0
:10A49000C1A401083DA501082FA501082FA50108A9
:10A4A0002FA501082FA501082FA501082FA5010838
:10A4B0002FA501082FA50108EBA4010815A5010887
:10A4C0007B6893F89C32DBB2032B07D107F10A03B8
:10A4D000022219467868FFF763FD32E03968786830
:10A4E000FFF7E1FC0323FB752BE07B6893F89C32BC
:10A4F000DBB2032B07D107F10D030122194678685F
:10A50000FFF74EFD1DE039687868FFF7CCFC0323A8
:10A51000FB7516E07B6893F89C32DBB2032B0FD0FF
:10A5200039687868FFF7BFFC0323FB7508E03968DA
:10A530007868FFF7B8FC0323FB7502E000BF08E072
:10A5400000BF06E039687868FFF7ADFC0323FB75B0
:10A5500000BFFB7D18461837BD4680BD80B584B06E
:10A5600000AF78600B46FB707B68D3F8C832FB60A5
:10A570007B68D3F8D4227B68B03253F82230002BAA
:10A5800001D1032365E07B68D3F8D4227B68B03225
:10A5900053F82230BB60FB7803F00F027968134652
:10A5A0009B0013449B000B4414331B68002B2FD0DB
:10A5B000FB7803F00F02796813469B0013449B005D
:10A5C0000B4414331A68FB7803F00F01F8680B464C
:10A5D000DB000B449B0003441C331B68B2FBF3F10C
:10A5E00001FB03F3D31A002B12D1FB7803F00F0207
:10A5F000796813469B0013449B000B4414330022DC
:10A600001A60F97800230022786804F056F81FE0F9
:10A61000BB680022C3F814227B68D3F8D4327A686E
:10A62000B0339B0013445B681B69002B10D07B6820
:10A63000D3F8D4327A68B0339B0013445B681B694B
:10A64000BA68D2F80802BA6802F50471FA78984735
:10A65000002318461037BD4680BD80B584B000AFDA
:10A6600078600B46FB707B68D3F8D4227B68B032ED
:10A6700053F82230FB607B68D3F8D4227B68B03279
:10A6800053F82230002B01D103231AE0FB7819463E
:10A69000786804F054F80246FB68C3F80C227B6823
:10A6A000D3F8D4327A68B0339B0013445B68DB681C
:10A6B000FA68D2F80402FA6802F503721146984764
:10A6C000002318461037BD4680BD80B584B000AF6A
:10A6D00078607B68D3F8D4227B68B03253F822309C
:10A6E000FB60FB68002B01D1032324E07B68D3F8D7
:10A6F000D4327A68B0339B0013445B68002B19D0C6
:10A70000FB6893F80032FF2B14D07B68D3F8D43267
:10A710007A68B0339B0013445B689B68FA6892F8D0
:10A720000002F968FA6892F801229847FB68FF2254
:10A7300083F80022002318461037BD4680BD000074
:10A7400080B586B000AF786082211848FEF748FDDA
:10A75000786101211548FEF743FD386181211348D6
:10A76000FEF73EFDF8607B69002B02D07B6910226A
:10A770009A713B69002B06D03B69002242F04002EF
:10A780001A7100225A71FB68002B06D0FB68002268
:10A7900042F040021A7100225A717B6843221A80EB
:10A7A000024B18461837BD4680BD00BF5000002040
:10A7B00080B586B000AF786082211848FEF710FDA2
:10A7C000786101211548FEF70BFD3861812113489E
:10A7D000FEF706FDF8607B69002B02D07B69102232
:10A7E0009A713B69002B06D03B6900221A71002246
:10A7F00042F002025A71FB68002B06D0FB6800226F
:10A800001A71002242F002025A717B6843221A80B8
:10A81000024B18461837BD4680BD00BF50000020CF
:10A8200080B586B000AF786082211848FEF7D8FC6A
:10A83000786101211548FEF7D3FC38618121134866
:10A84000FEF7CEFCF8607B69002B02D07B691022FA
:10A850009A713B69002B06D03B69002242F040020E
:10A860001A7100225A71FB68002B06D0FB68002287
:10A8700042F040021A7100225A717B6843221A800A
:10A88000024B18461837BD4680BD00BF500000205F
:10A8900080B483B000AF78607B680A221A80034BD3
:10A8A00018460C37BD465DF8047B70470C0000204D
:10A8B00080B483B000AF786039603B68002B01D171
:10A8C000032309E07B68D3F8D4327A68B0339B0065
:10A8D00013443A685A60002318460C37BD465DF8A9
:10A8E000047B704780B487B000AFF860B9607A60CD
:10A8F000FB68D3F8D422FB68B03253F822307B6176
:10A900007B69002B01D1032308E07B69BA68C3F897
:10A9100008227B697A68C3F81022002318461C3786
:10A92000BD465DF8047B704780B485B000AF7860A9
:10A9300039607B68D3F8D4227B68B03253F8223078
:10A94000FB60FB68002B01D1032304E0FB683A683D
:10A95000C3F80422002318461437BD465DF8047B73
:10A960007047000080B584B000AF78607B68D3F892
:10A97000D4227B68B03253F82230BB600123FB73D2
:10A98000BB68002B01D1032325E0BB68D3F8143248
:10A99000002B1FD1BB680122C3F81422104B1B7877
:10A9A00003F00F02BB68D3F81012786813469B00BF
:10A9B00013449B00034414331960094B1978BB6896
:10A9C000D3F80822BB68D3F81032786803F075FE1C
:10A9D0000023FB73FB7B18461037BD4680BD00BFCC
:10A9E0009300002080B584B000AF78607B68D3F816
:10A9F000D4227B68B03253F82230FB607B68D3F8F6
:10AA0000D4227B68B03253F82230002B01D10323CB
:10AA100018E07B681B7C002B0AD10C4B1978FB6873
:10AA2000D3F804224FF40073786803F067FE08E05F
:10AA3000064B1978FB68D3F804224023786803F0AA
:10AA40005DFE002318461037BD4680BD94000020EF
:10AA500080B483B000AF78607B6803F108027B6844
:10AA60005A607B684FF0FF329A607B6803F10802FE
:10AA70007B68DA607B6803F108027B681A617B6897
:10AA800000221A6000BF0C37BD465DF8047B70479A
:10AA900080B483B000AF78607B6800221A6100BF89
:10AAA0000C37BD465DF8047B704780B485B000AFBD
:10AAB000786039607B685B68FB603B68FA685A6065
:10AAC000FB689A683B689A60FB689B683A685A60C2
:10AAD000FB683A689A603B687A681A617B681B6811
:10AAE0005A1C7B681A6000BF1437BD465DF8047BB2
:10AAF000704780B485B000AF786039603B681B68F0
:10AB0000BB60BB68B3F1FF3F03D17B681B69FB608F
:10AB10000CE07B680833FB6002E0FB685B68FB606D
:10AB2000FB685B681B68BA689A42F6D2FB685A6891
:10AB30003B685A603B685B683A689A603B68FA68B1
:10AB40009A60FB683A685A603B687A681A617B6869
:10AB50001B685A1C7B681A6000BF1437BD465DF83D
:10AB6000047B704780B485B000AF78607B681B6958
:10AB7000FB607B685B687A6892689A607B689B6818
:10AB80007A6852685A60FB685B687A689A4203D1B7
:10AB90007B689A68FB685A607B6800221A61FB68D0
:10ABA0001B685A1EFB681A60FB681B68184614373E
:10ABB000BD465DF8047B704780B584B000AF786017
:10ABC00039607B68FB60FB68002B0DD14FF05003B0
:10ABD00072B683F31188BFF36F8FBFF34F8F62B6E6
:10ABE000BB6000BF00BFFDE703F0A0F9FB681A6877
:10ABF000FB68DB6BF968096C01FB03F31A44FB6823
:10AC00009A60FB6800229A63FB681A68FB685A60C6
:10AC1000FB681A68FB68DB6B013BF968096C01FB98
:10AC200003F31A44FB68DA60FB68FF2283F84420D0
:10AC3000FB68FF2283F845203B68002B14D1FB689A
:10AC40001B69002B1AD0FB681033184601F006FC74
:10AC50000346002B12D00D4B4FF080521A60BFF309
:10AC60004F8FBFF36F8F09E0FB6810331846FFF773
:10AC7000EFFEFB6824331846FFF7EAFE03F08CF979
:10AC8000012318461037BD4680BD00BF04ED00E02B
:10AC900080B58EB002AFF860B9607A603B60FB6847
:10ACA000002B0DD14FF0500372B683F31188BFF320
:10ACB0006F8FBFF34F8F62B6BB6200BF00BFFDE76F
:10ACC0003B68002B0DD14FF0500372B683F311880F
:10ACD000BFF36F8FBFF34F8F62B67B6200BF00BFC1
:10ACE000FDE77B68002B02D0BB68002B01D001235D
:10ACF00000E00023002B0DD14FF0500372B683F318
:10AD00001188BFF36F8FBFF34F8F62B63B6200BFF6
:10AD100000BFFDE77B68002B02D1BB68002B01D18F
:10AD2000012300E00023002B0DD14FF0500372B639
:10AD300083F31188BFF36F8FBFF34F8F62B6FB6150
:10AD400000BF00BFFDE750237B617B69502B0DD016
:10AD50004FF0500372B683F31188BFF36F8FBFF3C8
:10AD60004F8F62B6BB6100BF00BFFDE77B693B68E8
:10AD7000FB62FB6A002B0DD0FB6A012283F84620A0
:10AD800097F83820FB6A009313467A68B968F86828
:10AD900000F048F8FB6A18463037BD4680BD80B5E4
:10ADA0008AB002AFF860B9601346FB71FB68002BF4
:10ADB0000DD14FF0500372B683F31188BFF36F8F3C
:10ADC000BFF34F8F62B63B6100BF00BFFDE7BB68BA
:10ADD000002B02D10023FB6104E0FB68BA6802FB90
:10ADE00003F3FB61FB695033184602F0A9FDB8611B
:10ADF000BB69002B11D0BB697B617B6950337B61E0
:10AE0000BB69002283F84620FA79BB690093134698
:10AE10007A69B968F86800F005F8BB691846203708
:10AE2000BD4680BD80B584B000AFF860B9607A607F
:10AE3000FB70BB68002B03D1BB69BA691A6002E0E2
:10AE4000BB697A681A60BB69FA68DA63BB69BA6879
:10AE50001A640121B869FFF7AFFEBB69FA7883F87D
:10AE60004C2000BF1037BD4680BD80B582B000AF1A
:10AE700078607B68002B0ED07B6800229A607B682C
:10AE800000221A607B680022DA6000230022002181
:10AE9000786800F0A7F800BF0837BD4680BD80B5D0
:10AEA00086B000AF0346FB7101237B6100233B6149
:10AEB000FB791A4639697869FFF771FFF860F8681D
:10AEC000FFF7D3FFFB6818461837BD4680BD80B535
:10AED00088B002AF03463960FB7101237B61002318
:10AEE0003B61FB7900933B68002239697869FFF781
:10AEF000CFFEF860F868FFF7B8FFFB681846183710
:10AF0000BD4680BD90B587B000AF78607B683B617F
:10AF10003B69002B0DD14FF0500372B683F31188BB
:10AF2000BFF36F8FBFF34F8F62B6FB6000BF00BFF0
:10AF3000FDE73B699C6801F059FC03469C4211D136
:10AF40003B69DB685A1E3B69DA603B69DB68002BB2
:10AF500005D1002300220021386900F043F80123C5
:10AF60007B6101E000237B617B6918461C37BD468D
:10AF700090BD90B587B000AF786039607B683B6169
:10AF80003B69002B0DD14FF0500372B683F311884B
:10AF9000BFF36F8FBFF34F8F62B6FB6000BF00BF80
:10AFA000FDE73B699C6801F021FC03469C4207D108
:10AFB0003B69DB685A1C3B69DA6001237B610CE06A
:10AFC0003968386900F0A4FA78617B69002B04D0F5
:10AFD0003B69DB685A1C3B69DA607B6918461C37A1
:10AFE000BD4690BD80B58EB000AFF860B9607A60A4
:10AFF0003B6000237B63FB683B633B6B002B0DD105
:10B000004FF0500372B683F31188BFF36F8FBFF315
:10B010004F8F62B6BB6200BF00BFFDE7BB68002B6D
:10B0200003D13B6B1B6C002B01D1012300E00023FB
:10B03000002B0DD14FF0500372B683F31188BFF38C
:10B040006F8FBFF34F8F62B67B6200BF00BFFDE71B
:10B050003B68022B03D13B6BDB6B012B01D101233E
:10B0600000E00023002B0DD14FF0500372B683F3A4
:10B070001188BFF36F8FBFF34F8F62B63B6200BF83
:10B0800000BFFDE701F0C2FB0346002B02D17B6845
:10B09000002B01D1012300E00023002B0DD14FF044
:10B0A000500372B683F31188BFF36F8FBFF34F8FD6
:10B0B00062B6FB6100BF00BFFDE702F037FF3B6BEC
:10B0C0009A6B3B6BDB6B9A4202D33B68022B29D114
:10B0D0003A68B968386B00F04BFBF8623B6B5B6A0F
:10B0E000002B10D03B6B2433184601F0B7F9034610
:10B0F000002B13D03F4B4FF080521A60BFF34F8F9D
:10B10000BFF36F8F0AE0FB6A002B07D0394B4FF07B
:10B1100080521A60BFF34F8FBFF36F8F02F03CFF76
:10B12000012363E07B68002B03D102F035FF00238D
:10B130005CE07B6B002B06D107F11403184601F08D
:10B14000F3F901237B6302F027FF00F057FF02F0C1
:10B15000EDFE3B6B93F844305BB2B3F1FF3F03D19C
:10B160003B6B002283F844203B6B93F845305BB285
:10B17000B3F1FF3F03D13B6B002283F8452002F07F
:10B180000BFF3A1D07F114031146184601F0E2F9CE
:10B190000346002B24D1386B00F0E2FB0346002B62
:10B1A00018D03B6B10337A681146184601F000F94D
:10B1B000386B00F06DFB00F02FFF0346002B7FF48F
:10B1C0007CAF0C4B4FF080521A60BFF34F8FBFF330
:10B1D0006F8F72E7386B00F05BFB00F01DFF6CE7D0
:10B1E000386B00F055FB00F017FF00231846383786
:10B1F000BD4680BD04ED00E080B58EB000AFF860C4
:10B20000B9607A603B60FB683B633B6B002B0DD100
:10B210004FF0500372B683F31188BFF36F8FBFF303
:10B220004F8F62B67B6200BF00BFFDE7BB68002B9B
:10B2300003D13B6B1B6C002B01D1012300E00023E9
:10B24000002B0DD14FF0500372B683F31188BFF37A
:10B250006F8FBFF34F8F62B63B6200BF00BFFDE749
:10B260003B68022B03D13B6BDB6B012B01D101232C
:10B2700000E00023002B0DD14FF0500372B683F392
:10B280001188BFF36F8FBFF34F8F62B6FB6100BFB2
:10B2900000BFFDE702F032FFEFF311824FF05003E1
:10B2A00072B683F31188BFF36F8FBFF34F8F62B60F
:10B2B000BA617B61BB69FB623B6B9A6B3B6BDB6B7F
:10B2C0009A4202D33B68022B2CD13B6B93F845305A
:10B2D00087F82B303A68B968386B00F049FA97F96B
:10B2E0002B30B3F1FF3F12D13B6B5B6A002B16D0C2
:10B2F0003B6B2433184601F0B1F80346002B0ED007
:10B300007B68002B0BD07B6801221A6007E097F85E
:10B310002B300133DBB25AB23B6B83F8452001235B
:10B320007B6301E000237B63FB6A3B613B6983F342
:10B33000118800BF7B6B18463837BD4680BD0000C2
:10B3400080B58CB000AFF860B9607A600023FB6212
:10B35000FB68BB62BB6A002B0DD14FF0500372B685
:10B3600083F31188BFF36F8FBFF34F8F62B63B62D9
:10B3700000BF00BFFDE7BB68002B03D1BB6A1B6C9D
:10B38000002B01D1012300E00023002B0DD14FF051
:10B39000500372B683F31188BFF36F8FBFF34F8FE3
:10B3A00062B6FB6100BF00BFFDE701F02FFA034664
:10B3B000002B02D17B68002B01D1012300E0002388
:10B3C000002B0DD14FF0500372B683F31188BFF3F9
:10B3D0006F8FBFF34F8F62B6BB6100BF00BFFDE749
:10B3E00002F0A4FDBB6A9B6B7B627B6A002B1FD0C3
:10B3F000B968B86A00F026FA7B6A5A1EBB6A9A637B
:10B40000BB6A1B69002B0FD0BB6A1033184601F0D2
:10B4100025F80346002B07D03C4B4FF080521A60B2
:10B42000BFF34F8FBFF36F8F02F0B6FD012369E0CA
:10B430007B68002B03D102F0AFFD002362E0FB6AC2
:10B44000002B06D107F11003184601F06DF8012317
:10B45000FB6202F0A1FD00F0D1FD02F067FDBB6AC6
:10B4600093F844305BB2B3F1FF3F03D1BB6A0022D3
:10B4700083F84420BB6A93F845305BB2B3F1FF3FD9
:10B4800003D1BB6A002283F8452002F085FD3A1DF6
:10B4900007F110031146184601F05CF80346002B33
:10B4A00023D1B86A00F046FA0346002B17D0BB6AD6
:10B4B00024337A681146184600F07AFFB86A00F023
:10B4C000E7F900F0A9FD0346002B89D10F4B4FF09F
:10B4D00080521A60BFF34F8FBFF36F8F80E7B86A57
:10B4E00000F0D6F900F098FD7AE7B86A00F0D0F9DC
:10B4F00000F092FDB86A00F01DFA0346002B3FF4FD
:10B500006FAF002318463037BD4680BD04ED00E024
:10B5100080B58EB000AF7860396000237B637B68B4
:10B52000FB6200233B63FB6A002B0DD14FF05003FD
:10B5300072B683F31188BFF36F8FBFF34F8F62B67C
:10B540003B6200BF00BFFDE7FB6A1B6C002B0DD008
:10B550004FF0500372B683F31188BFF36F8FBFF3C0
:10B560004F8F62B6FB6100BF00BFFDE701F04EF9EF
:10B570000346002B02D13B68002B01D1012300E0E0
:10B580000023002B0DD14FF0500372B683F31188C6
:10B59000BFF36F8FBFF34F8F62B6BB6100BF00BFB9
:10B5A000FDE702F0C3FCFB6A9B6BBB62BB6A002B2E
:10B5B00024D0BB6A5A1EFB6A9A63FB6A1B68002B85
:10B5C00004D101F0A5FA0246FB6A9A60FB6A1B6986
:10B5D000002B0FD0FB6A1033184600F03FFF0346E4
:10B5E000002B07D0554B4FF080521A60BFF34F8F9E
:10B5F000BFF36F8F02F0D0FC01239AE03B68002B71
:10B6000014D13B6B002B0DD04FF0500372B683F377
:10B610001188BFF36F8FBFF34F8F62B67B6100BF9E
:10B6200000BFFDE702F0B8FC002382E07B6B002B3B
:10B6300006D107F10C03184600F076FF01237B6367
:10B6400002F0AAFC00F0DAFC02F070FCFB6A93F84E
:10B6500044305BB2B3F1FF3F03D1FB6A002283F8B1
:10B660004420FB6A93F845305BB2B3F1FF3F03D14E
:10B67000FB6A002283F8452002F08EFC3A4607F16F
:10B680000C031146184600F065FF0346002B32D12B
:10B69000F86A00F04FF90346002B26D0FB6A1B68BE
:10B6A000002B09D102F042FCFB6A9B68184601F0AE
:10B6B000CBF8386302F070FCFB6A24333A68114619
:10B6C000184600F075FEF86A00F0E2F800F0A4FCFD
:10B6D0000346002B7FF465AF184B4FF080521A6081
:10B6E000BFF34F8FBFF36F8F5BE7F86A00F0D0F8BE
:10B6F00000F092FC55E7F86A00F0CAF800F08CFC04
:10B70000F86A00F017F90346002B3FF44AAF3B6B91
:10B71000002B0DD002F00AFCF86A00F011F87862F4
:10B72000FB6A9B68796A184601F06AF902F034FCFA
:10B73000002318463837BD4680BD00BF04ED00E049
:10B7400080B485B000AF78607B685B6A002B06D060
:10B750007B681B6B1B68C3F13803FB6001E00023AF
:10B76000FB60FB6818461437BD465DF8047B7047E4
:10B7700080B586B000AFF860B9607A6000237B6165
:10B78000FB689B6B3B61FB681B6C002B0DD1FB685E
:10B790001B68002B4DD1FB689B68184601F0BCF874
:10B7A0007861FB6800229A6043E07B68002B19D126
:10B7B000FB685868FB681B6C1A46B96819F0FBFEF9
:10B7C000FB685A68FB681B6C1A44FB685A60FB688C
:10B7D0005A68FB689B689A422BD3FB681A68FB681F
:10B7E0005A6026E0FB68D868FB681B6C1A46B9688B
:10B7F00019F0E1FEFB68DA68FB681B6C5B421A44D7
:10B80000FB68DA60FB68DA68FB681B689A4207D25B
:10B81000FB689A68FB681B6C5B421A44FB68DA6041
:10B820007B68022B05D13B69002B02D03B69013BB1
:10B830003B613B695A1CFB689A637B691846183761
:10B84000BD4680BD80B582B000AF786039607B684E
:10B850001B6C002B18D07B68DA687B681B6C1A4461
:10B860007B68DA607B68DA687B689B689A4203D3FE
:10B870007B681A687B68DA607B68D9687B681B6CB8
:10B880001A46386819F097FE00BF0837BD4680BDDC
:10B8900080B584B000AF786002F048FB7B6893F815
:10B8A0004530FB7311E07B685B6A002B12D07B682C
:10B8B0002433184600F0D2FD0346002B01D000F0DF
:10B8C000B1FEFB7B013BDBB2FB7397F90F30002B22
:10B8D000E9DC00E000BF7B68FF2283F8452002F02E
:10B8E0005BFB02F023FB7B6893F84430BB7311E0F1
:10B8F0007B681B69002B12D07B681033184600F060
:10B90000ADFD0346002B01D000F08CFEBB7B013B5C
:10B91000DBB2BB7397F90E30002BE9DC00E000BF0F
:10B920007B68FF2283F8442002F036FB00BF10370B
:10B93000BD4680BD80B584B000AF786002F0F6FAF5
:10B940007B689B6B002B02D10123FB6001E000238D
:10B95000FB6002F021FBFB6818461037BD4680BD36
:10B9600080B584B000AF786002F0E0FA7B689A6B33
:10B970007B68DB6B9A4202D10123FB6001E000236C
:10B98000FB6002F009FBFB6818461037BD4680BD1E
:10B9900080B485B000AF786039600023FB6014E0AC
:10B9A0000F4AFB6852F83330002B0BD10C49FB686F
:10B9B0003A6841F833200A4AFB68DB0013447A688E
:10B9C0005A6006E0FB680133FB60FB68072BE7D990
:10B9D00000BF00BF1437BD465DF8047B704700BF51
:10B9E000B803002080B586B000AFF860B9607A6017
:10B9F000FB687B6102F09AFA7B6993F844305BB292
:10BA0000B3F1FF3F03D17B69002283F844207B69B7
:10BA100093F845305BB2B3F1FF3F03D17B6900225D
:10BA200083F8452002F0B8FA7B699B6B002B06D1A6
:10BA30007B6924337A68B968184600F0E1FC7869BC
:10BA4000FFF726FF00BF1837BD4680BD80B58EB01A
:10BA500004AFF860B9607A603B607B6B002B0DD15E
:10BA60004FF0500372B683F31188BFF36F8FBFF3AB
:10BA70004F8F62B63B6200BF00BFFDE7BB6B002B80
:10BA80000DD14FF0500372B683F31188BFF36F8F5F
:10BA9000BFF34F8F62B6FB6100BF00BFFDE75C23C1
:10BAA0003B613B695C2B0DD04FF0500372B683F3C2
:10BAB0001188BFF36F8FBFF34F8F62B6BB6100BFBA
:10BAC00000BFFDE73B69BB6B002B1ED07B6B002BDF
:10BAD0001BD0BB6B7B627B6A7A6B1A637B6A022228
:10BAE00083F85920002303937B6A029307F1140320
:10BAF00001933B6B00933B687A68B968F86800F083
:10BB000050F8786A00F0E0F801E000237B617B697F
:10BB100018462837BD4680BD80B58CB004AFF860AC
:10BB2000B9603B601346FB80FB889B00184601F020
:10BB300007FF78617B69002B0ED05C2001F000FFCD
:10BB4000F861FB69002B03D0FB697A691A6305E091
:10BB5000786901F0C3FF01E00023FB61FB69002B62
:10BB600017D0FB69002283F85920FA880023039339
:10BB7000FB690293FB6A0193BB6A00933B68B96857
:10BB8000F86800F00EF8F86900F09EF80123BB6138
:10BB900002E04FF0FF33BB61BB6918462037BD465A
:10BBA00080BD80B588B000AFF860B9607A603B6056
:10BBB0003B6B186B7B689B001A46A52119F0FCFBB8
:10BBC0003B6B1A6B79686FF040430B449B00134446
:10BBD000BB61BB6923F00703BB61BB6903F00703CB
:10BBE000002B0DD04FF0500372B683F31188BFF3D2
:10BBF0006F8FBFF34F8F62B67B6100BF00BFFDE761
:10BC0000BB68002B1FD00023FB6112E0BA68FB6900
:10BC1000134419783A6BFB69134434330A461A709B
:10BC2000BA68FB6913441B78002B06D0FB6901330B
:10BC3000FB61FB690F2BE9D900E000BF3B6B0022E1
:10BC400083F8432003E03B6B002283F83420BB6A77
:10BC5000372B01D93723BB623B6BBA6ADA623B6B85
:10BC6000BA6ADA643B6B00221A653B6B04331846F0
:10BC7000FEF70EFF3B6B18331846FEF709FF3B6BD0
:10BC80003A6B1A61BB6AC3F138023B6B9A613B6B3A
:10BC90003A6B5A623B6B00225A653B6B002283F879
:10BCA00058203A68F968B86902F034F802463B6BEC
:10BCB0001A60FB6A002B02D0FB6A3A6B1A6000BF65
:10BCC0002037BD4680BD000080B582B000AF7860EF
:10BCD00002F02CF92D4B1B6801332C4A13602C4BBE
:10BCE0001B68002B09D12A4A7B681360274B1B680D
:10BCF000012B10D100F0BAFC0DE0264B1B68002B85
:10BD000009D1234B1B68DA6A7B68DB6A9A4202D846
:10BD10001F4A7B681360204B1B6801331E4A136067
:10BD20001D4B1A687B685A647B68DA6A1B4B1B6878
:10BD30009A4203D97B68DB6A184A13607B68DA6A27
:10BD400013469B0013449B00154A1A447B68043336
:10BD500019461046FEF7A9FE02F01EF90D4B1B68AE
:10BD6000002B0ED00A4B1B68DA6A7B68DB6A9A42AA
:10BD700007D20C4B4FF080521A60BFF34F8FBFF3C6
:10BD80006F8F00BF0837BD4680BD00BFCC080020C4
:10BD9000F8030020D8080020E8080020D40800207C
:10BDA000FC03002004ED00E080B58AB000AF7860AD
:10BDB000396000237B627B68002B0DD14FF050036C
:10BDC00072B683F31188BFF36F8FBFF34F8F62B6E4
:10BDD0007B6100BF00BFFDE73B68002B0DD14FF03A
:10BDE000500372B683F31188BFF36F8FBFF34F8F89
:10BDF00062B63B6100BF00BFFDE72B4B1B68002B09
:10BE00000DD04FF0500372B683F31188BFF36F8FDC
:10BE1000BFF34F8F62B6FB6000BF00BFFDE700F0CD
:10BE2000EDF8224B1B683B627B681B683A68134441
:10BE3000FB617B681B683A6A9A420BD27B681B687D
:10BE4000FA699A4211D2FA693B6A9A420DD90123E2
:10BE50007B620AE07B681B68FA699A4203D3FA693D
:10BE60003B6A9A4201D901237B627B68FA691A60B6
:10BE70007B6A002B06D0FA693B6AD31A0021184668
:10BE800000F05AFE00F0C8F8B861BB69002B07D17A
:10BE9000074B4FF080521A60BFF34F8FBFF36F8F85
:10BEA00000BF2837BD4680BDF4080020D008002020
:10BEB00004ED00E080B584B000AF78600023FB6043
:10BEC0007B68002B1AD0154B1B68002B0DD04FF050
:10BED000500372B683F31188BFF36F8FBFF34F8F98
:10BEE00062B6BB6000BF00BFFDE700F087F800212D
:10BEF000786800F021FE00F08FF8F860FB68002BF6
:10BF000007D1074B4FF080521A60BFF34F8FBFF33A
:10BF10006F8F00BF1037BD4680BD00BFF408002002
:10BF200004ED00E080B58AB004AF0023BB600023BD
:10BF30007B603A46391D07F10803184601F0CCFC36
:10BF400039687B68BA68029201930023009300234A
:10BF50000A4624492448FFF779FD0346234A136023
:10BF6000224B1B68002B02D001237B6101E00023E0
:10BF70007B617B69012B02D100F032FE78617B6925
:10BF8000012B18D14FF0500372B683F31188BFF321
:10BF90006F8FBFF34F8F62B63B6100BF144B4FF002
:10BFA000FF321A60134B01221A60134B00221A60F1
:10BFB00001F03EFF11E07B69B3F1FF3F0DD14FF07F
:10BFC000500372B683F31188BFF36F8FBFF34F8FA7
:10BFD00062B6FB6000BF00BFFDE700BF1837BD467B
:10BFE00080BD00BF208503083DC60108F008002081
:10BFF000EC080020D8080020D008002080B400AF52
:10C00000044B1B680133034A136000BFBD465DF853
:10C01000047B7047F408002080B584B000AF002393
:10C02000FB600023BB60434B1B68002B0DD14FF01E
:10C03000500372B683F31188BFF36F8FBFF34F8F36
:10C0400062B63B6000BF00BFFDE701F06FFF394BF8
:10C050001B68013B374A1360364B1B68002B62D1CB
:10C06000354B1B68002B5ED02FE0344BDB68DB6860
:10C07000FB60FB6818331846FEF774FDFB68043359
:10C080001846FEF76FFDFB68DA6A2D4B1B689A4273
:10C0900003D9FB68DB6A2A4A1360FB68DA6A134635
:10C0A0009B0013449B00274A1A44FB68043319463B
:10C0B0001046FEF7FAFCFB68DA6A234B1B68DB6A62
:10C0C0009A4202D3214B01221A601C4B1B68002BA1
:10C0D000CBD1FB68002B01D000F068FB1C4B1B6828
:10C0E0007B607B68002B10D000F046F80346002BE5
:10C0F00002D0164B01221A607B68013B7B607B6893
:10C10000002BF1D1124B00221A60104B1B68002B40
:10C1100009D00123BB600F4B4FF080521A60BFF370
:10C120004F8FBFF36F8F01F037FFBB681846103792
:10C13000BD4680BDF4080020CC0800208C080020FB
:10C14000D4080020FC030020F8030020E0080020B1
:10C15000DC08002004ED00E080B483B000AF054BA4
:10C160001B687B607B6818460C37BD465DF8047B16
:10C17000704700BFD008002080B586B000AF002314
:10C180007B61504B1B68002B40F08C804E4B1B6832
:10C1900001333B614C4A3B6913603B69002B23D15F
:10C1A0004A4B1B681B68002B0DD04FF0500372B632
:10C1B00083F31188BFF36F8FBFF34F8F62B63B607D
:10C1C00000BF00BFFDE7414B1B68FB60404B1B6895
:10C1D0003E4A13603E4AFB6813603E4B1B680133C6
:10C1E0003C4A136000F0E2FA3B4B1B683A699A4202
:10C1F00049D3364B1B681B68002B04D1364B4FF0DC
:10C20000FF321A603FE0314B1B68DB68DB68BB60C4
:10C21000BB685B687B603A697B689A4203D22E4AAE
:10C220007B6813602FE0BB6804331846FEF79AFC66
:10C23000BB689B6A002B04D0BB6818331846FEF716
:10C2400091FCBB68DA6A254B1B689A4203D9BB682C
:10C25000DB6A224A1360BB68DA6A13469B00134408
:10C260009B001F4A1A44BB68043319461046FEF768
:10C270001CFCBB68DA6A1B4B1B68DB6A9A42B8D3AA
:10C2800001237B61B5E7174B1B68DA6A1449134633
:10C290009B0013449B000B441B68012B07D901230F
:10C2A0007B6104E0104B1B6801330F4A13600F4B96
:10C2B0001B68002B01D001237B617B69184618376E
:10C2C000BD4680BDF4080020D0080020840800206E
:10C2D00088080020E4080020EC080020D408002092
:10C2E000FC030020F8030020DC080020E008002008
:10C2F00080B485B000AF294B1B68002B03D0284BBE
:10C3000001221A6044E0264B00221A60254B1B686C
:10C31000FB6013E0FB68002B0DD14FF0500372B6A9
:10C3200083F31188BFF36F8FBFF34F8F62B67B60CB
:10C3300000BF00BFFDE7FB68013BFB601A49FA68DC
:10C3400013469B0013449B000B441B68002BE1D059
:10C35000FA6813469B0013449B00134A1344BB60C6
:10C36000BB685B685A68BB685A60BB685A68BB6840
:10C3700008339A4204D1BB685B685A68BB685A604C
:10C38000BB685B68DB68094A1360064AFB68136098
:10C3900000BF1437BD465DF8047B7047F4080020E9
:10C3A000E0080020D4080020FC030020F80300204F
:10C3B00080B584B000AF786039607B68002B0DD108
:10C3C0004FF0500372B683F31188BFF36F8FBFF342
:10C3D0004F8F62B6FB6000BF00BFFDE7074B1B68D5
:10C3E000183319467868FEF784FB0121386800F09D
:10C3F000A3FB00BF1037BD4680BD00BFF80300207F
:10C4000080B586B000AFF860B9607A60FB68002B39
:10C410000DD14FF0500372B683F31188BFF36F8FC5
:10C42000BFF34F8F62B67B6100BF00BFFDE70A4BD1
:10C430001B6818331946F868FEF737FB7B68002B3A
:10C4400002D04FF0FF33BB607968B86800F074FB2E
:10C4500000BF1837BD4680BDF803002080B586B008
:10C4600000AF78607B68DB68DB683B613B69002B71
:10C470000DD14FF0500372B683F31188BFF36F8F65
:10C48000BFF34F8F62B6FB6000BF00BFFDE73B69A3
:10C4900018331846FEF766FB1D4B1B68002B1DD199
:10C4A0003B6904331846FEF75DFB3B69DA6A194BBA
:10C4B0001B689A4203D93B69DB6A164A13603B69E1
:10C4C000DA6A13469B0013449B00134A1A443B69E3
:10C4D000043319461046FEF7E8FA05E03B691833C5
:10C4E00019460E48FEF7E1FA3B69DA6A0C4B1B6805
:10C4F000DB6A9A4205D901237B610A4B01221A604B
:10C5000001E000237B617B6918461837BD4680BD7A
:10C51000F4080020D4080020FC0300208C08002030
:10C52000F8030020E008002080B483B000AF7860FA
:10C53000064B1A687B681A60054B1A687B685A605C
:10C5400000BF0C37BD465DF8047B7047E40800204F
:10C55000D008002080B588B000AF786039607B6873
:10C56000002B0DD14FF0500372B683F31188BFF347
:10C570006F8FBFF34F8F62B63B6100BF00BFFDE717
:10C580003B68002B0DD14FF0500372B683F3118836
:10C59000BFF36F8FBFF34F8F62B6FB6000BF00BF6A
:10C5A000FDE701F0C3FC1D4B1B68BB617B685B684A
:10C5B000BA69D31A7B613B681B68B3F1FF3F02D1B4
:10C5C0000023FB6123E07B681A68154B1B689A42C5
:10C5D00007D07B685B68BA699A4202D30123FB618A
:10C5E00015E03B681B687A699A420BD23B681A686F
:10C5F0007B69D21A3B681A607868FFF795FF0023C1
:10C60000FB6104E03B6800221A600123FB6101F03A
:10C61000C3FCFB6918462037BD4680BDD00800200A
:10C62000E408002080B400AF034B01221A6000BF71
:10C63000BD465DF8047B7047E008002080B582B0FD
:10C6400000AF786000F052F8064B1B68012BF9D957
:10C65000054B4FF080521A60BFF34F8FBFF36F8FBF
:10C66000F0E700BFFC03002004ED00E080B582B0DD
:10C6700000AF00237B600CE07A6813469B001344F4
:10C680009B00124A13441846FEF7E2F97B68013317
:10C690007B607B68372BEFD90D48FEF7D9F90D4841
:10C6A000FEF7D6F90C48FEF7D3F90C48FEF7D0F99F
:10C6B0000B48FEF7CDF90B4B054A1A600A4B054AA9
:10C6C0001A6000BF0837BD4680BD00BFFC030020D4
:10C6D0005C080020700800208C080020A0080020C2
:10C6E000B8080020840800208808002080B582B0A7
:10C6F00000AF19E001F01AFC104BDB68DB687B60CF
:10C700007B6804331846FEF72DFA0D4B1B68013B7E
:10C710000B4A13600B4B1B68013B0A4A136001F084
:10C720003BFC786800F010F8064B1B68002BE1D149
:10C7300000BF00BF0837BD4680BD00BFA008002075
:10C74000CC080020B408002080B584B000AF786029
:10C750007B6893F85930002B08D17B681B6B184617
:10C7600001F0BCF9786801F0B9F91BE07B6893F837
:10C770005930012B03D1786801F0B0F912E07B68E1
:10C7800093F85930022B0DD04FF0500372B683F35B
:10C790001188BFF36F8FBFF34F8F62B6FB6000BF8E
:10C7A00000BFFDE700BF1037BD4680BD80B483B039
:10C7B00000AF0C4B1B681B68002B04D10A4B4FF0D9
:10C7C000FF321A6008E0074B1B68DB68DB687B60A0
:10C7D0007B685B68044A136000BF0C37BD465DF898
:10C7E000047B704784080020EC08002080B483B0EC
:10C7F00000AF054B1B687B607B6818460C37BD4655
:10C800005DF8047B704700BFF803002080B483B05C
:10C8100000AF0B4B1B68002B02D101237B6008E0AB
:10C82000084B1B68002B02D102237B6001E0002330
:10C830007B607B6818460C37BD465DF8047B70470B
:10C84000D8080020F408002080B584B000AF7860DC
:10C850007B68BB600023FB607B68002B51D0BB680A
:10C86000DA6A2A4B1B68DB6A9A4241D2BB689B6931
:10C87000002B06DB254B1B68DB6AC3F13802BB6863
:10C880009A61BB685969BB68DA6A13469B00134416
:10C890009B001F4A1344994222D1BB6804331846B7
:10C8A000FEF760F9194B1B68DA6ABB68DA62BB688D
:10C8B000DA6A184B1B689A4203D9BB68DB6A154ACF
:10C8C0001360BB68DA6A13469B0013449B00104A4E
:10C8D0001A44BB68043319461046FEF7E6F804E034
:10C8E0000A4B1B68DA6ABB68DA620123FB6008E066
:10C8F000BB68DA6C054B1B68DB6A9A4201D20123E4
:10C90000FB60FB6818461037BD4680BDF803002069
:10C91000FC030020D408002080B586B000AF78600A
:10C920007B683B6100237B617B68002B5CD0314BD3
:10C930001B683A699A420DD04FF0500372B683F3E8
:10C940001188BFF36F8FBFF34F8F62B6FB6000BFDC
:10C9500000BFFDE73B691B6D002B0DD14FF050036D
:10C9600072B683F31188BFF36F8FBFF34F8F62B638
:10C97000BB6000BF00BFFDE73B691B6D5A1E3B69F2
:10C980001A653B69DA6A3B69DB6C9A422CD03B69D9
:10C990001B6D002B28D13B6904331846FEF7E2F8E3
:10C9A0003B69DA6C3B69DA623B69DB6AC3F13802E6
:10C9B0003B699A613B69DA6A0F4B1B689A4203D95B
:10C9C0003B69DB6A0C4A13603B69DA6A13469B00D9
:10C9D00013449B00094A1A443B6904331946104624
:10C9E000FEF763F801237B617B6918461837BD4663
:10C9F00080BD00BFF8030020D4080020FC03002005
:10CA000080B588B000AF786039607B68BB61012376
:10CA10007B617B68002B70D0BB691B6D002B0DD137
:10CA20004FF0500372B683F31188BFF36F8FBFF3DB
:10CA30004F8F62B6FB6000BF00BFFDE7BB69DB6CD8
:10CA40003A689A4202D93B68FB6102E0BB69DB6C41
:10CA5000FB61BB69DB6AFA699A424ED0BB691B6D08
:10CA60007A699A4249D1274B1B68BA699A420DD11B
:10CA70004FF0500372B683F31188BFF36F8FBFF38B
:10CA80004F8F62B6BB6000BF00BFFDE7BB69DB6ACA
:10CA90003B61BB69FA69DA62BB699B69002B04DB05
:10CAA000FB69C3F13802BB699A61BB6959693A698C
:10CAB00013469B0013449B00134A134499421CD114
:10CAC000BB6904331846FEF74DF8BB69DA6A0F4BB1
:10CAD0001B689A4203D9BB69DB6A0C4A1360BB69C5
:10CAE000DA6A13469B0013449B00074A1A44BB6949
:10CAF000043319461046FDF7D8FF00BF2037BD4666
:10CB000080BD00BFF8030020FC030020D4080020F3
:10CB100080B400AF074B1B68002B04D0054B1B688B
:10CB20001A6D01321A65034B1B681846BD465DF845
:10CB3000047B7047F803002080B584B000AF7860B4
:10CB40003960214B1B68FB60204B1B68043318467F
:10CB5000FEF708F87B68B3F1FF3F0AD13B68002B72
:10CB600007D01A4B1B68043319461948FDF79DFF7F
:10CB700026E0FA687B681344BB60144B1B68BA68F4
:10CB80005A60BA68FB689A4209D2124B1A680F4B76
:10CB90001B68043319461046FDF7ABFF10E00E4B3F
:10CBA0001A680A4B1B68043319461046FDF7A1FFAB
:10CBB0000A4B1B68BA689A4202D2084ABB681360E3
:10CBC00000BF1037BD4680BDD0080020F80300200C
:10CBD000B80800208808002084080020EC08002005
:10CBE00080B58AB004AF00237B6100F021FB1E4BAF
:10CBF0001B68002B21D00023FB600023BB603A1D83
:10CC000007F1080107F10C03184600F07FFE796870
:10CC1000BB68FA68029201930223009300230A463C
:10CC200012491348FEF712FF0346124A1360114BD4
:10CC30001B68002B01D001237B617B69002B0DD188
:10CC40004FF0500372B683F31188BFF36F8FBFF3B9
:10CC50004F8F62B63B6100BF00BFFDE77B6918469E
:10CC60001837BD4680BD00BF28090020288503086D
:10CC7000B9CD01082C09002080B58AB000AFF8605A
:10CC8000B9607A603B6000237B62FB68002B0DD1AA
:10CC90004FF0500372B683F31188BFF36F8FBFF369
:10CCA0004F8F62B63B6200BF00BFFDE7194B1B68A8
:10CCB000002B2AD0BB683B617B687B61FB68BB6152
:10CCC000BB68052B18DCFFF7A1FD0346022B09D139
:10CCD000104B186807F1100100233A6BFEF782F938
:10CCE000786212E00B4B186807F110010023002254
:10CCF000FEF778F9786208E0064B186807F1100132
:10CD000000233A68FEF778FA78627B6A184628377B
:10CD1000BD4680BD2809002080B588B002AF78608C
:10CD20003960244B1B68DB68DB687B617B690433FB
:10CD30001846FDF717FF7B6993F8283003F00403CA
:10CD4000002B25D07B699A697B68D1187B683A688B
:10CD5000786900F0D7F80346002B22D00023009317
:10CD600000237A6800217869FFF786FF38613B6904
:10CD7000002B16D14FF0500372B683F31188BFF326
:10CD80006F8FBFF34F8F62B6FB6000BF00BFFDE740
:10CD90007B6993F8283023F00103DAB27B6983F8CA
:10CDA00028207B691B6A7869984700BF1837BD4601
:10CDB00080BD00BF2009002080B584B000AF78603E
:10CDC00007F10803184600F059F8F860BB681946E7
:10CDD000F86800F005F800F0D7F800BFF0E70000B1
:10CDE00080B584B000AF78603960FFF707F907F1CC
:10CDF0000803184600F066F8F860BB68002B30D1D5
:10CE00003B68002B0AD17A68FB689A4206D8FFF784
:10CE100003F9F9687868FFF77FFF24E03B68002B8F
:10CE200008D0134B1B681B68002B01D1012300E0C5
:10CE300000233B600F4B18687A68FB68D31A3A6886
:10CE40001946FEF7CFFDFFF7E7F80346002B0AD19E
:10CE5000094B4FF080521A60BFF34F8FBFF36F8FB3
:10CE600001E0FFF7D9F800BF1037BD4680BD00BF15
:10CE7000240900202809002004ED00E080B485B0DA
:10CE800000AF78600E4B1B681B68002B01D101229C
:10CE900000E000227B681A607B681B68002B05D1CC
:10CEA000074B1B68DB681B68FB6001E00023FB602D
:10CEB000FB6818461437BD465DF8047B704700BF19
:10CEC0002009002080B584B000AF7860FFF744F9F6
:10CED000F8600B4B1B68FA689A4205D200F040F9E3
:10CEE0007B6801221A6002E07B6800221A60044A13
:10CEF000FB681360FB6818461037BD4680BD00BF55
:10CF00003009002080B586B000AFF860B9607A6063
:10CF10003B6000237B61FB68BA685A60FB68FA6873
:10CF20001A61BA687B689A4212D87A683B68D21A4A
:10CF3000FB689B699A4202D301237B611BE0104B83
:10CF40001A68FB68043319461046FDF7D2FD12E05B
:10CF50007A683B689A4206D2BA683B689A4202D322
:10CF600001237B6107E0074B1A68FB68043319460D
:10CF70001046FDF7BEFD7B6918461837BD4680BDDB
:10CF8000240900202009002080B58EB002AFD4E033
:10CF90007B68002B1BDA3B1D0433FB62FB6A002B12
:10CFA0000DD14FF0500372B683F31188BFF36F8F2A
:10CFB000BFF34F8F62B6FB6100BF00BFFDE7FB6AA6
:10CFC0001B68FA6A5068FA6A9268114698477B684B
:10CFD000002BC0F2B280FB68BB62BB6A5B69002BAE
:10CFE00004D0BB6A04331846FDF7BCFD3B46184627
:10CFF000FFF768FF78627B68092B00F29B8001A233
:10D0000052F823F02DD001082DD001082DD00108B1
:10D01000A7D00108BBD001080BD101082DD0010811
:10D020002DD00108A7D00108BBD00108BB6A93F836
:10D03000283043F00103DAB2BB6A83F82820BA68CB
:10D04000BB6A9B69D118BB687A6AB86AFFF75AFF56
:10D050000346002B70D0BB6A1B6AB86A9847BB6A4C
:10D0600093F8283003F00403002B65D0BA68BB6A3C
:10D070009B691A440023009300230021B86AFFF73C
:10D08000FBFD38623B6A002B56D14FF0500372B65D
:10D0900083F31188BFF36F8FBFF34F8F62B6BB610D
:10D0A00000BF00BFFDE7BB6A93F8283023F00103FF
:10D0B000DAB2BB6A83F828203FE0BB6A93F82830D5
:10D0C00043F00103DAB2BB6A83F82820BA68BB6A6E
:10D0D0009A61BB6A9B69002B0DD14FF0500372B669
:10D0E00083F31188BFF36F8FBFF34F8F62B67B61FD
:10D0F00000BF00BFFDE7BB6A9A697B6AD1187B6AF3
:10D100007A6AB86AFFF7FEFE17E0BB6A93F8283028
:10D1100003F00203002B03D1B86A00F0DFFC0CE03F
:10D12000BB6A93F8283023F00103DAB2BB6A83F8B4
:10D13000282002E000BF00E000BF084B1B68391D3B
:10D1400000221846FEF7FCF80346002B7FF420AFC0
:10D1500000BF00BF3037BD4680BD00BF280900209A
:10D1600080B588B002AF4BE02F4B1B68DB681B68B3
:10D170003B612D4B1B68DB68DB68FB60FB6804339D
:10D180001846FDF7EFFCFB681B6AF8689847FB68D8
:10D1900093F8283003F00403002B31D0FB689B691F
:10D1A0003A691344BB60BA683B699A420ED9FB687E
:10D1B000BA685A60FB68FA681A611B4B1A68FB6808
:10D1C000043319461046FDF794FC19E00023009340
:10D1D00000233A690021F868FFF74EFD78607B680C
:10D1E000002B0DD14FF0500372B683F31188BFF3BB
:10D1F0006F8FBFF34F8F62B63B6000BF00BFFDE78C
:10D20000094B1B681B68002BAED1074B1B687B6169
:10D21000064B1B68044A1360044A7B69136000BF15
:10D220001837BD4680BD00BF20090020240900201A
:10D2300080B582B002AF00F079FE154B1B68002B61
:10D2400020D11448FDF704FC1348FDF701FC134BF3
:10D25000104A1A60124B104A1A6000230093114BB7
:10D26000114A10210A20FDF713FD0346084A1360F6
:10D27000074B1B68002B05D0054B1B680B49184654
:10D28000FEF786FB00F088FE00BFBD4680BD00BFF4
:10D2900028090020F80800200C090020200900209F
:10D2A00024090020D4090020340900203085030817
:10D2B00080B400AF00BFBD465DF8047B704700003E
:10D2C00080B485B000AFEFF30583BB60BB68002B73
:10D2D0000FD1EFF310837B607B68002B05D1EFF358
:10D2E00011833B603B68002B07D00E4B1B68022B61
:10D2F00003D16FF00503FB600CE00A4B1B68002BA9
:10D3000005D1084B01221A600023FB6002E04FF0B8
:10D31000FF33FB60FB6818461437BD465DF8047B9D
:10D32000704700BF240A002080B584B000AFEFF33F
:10D330000583BB60BB68002B0FD1EFF310837B60CC
:10D340007B68002B05D1EFF311833B603B68002B1A
:10D3500007D00F4B1B68022B03D16FF00503FB6056
:10D3600010E00B4B1B68012B09D1FFF7A1FF084B05
:10D3700002221A60FEF7D6FD0023FB6002E04FF0A8
:10D38000FF33FB60FB6818461037BD4680BD00BF09
:10D39000240A002080B590B004AFF860B9607A60CC
:10D3A00000233B61EFF30583FB61FB69002B40F039
:10D3B0008F80EFF31083BB61BB69002B05D1EFF3C6
:10D3C00011837B617B69002B03D0444B1B68022BCC
:10D3D0007ED0FB68002B7BD08023BB6218237B624E
:10D3E0000023FB624FF0FF333B627B68002B45D08C
:10D3F0007B681B68002B02D07B681B68FB627B6824
:10D400009B69002B02D07B689B697B627B6A002B47
:10D4100008D07B6A382B05D87B685B6803F0010372
:10D42000002B01D0002354E07B685B69002B03D004
:10D430007B685B699B08BB627B689B68002B0ED096
:10D440007B68DB685B2B0AD97B681B69002B06D0E5
:10D450007B685B69002B02D001233B6210E07B6894
:10D460009B68002B0CD17B68DB68002B08D17B68A4
:10D470001B69002B04D100233B6201E000233B62C7
:10D480003B6A012B10D17B681B697A689268029213
:10D4900001937B6A0093BB68BA6AF96AF868FEF781
:10D4A000D5FA03463B6113E03B6A002B10D1BB6AFF
:10D4B0009AB207F1100301937B6A0093BB68F96A83
:10D4C000F868FEF729FB0346012B01D000233B61DE
:10D4D0003B6918463037BD4680BD00BF240A002096
:10D4E00080B586B000AF7860EFF305833B613B69A0
:10D4F000002B0FD1EFF31083FB60FB68002B05D1ED
:10D50000EFF31183BB60BB68002B07D00A4B1B688D
:10D51000022B03D16FF005037B6107E000237B61E1
:10D520007B68002B02D07868FEF7C4FC7B69184644
:10D530001837BD4680BD00BF240A002080B58AB0E0
:10D5400000AF786000237B62EFF305833B613B69AA
:10D55000002B40F08580EFF31083FB60FB68002B0D
:10D5600005D1EFF31183BB60BB68002B03D03F4BA9
:10D570001B68022B74D07B68002B03D07B685B6830
:10D580003B6201E000233B623B6A03F00103002B96
:10D5900002D00123FB6101E00023FB613B6A03F041
:10D5A0000803002B5CD14FF0FF33BB617B68002B7D
:10D5B00015D07B689B68002B06D07B68DB684F2BFF
:10D5C00002D90123BB610CE07B689B68002B08D16A
:10D5D0007B68DB68002B04D10023BB6101E00023E2
:10D5E000BB61BB69012B12D1FB69002B07D07B68A3
:10D5F0009B6819460420FDF76AFC786216E07B6898
:10D600009B6819460120FDF762FC78620EE0BB6959
:10D61000002B0BD1FB69002B04D00420FDF73FFC4D
:10D62000786203E00120FDF73AFC78627B6A002B08
:10D630000CD07B68002B03D07B681B687B6101E00A
:10D6400000237B617969786AFEF7A2F97B6A002B77
:10D6500006D0FB69002B03D07B6A43F001037B6299
:10D660007B6A18462837BD4680BD00BF240A0020CB
:10D6700080B588B000AF786039607B6823F0010323
:10D68000BB617B6803F001037B610023FB61EFF367
:10D6900005833B613B69002B0FD1EFF31083FB60E7
:10D6A000FB68002B05D1EFF31183BB60BB68002B37
:10D6B00007D01D4B1B68022B03D16FF00503FB61E4
:10D6C0002CE0BB69002B03D16FF00303FB6125E065
:10D6D0007B69002B11D03968B869FDF74AFC034615
:10D6E000012B1BD03B68002B03D06FF00103FB61C3
:10D6F00014E06FF00203FB6110E03968B869FDF7D0
:10D7000007FF0346012B09D03B68002B03D06FF0C5
:10D710000103FB6102E06FF00203FB61FB69184645
:10D720002037BD4680BD00BF240A002080B588B0E8
:10D7300000AF78607B6823F00103BB617B6803F076
:10D7400001037B610023FB61EFF305833B613B69D0
:10D75000002B0FD1EFF31083FB60FB68002B05D18A
:10D76000EFF31183BB60BB68002B07D0164B1B681F
:10D77000022B03D16FF00503FB611FE0BB69002B97
:10D7800003D16FF00303FB6118E07B69002B09D024
:10D79000B869FDF7B7FB0346012B0FD06FF002030A
:10D7A000FB610BE0002300220021B869FDF71AFCA1
:10D7B0000346012B02D06FF00203FB61FB691846A0
:10D7C0002037BD4680BD00BF240A002080B58CB044
:10D7D00002AFF860B9607A6000237B62EFF30583E3
:10D7E000BB61BB69002B6FD1EFF310837B617B6959
:10D7F000002B05D1EFF311833B613B69002B03D074
:10D80000344B1B68022B5FD0FB68002B5CD0BB68DD
:10D81000002B59D04FF0FF333B627B68002B29D09F
:10D820007B689B68002B12D07B68DB684F2B0ED97E
:10D830007B681B69002B0AD07B685A69FB68B96852
:10D8400001FB03F39A4202D301233B6214E07B689D
:10D850009B68002B10D17B68DB68002B0CD17B68A8
:10D860001B69002B08D17B685B69002B04D1002366
:10D870003B6201E000233B623B6A012B0BD17B68DA
:10D880001A697B689B6800210091B968F868FDF708
:10D89000FFF9786208E03B6A002B05D10022B968E5
:10D8A000F868FDF77CFA78627B6A002B0CD07B6805
:10D8B000002B03D07B681B68FB6101E00023FB6148
:10D8C000F969786AFEF764F87B6A18462837BD461E
:10D8D00080BD00BF240A002080B485B000AFF8608E
:10D8E000B9607A60FB68074A1A60BB68064A1A602A
:10D8F0007B6880221A6000BF1437BD465DF8047B48
:10D90000704700BF280A0020840A002080B485B038
:10D9100000AFF860B9607A60FB68074A1A60BB68BC
:10D92000064A1A607B684FF480721A6000BF143791
:10D93000BD465DF8047B7047840C0020E00C00209D
:10D9400080B58AB000AF78600023FB61FEF756FB1C
:10D950005D4B1B68002B01D100F020F95B4B1A686E
:10D960007B681340002B40F094807B68002B20D014
:10D9700008227B6813447B607B6803F00703002B5D
:10D9800017D07B6823F0070308337B607B6803F0C4
:10D990000703002B0DD04FF0500372B683F31188AC
:10D9A000BFF36F8FBFF34F8F62B67B6100BF00BFC5
:10D9B000FDE77B68002B6CD0454B1B687A689A4268
:10D9C00067D8444B3B62434B1B687B6204E07B6A35
:10D9D0003B627B6A1B687B627B6A5B687A689A42FF
:10D9E00003D97B6A1B68002BF1D1374B1B687A6A1D
:10D9F0009A424ED03B6A1B6808221344FB617B6A43
:10DA00001A683B6A1A607B6A5A687B68D21A0823D4
:10DA10005B009A4222D97A6A7B681344BB61BB6976
:10DA200003F00703002B0DD04FF0500372B683F3C1
:10DA30001188BFF36F8FBFF34F8F62B63B6100BF9A
:10DA400000BFFDE77B6A5A687B68D21ABB695A60DF
:10DA50007B6A7A685A60B86900F002F91C4B1A6850
:10DA60007B6A5B68D31A1A4A1360194B1A681A4BFF
:10DA70001B689A4203D2164B1B68174A13607B6AD5
:10DA80005A68124B1B681A437B6A5A607B6A0022F1
:10DA90001A60FEF7C1FAFB6903F00703002B0DD0F3
:10DAA0004FF0500372B683F31188BFF36F8FBFF34B
:10DAB0004F8F62B6FB6000BF00BFFDE7FB691846F1
:10DAC0002837BD4680BD00BFE8900020F4900020BC
:10DAD000EC900020E0900020F090002080B586B00F
:10DAE00000AF78607B687B617B68002B4ED0082399
:10DAF0005B427A6913447B617B693B613B695A688D
:10DB0000244B1B681340002B0DD14FF0500372B60D
:10DB100083F31188BFF36F8FBFF34F8F62B6FB6043
:10DB200000BF00BFFDE73B691B68002B0DD04FF025
:10DB3000500372B683F31188BFF36F8FBFF34F8F1B
:10DB400062B6BB6000BF00BFFDE73B695A68114B7E
:10DB50001B681340002B19D03B691B68002B15D1A3
:10DB60003B695A680B4B1B68DB431A403B695A60A0
:10DB7000FEF744FA3B695A68074B1B681344064A90
:10DB80001360386900F06CF8FEF746FA00BF1837EA
:10DB9000BD4680BDF4900020EC90002080B485B09C
:10DBA00000AF4FF40043BB60274BFB60FB6803F002
:10DBB0000703002B0CD0FB680733FB60FB6823F0E6
:10DBC0000703FB60BA68FB68D31A1F4A1344BB60A3
:10DBD000FB687B601D4A7B6813601C4B00225A6007
:10DBE0007B68BA681344FB600822FB689B1AFB60E1
:10DBF000FB6823F00703FB60FB68154A1360144BB6
:10DC00001B6800225A60124B1B6800221A607B6856
:10DC10003B603B68FA68D21A3B685A600C4B1A6842
:10DC20003B681A603B685B680A4A13603B685B6844
:10DC3000094A1360094B4FF000421A6000BF1437C5
:10DC4000BD465DF8047B7047E0100020E0900020A6
:10DC5000E8900020F0900020EC900020F49000204C
:10DC600080B485B000AF7860284BFB6002E0FB68B1
:10DC70001B68FB60FB681B687A689A42F7D8FB68F0
:10DC8000BB60FB685B68BA6813447A689A4208D143
:10DC9000FB685A687B685B681A44FB685A60FB68DB
:10DCA0007B607B68BB607B685B68BA681A44FB6812
:10DCB0001B689A4218D1FB681A68154B1B689A4278
:10DCC0000DD07B685A68FB681B685B681A447B68E8
:10DCD0005A60FB681B681A687B681A6008E00C4B86
:10DCE0001A687B681A6003E0FB681A687B681A6030
:10DCF000FA687B689A4202D0FB687A681A6000BFB3
:10DD00001437BD465DF8047B704700BFE0900020EB
:10DD1000E890002080B485B000AFF860B9607A6008
:10DD2000FB68043BFB60FB684FF080721A60FB6885
:10DD3000043BFB60BB6823F00102FB681A60FB68D0
:10DD4000043BFB600C4AFB681A60FB68143BFB60F9
:10DD50007A68FB681A60FB68043BFB60FB686FF045
:10DD600002021A60FB68203BFB60FB681846143710
:10DD7000BD465DF8047B70477DDD010880B485B049
:10DD800000AF00237B60154B1B68B3F1FF3F0DD044
:10DD90004FF0500372B683F31188BFF36F8FBFF358
:10DDA0004F8F62B6FB6000BF00BFFDE74FF050032E
:10DDB00072B683F31188BFF36F8FBFF34F8F62B6D4
:10DDC000BB6000BF00BF7B68002BFCD000BF00BF62
:10DDD0001437BD465DF8047B704700BF98000020F3
:10DDE000074B19680868B0E8F04F80F30988BFF363
:10DDF0006F8F4FF0000080F311887047AFF3008001
:10DE0000F803002000BF00BF08480068006880F3E6
:10DE100008884FF0000080F3148862B661B6BFF343
:10DE20004F8FBFF36F8F00DF00BF00BF08ED00E032
:10DE300080B584B000AF374BFB60FB681B78DBB26A
:10DE40007B60FB68FF221A70FB681B78DBB2FB70FB
:10DE5000FB78DBB203F05003DAB22F4B1A702F4B72
:10DE600007221A6009E02D4B1B68013B2B4A136007
:10DE7000FB78DBB25B00DBB2FB70FB78DBB203F05C
:10DE80008003802BEFD0254B1B68C3F10703042BC5
:10DE90000DD04FF0500372B683F31188BFF36F8F2C
:10DEA000BFF34F8F62B6BB6000BF00BFFDE71B4BE7
:10DEB0001B681B02194A1360184B1B6803F4E063CC
:10DEC000164A13607B68DAB2FB681A70144B1B6841
:10DED000134A43F470031360114B1B68104A43F05C
:10DEE0007043136000F0DCF80E4B00221A6000F063
:10DEF000FBF80D4B1B680C4A43F040431360FFF7DF
:10DF000083FFFEF7F5F9FFF739FF002318461037B6
:10DF1000BD4680BD00E400E0F8900020FC900020A9
:10DF200020ED00E09800002034EF00E080B483B0E2
:10DF300000AF4FF0500372B683F31188BFF36F8FB9
:10DF4000BFF34F8F62B67B6000BF114B1B6801337C
:10DF50000F4A13600E4B1B68012B12D10D4B1B682F
:10DF6000DBB2002B0DD04FF0500372B683F3118853
:10DF7000BFF36F8FBFF34F8F62B63B6000BF00BF30
:10DF8000FDE700BF0C37BD465DF8047B704700BF5E
:10DF90009800002004ED00E080B483B000AF134B84
:10DFA0001B68002B0DD14FF0500372B683F311881C
:10DFB000BFF36F8FBFF34F8F62B67B6000BF00BFB0
:10DFC000FDE70A4B1B68013B084A1360074B1B68BF
:10DFD000002B05D100233B603B6883F3118800BF11
:10DFE00000BF0C37BD465DF8047B704798000020E9
:10DFF000EFF30980BFF36F8F154B1A681EF0100FF7
:10E0000008BF20ED108A20E9F04F10602DE90900CB
:10E010004FF0500072B680F31188BFF34F8FBFF3FB
:10E020006F8F62B6FEF764F94FF0000080F311883D
:10E0300009BC19680868B0E8F04F1EF0100F08BF5F
:10E04000B0EC108A80F30988BFF36F8F704700BF70
:10E05000F803002000BF00BF80B582B000AF4FF0D2
:10E06000500372B683F31188BFF36F8FBFF34F8FE6
:10E0700062B67B6000BFFEF77FF80346002B03D03B
:10E08000064B4FF080521A6000233B603B6883F3DD
:10E09000118800BF00BF0837BD4680BD04ED00E019
:10E0A00080B400AF0B4B00221A600B4B00221A60A9
:10E0B0000A4B1B680A4AA2FB03239B09094A013B3E
:10E0C0001360044B07221A6000BFBD465DF8047B55
:10E0D000704700BF10E000E018E000E00000002002
:10E0E000D34D621014E000E0DFF80C00016841F449
:10E0F00070010160704700BF88ED00E080B485B01A
:10E1000000AFEFF30583FB60FB680F2B17D91A4AAA
:10E11000FB6813441B78FB72184B1B78FA7A9A42FF
:10E120000DD24FF0500372B683F31188BFF36F8F97
:10E13000BFF34F8F62B67B6000BF00BFFDE7104B9F
:10E140001B6803F4E0620F4B1B689A420DD94FF035
:10E15000500372B683F31188BFF36F8FBFF34F8FF5
:10E1600062B63B6000BF00BFFDE700BF1437BD468D
:10E170005DF8047B704700BFF0E300E0F8900020FA
:10E180000CED00E0FC90002080B5AEB000AF7860F0
:10E1900007F1A40300221A605A609A60DA601A61DB
:10E1A00007F1140390220021184617F005F97B6847
:10E1B0001B68B3F1A04F51D14FF400137B610023D2
:10E1C000C7F8903007F114031846F7F7B9FC034677
:10E1D000002B01D002F02EF8224B1B6B214A43F09A
:10E1E000010313631F4B1B6B03F001033B613B698E
:10E1F0004FF4C053C7F8A4300223C7F8A830002357
:10E20000C7F8AC300323C7F8B0300A23C7F8B430DE
:10E2100007F1A40319461448F8F77EFB114B5B6B1A
:10E22000104A43F0800353630E4B5B6B03F0800393
:10E23000FB60FB680B4B5B6C0A4A43F480435364FE
:10E24000084B5B6C03F48043BB60BB680022052174
:10E250004320F8F763FF4320F8F77CFF00BFB8378F
:10E26000BD4680BD003802400000024080B582B04B
:10E2700000AF78607B68D3F8DC247B6803F29C43B2
:10E2800019461046FAF77DFC00BF0837BD4680BD31
:10E2900080B582B000AF78600B46FB707B68D3F826
:10E2A000DC04FA7879681346DB0013449B000B44C6
:10E2B00003F518731A68FB781946FAF7B7FC00BF24
:10E2C0000837BD4680BD80B582B000AF78600B4690
:10E2D000FB707B68D3F8DC04FA7879681346DB00BE
:10E2E00013449B000B4420331A68FB781946FAF755
:10E2F00059FD00BF0837BD4680BD80B582B000AF74
:10E3000078607B68D3F8DC341846FAF79DFE00BFCE
:10E310000837BD4680BD80B584B000AF786001236A
:10E32000FB737B68DB79002B02D10023FB7308E0D1
:10E330007B68DB79022B02D10123FB7301E001F042
:10E3400079FF7B68D3F8DC34FA7B11461846FAF77C
:10E3500037FE7B68D3F8DC341846FAF7DEFD00BFE1
:10E360001037BD4680BD000080B582B000AF786038
:10E370007B68D3F8DC341846FAF732FE7B681B68FA
:10E3800003F560631B687A68126802F5606243F007
:10E39000010313607B68DB7A002B05D0044B1B69FB
:10E3A000034A43F00603136100BF0837BD4680BD32
:10E3B00000ED00E080B582B000AF78607B68D3F8F4
:10E3C000DC341846FAF728FE00BF0837BD4680BD8A
:10E3D00080B582B000AF78600B46FB707B68D3F8E5
:10E3E000DC34FA7811461846FAF780FE00BF083789
:10E3F000BD4680BD80B582B000AF78600B46FB7033
:10E400007B68D3F8DC34FA7811461846FAF73CFEFC
:10E4100000BF0837BD4680BD80B582B000AF7860D0
:10E420007B68D3F8DC341846FAF792FE00BF083751
:10E43000BD4680BD80B582B000AF78607B68D3F800
:10E44000DC341846FAF78FFE00BF0837BD4680BDA2
:10E4500080B582B000AF78607B681B78002B3CD120
:10E46000204A7B68C2F8DC347B681E4AC3F8C822A5
:10E470001C4B4FF0A0421A601A4B06221A71194B1E
:10E480000222DA71174B00229A71164B02225A723D
:10E49000144B00229A72134B0022DA72114B0022A5
:10E4A0001A73104B00229A730E4B0022DA730D4838
:10E4B000F3F7E4FF0346002B01D001F0BBFE8021FF
:10E4C0000848F5F732FA402200210648F5F7E6F948
:10E4D000802201210348F5F7E1F9002318460837A7
:10E4E000BD4680BD0091002080B584B000AF78604B
:10E4F0000023FB730023BB737B68D3F8C832184634
:10E50000F4F7D2F80346FB73FB7B184600F07EF964
:10E510000346BB73BB7B18461037BD4680BD80B534
:10E5200084B000AF7860084611461A460346FB7077
:10E530000B46BB7013463B800023FB730023BB7369
:10E540007B68D3F8C802BB783A88F978F4F7C0FD45
:10E550000346FB73FB7B184600F058F90346BB7378
:10E56000BB7B18461037BD4680BD80B584B000AF78
:10E5700078600B46FB700023FB730023BB737B6842
:10E58000D3F8C832FA7811461846F4F70BFE034662
:10E59000FB73FB7B184600F039F90346BB73BB7B6A
:10E5A00018461037BD4680BD80B584B000AF786096
:10E5B0000B46FB700023FB730023BB737B68D3F80F
:10E5C000C832FA7811461846F4F7C3FE0346FB73C7
:10E5D000FB7B184600F01AF90346BB73BB7B184659
:10E5E0001037BD4680BD80B584B000AF78600B4663
:10E5F000FB700023FB730023BB737B68D3F8C83226
:10E60000FA7811461846F4F707FF0346FB73FB7BC5
:10E61000184600F0FBF80346BB73BB7B1846103767
:10E62000BD4680BD80B485B000AF78600B46FB70FE
:10E630007B68D3F8C832FB6097F90330002B0BDA04
:10E64000FB7803F07F02F9681346DB0013449B005C
:10E650000B4416331B780BE0FB7803F07F02F9685C
:10E660001346DB0013449B000B4403F256231B7834
:10E6700018461437BD465DF8047B704780B584B0FA
:10E6800000AF78600B46FB700023FB730023BB7365
:10E690007B68D3F8C832FA7811461846F4F7F4FCD0
:10E6A0000346FB73FB7B184600F0B0F80346BB73D0
:10E6B000BB7B18461037BD4680BD80B586B000AF25
:10E6C000F8607A603B600B46FB720023FB75002309
:10E6D000BB75FB68D3F8C802F97A3B687A68F4F72F
:10E6E000FEFD0346FB75FB7D184600F08FF80346E0
:10E6F000BB75BB7D18461837BD4680BD80B586B05A
:10E7000000AFF8607A603B600B46FB720023FB753C
:10E710000023BB75FB68D3F8C802F97A3B687A68B6
:10E72000F4F78AFD0346FB75FB7D184600F06EF892
:10E730000346BB75BB7D18461837BD4680BD80B506
:10E7400082B000AF78600B46FB707B68D3F8C832AC
:10E75000FA7811461846F4F7AAFD0346184608371A
:10E76000BD4680BD80B582B000AF78600B46FB70BF
:10E77000FB78002B02D0012B1FD03BE07B68DB7ABB
:10E78000002B07D000F03CF81C4B1B691B4A23F000
:10E79000060313617B681B6803F560631B687A6876
:10E7A000126802F5606223F0010313607B68D3F8FE
:10E7B000DC341846FAF730FC1CE07B681B6803F574
:10E7C00060631B687A68126802F5606243F00103B7
:10E7D00013607B68D3F8DC341846FAF701FC7B68D9
:10E7E000DB7A002B05D0054B1B69044A43F0060376
:10E7F000136100BF00BF0837BD4680BD00ED00E0DB
:10E8000080B500AF00F020FD00BF80BD80B485B0B2
:10E8100000AF0346FB710023FB73FB79032B17D872
:10E8200001A252F823F000BF39E801083FE80108CF
:10E8300045E801084BE801080023FB730BE00323C4
:10E84000FB7308E00123FB7305E00323FB7302E085
:10E850000323FB7300BFFB7B18461437BD465DF8EE
:10E86000047B704780B500AF002214491448FAF7C2
:10E87000D5F80346002B01D001F0DCFC114910480B
:10E88000FAF7FCF80346002B01D001F0D3FC0E4947
:10E890000B48FCF70DF80346002B01D001F0CAFC31
:10E8A0000748FAF721F90346002B01D001F0C2FC1A
:10E8B0004FF47A70F8F78AFC00BF80BD9C000020FE
:10E8C000E095002018000020FC00002080B483B0F8
:10E8D00000AF03463960FB713B6812221A80034B7C
:10E8E00018460C37BD465DF8047B7047BC0000201D
:10E8F00080B483B000AF03463960FB713B680422EB
:10E900001A80034B18460C37BD465DF8047B7047F0
:10E91000DC00002080B582B000AF03463960FB7197
:10E92000FB79002B05D13A6807490848FBF7CCFA78
:10E9300004E03A6804490548FBF7C6FA024B18465A
:10E940000837BD4680BD00BFBC980020388503084D
:10E9500080B582B000AF03463960FB713A68044964
:10E960000448FBF7B1FA024B18460837BD4680BD94
:10E97000BC9800205085030880B582B000AF0346E4
:10E980003960FB713B681A221A8000F055F8024B7F
:10E9900018460837BD4680BDE000002080B582B033
:10E9A00000AF03463960FB71FB79002B05D13A6853
:10E9B00007490848FBF788FA04E03A680449054823
:10E9C000FBF782FA024B18460837BD4680BD00BFF0
:10E9D000BC9800206485030880B582B000AF034670
:10E9E0003960FB71FB79002B05D13A68074908486B
:10E9F000FBF76AFA04E03A6804490548FBF764FA51
:10EA0000024B18460837BD4680BD00BFBC980020A9
:10EA10007085030880B483B000AF03463960FB7192
:10EA20003B680C221A80034B18460C37BD465DF834
:10EA3000047B7047D000002080B584B000AF0F4B3E
:10EA40001B68FB600E4B1B68BB600E4B1B687B603A
:10EA5000FA687B681344FB60FB68002B09D008222E
:10EA60000949F86800F014F804220849B86800F071
:10EA70000FF800BF1037BD4680BD00BF20F4F01F67
:10EA800024F4F01F28F4F01FE2000020F200002020
:10EA900080B487B000AFF860B9601346FB71002303
:10EAA000FB750023FB7527E0FB681B0F092B0BD8B8
:10EAB000FB681B0FDAB2FB7D5B001946BB680B4499
:10EAC0003032D2B21A700AE0FB681B0FDAB2FB7D5B
:10EAD0005B001946BB680B443732D2B21A70FB6830
:10EAE0001B01FB60FB7D5B000133BA68134400220D
:10EAF0001A70FB7D0133FB75FA7DFB799A42D3D303
:10EB000000BF00BF1C37BD465DF8047B70470000A6
:10EB100080B500AF002205490548FBF7E3FE054933
:10EB20000348FBF701FF0023184680BDBCA200206C
:10EB3000E0950020BC9A002080B400AF0023184666
:10EB4000BD465DF8047B704780B483B000AF0346D8
:10EB50003960FB711346BB80FB79232B4AD801A295
:10EB600052F823F0F5EB0108F5EB0108F5EB01088D
:10EB7000F5EB0108F5EB0108F5EB0108F5EB0108F1
:10EB8000F5EB0108F5EB0108F5EB0108F5EB0108E1
:10EB9000F5EB0108F5EB0108F5EB0108F5EB0108D1
:10EBA000F5EB0108F5EB0108F5EB0108F5EB0108C1
:10EBB000F5EB0108F5EB0108F5EB0108F5EB0108B1
:10EBC000F5EB0108F5EB0108F5EB0108F5EB0108A1
:10EBD000F5EB0108F5EB0108F5EB0108F5EB010891
:10EBE000F5EB0108F5EB0108F5EB0108F5EB010881
:10EBF000F5EB010800BF002318460C37BD465DF851
:10EC0000047B704780B582B000AF786039603B68A4
:10EC10001B68194678680CF0ADFB79680548FBF76E
:10EC200083FE0448FBF7DEFE002318460837BD4686
:10EC300080BD00BFE095002080B584B000AF786053
:10EC40000B467B800023FB730D4BD3F8BC32BB60BB
:10EC5000BB68D3F81432002B01D001230BE07B8872
:10EC60001A4679680648FBF73DFE0548FBF77AFE31
:10EC70000346FB73FB7B18461037BD4680BD00BFC3
:10EC8000E095002080B487B000AFF860B96013460B
:10EC9000FB710023FB7597F9173018461C37BD46EA
:10ECA0005DF8047B7047000080B400AF064B93F81A
:10ECB0009C32DBB2032B0CBF01230023DBB21846CE
:10ECC000BD465DF8047B7047E095002080B5D8B064
:10ECD00002AF834BC7F85031D7F850311B68814AD7
:10ECE000934231D1D7F8503100221A6072B600BF7A
:10ECF00007F5AC73A3F5AC737B4A1A60F6F790F98D
:10ED00007A4B00221A60794B00225A60774B00221E
:10ED10009A6007F5AC73A3F5AC731B681B68C7F862
:10ED20004831D7F8483183F3088800BF07F5AC7342
:10ED3000A3F5AC731B6804331B68C7F84C31D7F8D4
:10ED40004C31984700BFFDE7F8F712FA00F07CFA63
:10ED500001F0FCF800F090FB07F05CFC02F0EAFE2A
:10ED60000DF0C6F800F0AEFB00F080FC00F056FDA0
:10ED700000F02CFE5E4B1B78DBB2012B04D15D480A
:10ED8000F2F7CCF800F07CFE5B4B1B78DBB2012B7A
:10ED900004D15A48F2F7C2F800F0BEFC584B1B7879
:10EDA000DBB2012B04D15748F2F7B8F800F0DEFBD4
:10EDB000554B1B78DBB2012B04D15448F2F7AEF867
:10EDC00000F082FD00F0A2FF00F0E4FF01F02EF859
:10EDD00001F070F800F0ACFA00F0FCFAFFF742FD29
:10EDE000002240214A48F8F767F8C820F8F7EEF902
:10EDF000012240214648F8F75FF8C820F8F7E6F905
:10EE000002F0B6FE04F0A8FB0023C7F854310AE074
:10EE100044F62061D7F8540105F040FAD7F8543190
:10EE20000133C7F85431D7F85431032BF0DD304BA0
:10EE30001B78DBB21946304B1B78DBB21A46304BDD
:10EE40001B78DBB21846304B1B78DBB200930346CD
:10EE500030480CF0B7FE264B1B78DBB2012B08D1F3
:10EE600000212448F1F73EFE04212248F1F73AFE42
:10EE700003E03C211F48F2F797F81F4B1B78DBB2E9
:10EE8000012B08D100211D48F1F72CFE04211B485D
:10EE9000F1F728FE03E03C211848F2F785F8184BFB
:10EEA0001B78DBB2012B08D100211648F1F71AFEBE
:10EEB00004211448F1F716FE03E03C211148F2F753
:10EEC00073F8114B1B78DBB2012B25D100210F48C1
:10EED000F1F708FE04210D48F1F704FE20E000BF21
:10EEE000F0FF0720EFBEADDE0000F01F10E000E0F5
:10EEF000D8AE002078AC0020D9AE0020E0AB0020D6
:10EF0000DAAE002094AB0020DBAE00202CAC002059
:10EF1000001802408C8503083C21AC48F2F744F805
:10EF20000DF07EFB002301220121012003F024FECD
:10EF3000002301220121022003F01EFE00230122F2
:10EF40000121032003F018FEFEF7BAF903F06CFF6D
:10EF50000DF0D2F99E4A00219E48FEF71BFA0346A7
:10EF60009D4A136007F5927324220021184616F07B
:10EF700023FA9A4BC7F824314FF48053C7F838313D
:10EF80001023C7F83C3107F580732422002118466E
:10EF900016F012FA924BC7F800314FF40063C7F82D
:10EFA00014311823C7F8183107F1DC03242200219B
:10EFB000184616F001FA8B4BC7F8DC304FF40063AB
:10EFC000C7F8F0302823C7F8F43007F1B80324223B
:10EFD0000021184616F0F0F9834BC7F8B8304FF40B
:10EFE000C063C7F8CC301823C7F8D03007F19403BA
:10EFF00024220021184616F0DFF97C4BC7F8943024
:10F000004FF48063C7F8A8300823C7F8AC3007F185
:10F01000700324220021184616F0CEF9744B3B678A
:10F020004FF4C063C7F884302823C7F8883007F549
:10F03000AC73A3F58673184624231A46002116F0F4
:10F04000BBF907F5AC73A3F586736A4A1A6007F536
:10F05000AC73A3F586734FF4C0625A6107F5AC73C5
:10F06000A3F5867328229A6107F5AC73A3F598730C
:10F07000184624231A46002116F09EF907F5AC73B2
:10F08000A3F598735C4A1A6007F5AC73A3F59873FF
:10F090004FF480625A6107F5AC73A3F598730822A8
:10F0A0009A6107F5AC73A3F5AA73184624231A4690
:10F0B000002116F081F907F5AC73A3F5AA734F4A46
:10F0C0001A6007F5AC73A3F5AA734FF480625A6116
:10F0D00007F5AC73A3F5AA7308229A6107F592733A
:10F0E0001A4600214648FEF755F90346002B02D187
:10F0F00044480CF067FD07F580731A46002142482A
:10F10000FEF748F90346002B02D140480CF05AFDA7
:10F1100007F1DC031A4600213D48FEF73BF90346A0
:10F12000002B02D13B480CF04DFD07F1B8031A4605
:10F1300000213948FEF72EF90346002B02D137484B
:10F140000CF040FD07F194031A4600213448FEF705
:10F1500021F90346002B02D132480CF033FD07F1B0
:10F1600070031A4600213048FEF714F90346002BBD
:10F1700002D12E480CF026FD07F14C031A4600215F
:10F180002B48FEF707F90346002B02D129480CF063
:10F1900019FD07F128031A4600212748FEF7FAF85F
:10F1A0000346002B02D125480CF00CFD3B1D1A46EE
:10F1B00000212348FEF7EEF80346002B02D1214838
:10F1C0000CF000FDFEF7B0F800BFFDE72CAC00200E
:10F1D000DCB4030801020208F4AD0020DC8503085A
:10F1E000E8850308F4850308008603080C860308F5
:10F1F00014860308208603082C8603083886030833
:10F200008502020844860308C503020858860308DD
:10F21000DD0302086C86030879060208808603086D
:10F220009106020898860308A9060208AC8603081E
:10F23000750D0208C0860308A50D0208D4860308D0
:10F24000E30D0208E886030880B594B000AF07F12B
:10F250001C0334220021184616F0AEF807F108030B
:10F2600000221A605A609A60DA601A61F7F73EFE6F
:10F270002D4B1B6C2C4A43F0805313642A4B1B6CA0
:10F2800003F080537B607B68284B1B68274A43F45C
:10F2900040431360254B1B6803F440433B603B68CD
:10F2A0000923FB614FF480333B6201233B6302235C
:10F2B0007B634FF48003BB631923FB634FF4C0737C
:10F2C0003B6402237B640823BB640223FB6407F1D5
:10F2D0001C031846F5F784FF0346002B01D000F00D
:10F2E000A9FFF7F713FE0346002B01D000F0A2FFA1
:10F2F0000F23BB600223FB6000233B614FF4A0534C
:10F300007B614FF48053BB6107F108030621184667
:10F31000F6F714FA0346002B01D000F08BFF00BF74
:10F320005037BD4680BD00BF00380240007000402D
:10F3300080B584B000AF3B4600221A605A609A60E4
:10F34000DA60214B214A1A601F4B4FF480325A6019
:10F350001D4B00229A601C4B00221A611A4B00229E
:10F360009A61194B002283F82020174B0022DA62A1
:10F37000154B174A9A62144B0022DA60124B012295
:10F38000DA61114B002283F830200F4B01225A61C1
:10F390000D48F7F763FF0346002B01D000F04AFF4A
:10F3A00006233B6001237B600023BB603B4619467C
:10F3B0000548F8F731F90346002B01D000F03AFF79
:10F3C00000BF1037BD4680BDBCAA00200020014010
:10F3D0000100000F80B584B000AF3B4600221A60E8
:10F3E0005A609A60DA60214B214A1A601F4B4FF431
:10F3F00080325A601D4B00229A601C4B00221A6119
:10F400001A4B00229A61194B002283F82020174BD7
:10F410000022DA62154B174A9A62144B0022DA6016
:10F42000124B0122DA61114B002283F830200F4B7E
:10F4300001225A610D48F7F711FF0346002B01D056
:10F4400000F0F8FE01233B6001237B600023BB60DA
:10F450003B4619460548F8F7DFF80346002B01D074
:10F4600000F0E8FE00BF1037BD4680BD04AB0020B1
:10F47000002101400100000F80B500AF0F4B104A82
:10F480001A600E4B00225A600C4B7F229A600B4B85
:10F49000FF22DA60094B00221A61084B00225A61F0
:10F4A000064B00229A610548F9F7B4F90346002B90
:10F4B00001D000F0BFFE00BF80BD00BF74AB0020D4
:10F4C0000028004080B58CB000AF07F10C03242267
:10F4D0000021184615F070FF3B4600221A605A6062
:10F4E0009A60214B4FF080421A601F4B00225A60F5
:10F4F0001D4B00229A601C4B4FF6FF72DA601A4BCC
:10F5000000221A61184B00229A610323FB6000233A
:10F510003B6101237B610023BB610523FB61002369
:10F520003B6201237B620023BB620523FB6207F180
:10F530000C0319460C48F1F74BFC0346002B01D095
:10F5400000F078FE00233B600023BB603B46194679
:10F550000548F2F7E7FE0346002B01D000F06AFEF3
:10F5600000BF3037BD4680BD94AB002080B58CB065
:10F5700000AF07F11C0300221A605A609A60DA603B
:10F580001A6107F10C0300221A605A609A60DA606F
:10F590003B4600221A605A609A60334B4FF080421B
:10F5A0001A60314B04225A602F4B00229A602E4B76
:10F5B0004AF6B332DA602C4B00221A612A4B002241
:10F5C0009A612948F1F7CEF90346002B01D000F0EB
:10F5D00031FE0423FB6150233B6200237B62002346
:10F5E000BB620023FB6207F11C0319461E48F2F7B9
:10F5F000C9F80346002B01D000F01CFE0023FB607D
:10F6000001233B6100237B610023BB6107F10C03F5
:10F61000002219461448F1F704FF0346002B01D0DD
:10F6200000F008FE0223FB6002233B6107F10C039C
:10F63000042219460C48F1F7F4FE0346002B01D0D2
:10F6400000F0F8FD00233B600023BB603B461946F9
:10F650000548F2F767FE0346002B01D000F0EAFDF3
:10F6600000BF3037BD4680BD94AB002080B58CB064
:10F6700000AF07F10C0324220021184615F09CFE70
:10F680003B4600221A605A609A60214B214A1A6058
:10F690001F4B00225A601E4B00229A601C4B4FF6F3
:10F6A000FF72DA601A4B00221A61194B00229A612C
:10F6B0000323FB6000233B6101237B610023BB61CB
:10F6C0000023FB6100233B6201237B620023BB62BA
:10F6D0000523FB6207F10C0319460D48F1F778FB8F
:10F6E0000346002B01D000F0A5FD00233B60002362
:10F6F000BB603B4619460648F2F714FE0346002B52
:10F7000001D000F097FD00BF3037BD4680BD00BF7F
:10F71000E0AB00200004004080B58CB000AF07F1E2
:10F720001C0300221A605A609A60DA601A6107F1BD
:10F730000C0300221A605A609A60DA603B4600228D
:10F740001A605A609A60334B334A1A60314B042274
:10F750005A60304B00229A602E4B4AF6B332DA6080
:10F760002C4B00221A612B4B00229A612948F1F799
:10F77000F9F80346002B01D000F05CFD0423FB6187
:10F7800050233B6200237B620023BB620023FB62A9
:10F7900007F11C0319461F48F1F7F4FF0346002B3D
:10F7A00001D000F047FD0023FB6001233B610023F3
:10F7B0007B610023BB6107F10C0300221946154849
:10F7C000F1F72FFE0346002B01D000F033FD02239A
:10F7D000FB6002233B6107F10C03042219460D482C
:10F7E000F1F71FFE0346002B01D000F023FD00239C
:10F7F0003B600023BB603B4619460648F2F792FD8A
:10F800000346002B01D000F015FD00BF3037BD4688
:10F8100080BD00BFE0AB00200004004080B58CB08C
:10F8200000AF07F10C0324220021184615F0C4FD97
:10F830003B4600221A605A609A60214B214A1A60A6
:10F840001F4B00225A601E4B00229A601C4B4FF641
:10F85000FF72DA601A4B00221A61194B00229A617A
:10F860000323FB6000233B6101237B610023BB6119
:10F870000023FB6100233B6201237B620023BB6208
:10F880000023FB6207F10C0319460D48F1F7A0FABB
:10F890000346002B01D000F0CDFC00233B60002389
:10F8A000BB603B4619460648F2F73CFD0346002B79
:10F8B00001D000F0BFFC00BF3037BD4680BD00BFA7
:10F8C0002CAC0020000C004080B58CB000AF07F1DC
:10F8D0001C0300221A605A609A60DA601A6107F10C
:10F8E0000C0300221A605A609A60DA603B460022DC
:10F8F0001A605A609A60334B334A1A60314B0422C3
:10F900005A60304B00229A602E4B4AF6B332DA60CE
:10F910002C4B00221A612B4B00229A612948F1F7E7
:10F9200021F80346002B01D000F084FC0423FB6186
:10F9300050233B6200237B620023BB620023FB62F7
:10F9400007F11C0319461F48F1F71CFF0346002B63
:10F9500001D000F06FFC0023FB6001233B6100231A
:10F960007B610023BB6107F10C0300221946154897
:10F97000F1F757FD0346002B01D000F05BFC02239A
:10F98000FB6002233B6107F10C03042219460D487A
:10F99000F1F747FD0346002B01D000F04BFC00239C
:10F9A0003B600023BB603B4619460648F2F7BAFCB1
:10F9B0000346002B01D000F03DFC00BF3037BD46B0
:10F9C00080BD00BF2CAC0020000C004080B58CB086
:10F9D00000AF07F10C0324220021184615F0ECFCBF
:10F9E0003B4600221A605A609A60234B234A1A60F1
:10F9F000214B00225A60204B00229A601E4B4FF68A
:10FA0000FF72DA601C4B00221A611B4B00225A6104
:10FA1000194B00229A610323FB6000233B61012301
:10FA20007B610023BB610523FB6100233B62012353
:10FA30007B620023BB620023FB6207F10C031946C3
:10FA40000D48F1F7C5F90346002B01D000F0F2FB99
:10FA500000233B6000237B600023BB603B461946CC
:10FA60000548F2F75FFC0346002B01D000F0E2FBF3
:10FA700000BF3037BD4680BD78AC00200004014097
:10FA800080B58CB000AF07F11C0300221A605A60E9
:10FA90009A60DA601A6107F10C0300221A605A605A
:10FAA0009A60DA603B4600221A605A609A60354BD1
:10FAB000354A1A60334B04225A60324B00229A6056
:10FAC000304B4AF6B332DA602E4B00221A612D4BCE
:10FAD00000225A612B4B00229A612A48F0F742FF1C
:10FAE0000346002B01D000F0A5FB0423FB6150234B
:10FAF0003B6200237B620023BB620023FB6207F1B1
:10FB00001C0319461F48F1F73DFE0346002B01D0A8
:10FB100000F090FB0023FB6001233B6100237B612D
:10FB20000023BB6107F10C03002219461548F1F7C9
:10FB300078FC0346002B01D000F07CFB0223FB6025
:10FB400002233B6107F10C03042219460D48F1F72B
:10FB500068FC0346002B01D000F06CFB00233B60E7
:10FB600000237B600023BB603B4619460548F2F743
:10FB7000D9FB0346002B01D000F05CFB00BF3037FF
:10FB8000BD4680BD78AC00200004014080B582B045
:10FB900000AF78600B46FB707B68002BC0F2A98039
:10FBA0007B68032B00F3A5807B68002B26D1FB78B4
:10FBB000012B11D13C215148F1F784FA4F48F1F75C
:10FBC000ADF9FFF75DFF00214C48F0F78BFF0421F2
:10FBD0004A48F0F787FF8DE000214848F1F786F8A2
:10FBE00004214648F1F782F84448F0F713FFFFF785
:10FBF000EDFE3C214148F1F7D7F97BE07B68012B12
:10FC000026D1FB78012B11D13C213D48F1F75AFA5E
:10FC10003B48F1F783F9FFF77FFD00213848F0F703
:10FC200061FF04213648F0F75DFF63E000213448AE
:10FC3000F1F75CF804213248F1F758F83048F0F752
:10FC4000E9FEFFF713FD3C212D48F1F7ADF951E036
:10FC50007B68022B26D1FB78012B11D13C2129484E
:10FC6000F1F730FA2748F1F759F9FFF77FFC002147
:10FC70002448F0F737FF04212248F0F733FF39E03A
:10FC800000212048F1F732F804211E48F1F72EF840
:10FC90001C48F0F7BFFEFFF715FC3C211948F1F7AF
:10FCA00083F927E0FB78012B11D13C211648F1F7AD
:10FCB00009FA1548F1F732F9FFF706FE002112485C
:10FCC000F0F710FF04211048F0F70CFF12E00021BC
:10FCD0000D48F1F70BF804210B48F1F707F80A4833
:10FCE000F0F798FEFFF79AFD3C210748F1F75CF921
:10FCF00000E000BF0837BD4680BD00BF78AC0020E3
:10FD0000E0AB002094AB00202CAC002080B588B084
:10FD100000AF3B1D00221A605A609A60DA601A61D7
:10FD20005A619A61194B1A4A1A60184B00225A609C
:10FD3000164B00229A60154B0022DA60134B00220A
:10FD40001A61124B00229A611048F0F7B9FC034681
:10FD5000002B01D000F06EFA60237B600023BB60B3
:10FD60000023FB6000237B613B1D002219460748EE
:10FD7000F1F7F4FB0346002B01D000F05BFA0348D7
:10FD800001F04CFC00BF2037BD4680BDC4AC002054
:10FD90000040014080B588B000AF3B1D00221A60D2
:10FDA0005A609A60DA601A615A619A611D4B1E4A64
:10FDB0001A601C4B00225A601A4B00229A60194BA1
:10FDC0000022DA60174B00221A61164B00229A615A
:10FDD0001448F0F7A5FB0346002B01D000F02AFAE7
:10FDE0001048F0F76DFC0346002B01D000F022FA1A
:10FDF00060237B600023BB600023FB6000237B61EA
:10FE00003B1D002219460748F1F7A8FB0346002BCB
:10FE100001D000F00FFA034801F000FC00BF2037CA
:10FE2000BD4680BD10AD00200048014080B588B0BF
:10FE300000AF3B1D00221A605A609A60DA601A61B6
:10FE40005A619A61194B1A4A1A60184B00225A607B
:10FE5000164B00229A60154B0022DA60134B0022E9
:10FE60001A61124B00229A611048F0F729FC0346F0
:10FE7000002B01D000F0DEF960237B600023BB6023
:10FE80000023FB6000237B613B1D002219460748CD
:10FE9000F1F764FB0346002B01D000F0CBF90348D7
:10FEA00001F0BCFB00BF2037BD4680BD5CAD00202B
:10FEB0000018004080B588B000AF3B1D00221A60DA
:10FEC0005A609A60DA601A615A619A611D4B1E4A43
:10FED0001A601C4B00225A601A4B00229A60194B80
:10FEE0000022DA60174B00221A61164B00229A6139
:10FEF0001448F0F715FB0346002B01D000F09AF9E7
:10FF00001048F0F7DDFB0346002B01D000F092F91A
:10FF100060237B600023BB600023FB6000237B61C8
:10FF20003B1D002219460748F1F718FB0346002B3A
:10FF300001D000F07FF9034801F070FB00BF2037CB
:10FF4000BD4680BDA8AD0020001C004080B590B02B
:10FF500000AF07F12C0300221A605A609A60DA6041
:10FF60001A619E4B1B6B9D4A43F0100313639B4B1E
:10FF70001B6B03F01003BB62BB6A984B1B6B974A69
:10FF800043F040031363954B1B6B03F040037B620C
:10FF90007B6A924B1B6B914A43F0020313638F4BB6
:10FFA0001B6B03F002033B623B6A8C4B1B6B8B4A5F
:10FFB00043F001031363894B1B6B03F00103FB61E7
:10FFC000FB69864B1B6B854A43F480731363834B39
:10FFD0001B6B03F48073BB61BB69804B1B6B7F4A57
:10FFE00043F4806313637D4B1B6B03F480637B617D
:10FFF0007B697A4B1B6B794A43F008031363774B99
:020000040802F0
:100000001B6B03F008033B613B69744B1B6B734A2A
:1000100043F004031363714B1B6B03F00403FB6099
:10002000FB686E4B1B6B6D4A43F0800313636B4B95
:100030001B6B03F08003BB60BB68684B1B6B674A9C
:1000400043F020031363654B1B6B03F020037B60BD
:100050007B68002242F218016148F6F72DFF00226A
:1000600044F240015F48F6F727FF00224FF4086191
:100070005D48F6F721FF0022C0215C48F6F71CFF1F
:1000800000224FF410715A48F6F716FF42F2180397
:10009000FB6201233B6300237B630023BB6307F107
:1000A0002C0319464E48F6F737FC49F24403FB622D
:1000B00000233B6300237B6307F12C031946484868
:1000C000F6F72AFC44F24003FB6201233B63002362
:1000D0007B630023BB6307F12C0319464148F6F705
:1000E0001BFC4FF40053FB6200233B6300237B6344
:1000F00007F12C0319463B48F6F70EFC4FF4086352
:10010000FB6201233B6300237B630023BB6307F196
:100110002C0319463448F6F7FFFB4CF24003FB6210
:1001200000233B6300237B6307F12C0319462E4811
:10013000F6F7F2FB4FF48073FB6200233B6300236E
:100140007B6307F12C0319462A48F6F7E5FBE02309
:10015000FB6200233B6300237B6307F12C031946FA
:100160002548F6F7D9FBC023FB6201233B6300233C
:100170007B630023BB6307F12C0319461B48F6F78A
:10018000CBFB2023FB6200233B6300237B6307F14F
:100190002C0319461948F6F7BFFB4FF49463FB6232
:1001A00000233B6300237B6307F12C0319461048AF
:1001B000F6F7B2FB4FF41073FB6201233B6300239D
:1001C0007B630023BB6307F12C0319460848F6F74D
:1001D000A3FB00BF4037BD4680BD00BF00380240D2
:1001E00000100240001802400004024000080240D3
:1001F000001402400020024000280240001C02407F
:1002000080B582B000AF78600120FDF769F9FBE7A7
:1002100080B582B000AF78607B681B68044A934267
:1002200001D1F6F7B3FF00BF0837BD4680BD00BF60
:100230000010004080B582B000AF72B600BF00224F
:1002400080210E48F6F738FE00237B6002E07B68D1
:1002500001337B607B680A4A9342F8DD01228021EA
:100260000648F6F729FE00233B6002E03B680133B5
:100270003B603B68024A9342F8DDE0E70008024039
:100280001FA1070080B588B000AF78604FF4967367
:10029000BB61FA237B614FF4FA733B619623FB60E9
:1002A0000023FB613D4B00221A603C4B1B68002B76
:1002B00012D000220021002002F03AFCF868FDF77D
:1002C0000FF901220121012002F032FCF868FDF74C
:1002D00007F90523FB61E8E7FB69002B0FD1304BE1
:1002E0001B68304A1168304A1268184602F020FC38
:1002F000B869FDF7F5F8FB690133FB61D5E7FB69E8
:10030000012B0BD101220121012002F011FC78699F
:10031000FDF7E6F8FB690133FB61C6E7FB69022BD9
:100320000FD1224B1B68224A1168224A12681846D4
:1003300002F0FEFBB869FDF7D3F8FB690133FB61FE
:10034000B3E7FB69032B0BD101220121012002F04D
:10035000EFFB7869FDF7C4F8FB690133FB61A4E7A3
:10036000FB69042B0FD1144B1B68144A1168144A03
:100370001268184602F0DCFBB869FDF7B1F8FB69BA
:100380000133FB6191E701220121012002F0D0FB42
:100390003869FDF7A5F80023FB6186E764AF00200C
:1003A0004C0100205001002058AF002054010020D3
:1003B000580100205CAF00205C010020600100209B
:1003C00060AF002080B582B000AF78600AF0E2FF35
:1003D0000A20FDF785F800BFF8E7000080B58CB073
:1003E00000AF78609D4B1B78002B53D19C4B1B7842
:1003F000002B4FD19B4B1B68002B04D1F6F7DAFE84
:100400000346984A1360F6F7D5FE0246954B1B68E3
:10041000D31AB3F5FA6F1DD3FEF746FC0346002B43
:1004200007D0914B1B68002B03D18D4B01221A7012
:1004300010E009F063FF0346002B08D109F098FC97
:100440000346002B03D1854B01221A7002E0854B35
:1004500000221A60854B1B68002B17D1012002F087
:100460000BFF834B01221A6000230122012101208E
:1004700002F082FB002301220121022002F07CFB1A
:10048000002301220121032002F076FB0120FDF769
:1004900027F8E1E0724B1B78002B4AD0724B1B68A7
:1004A000002B1DD0F6F786FE0246724B1B68D31A4E
:1004B000B3F5FA6F14D3F6F77DFE03466D4A136069
:1004C00009F01CFF0346002B0AD109F051FC03463A
:1004D000002B05D1624B00221A70604B01221A706A
:1004E0005F4B1B78002B1BD0604B1B68002B17D178
:1004F000012002F0C1FE5E4B01221A60002301229E
:100500000121012002F038FB0023012201210220F9
:1005100002F032FB002301220121032002F02CFB18
:100520000120FCF7DDFF97E007F10C03184609F006
:1005300031FF07F10C030021184609F0FDFC0346CA
:10054000002BF1D009F036FD7862484B1B68002B78
:1005500004D00AF0EDF90346002B7AD07B6A42F210
:100560001072934227D90AF0EFF90023FB6206E0EC
:100570000121F86A03F06AFFFB6A0133FB62FB6A40
:10058000032BF5DD012002F077FE394B01221A60C2
:10059000002301220121012002F0EEFA00230122B2
:1005A0000121022002F0E8FA0023012201210320A8
:1005B00002F0E2FA4DE07B6AC82B30D90AF0C4F9A8
:1005C00002F0A8FE38620023BB620CE03B6A012BFC
:1005D00014BF01230023DBB21946B86A03F036FFCB
:1005E000BB6A0133BB62BB6A032BEFDD012002F063
:1005F00043FE1F4B01221A6000230122012101202A
:1006000002F0BAFA002301220121022002F0B4FA1A
:10061000002301220121032002F0AEFA19E07B6AD7
:10062000002B16D002F042FE0346002B11D100230E
:1006300001220021012002F09FFA00230122002163
:10064000022002F099FA002301220021032002F087
:1006500093FA0120FCF744FFC4E600BF6DAE002012
:100660006EAE002070AE0020D4AE0020C8AE0020D8
:100670002001002074AE002080B582B000AF786009
:1006800002F014FE09F0C8FF0A20FCF729FFF7E783
:1006900080B582B000AF78600AF018F94FF47A7034
:1006A000FCF71EFF00BFF7E780B584B000AF7860AD
:1006B00009F0ADFA03461D4A1360FBF74DFD0346F2
:1006C000FB601A4B1B68002B17D102F0EFFD0346AD
:1006D000002B03D0164B1B68012B01D105F098F9B4
:1006E000134B1B68012B01D10AF03AF9F6F762FDB2
:1006F0000346184606F006FE11E002F0D7FD034659
:10070000002B03D00A4B1B68012B06D1F6F752FDD4
:100710000346184608F0E0FB01E008F0F1FD07F1A0
:100720000C030A211846FBF73FFBCAE7BCBF0020B9
:10073000C8AE00200000000080B582B000AF0023EA
:100740007B601DE0144A7B689B0013444FF000025D
:100750001A60124A7B68002142F82310104A7B6815
:10076000002142F823100F4A7B68002142F8231031
:100770009FED070B786802F007FC7B6801337B6014
:100780007B68032BDEDD00BF00BF0837BD4680BDA0
:1007900000000000000000002CAE00203CAE002055
:1007A0004CAE00205CAE002080B487B000AFF86093
:1007B00087ED000BFB68002B60DBFB68032B5DDC27
:1007C00097ED007BB7EE006BB4EEC67BF1EE10FA4E
:1007D00004D54FF00002364BC7E9002397ED007BAC
:1007E0009FED296BB4EEC67BF1EE10FA04DD26A373
:1007F000D3E90023C7E9002397ED007B9FED246B2D
:10080000B4EEC67BF1EE10FA02D82A4B7B612EE0E3
:1008100097ED007B9FED206BB4EEC67BF1EE10FAF6
:1008200003DB4FF07D537B6121E097ED007B9FED73
:100830001C6BB4EEC67BF1EE10FA02D81E4B7B6146
:1008400015E097ED007B9FED166B37EE466B9FED45
:10085000165B86EE057BF7EEC77B9FED187A67EE99
:10086000877A9FED177A77EE677AC7ED057A154A92
:10087000FB689B0013447A691A6000E000BF1C37D4
:10088000BD465DF8047B7047000000000088C3404F
:1008900000000000000058400000000000C092402E
:1008A0000000000000407F400000000000E08540A4
:1008B0000000F03FEC51783F1F856B3F7C142E3ECB
:1008C0001F856B3F1001002090B59FB000AFB24B69
:1008D0003B64B24BFB63B24BBB63B24B7B63B24B2B
:1008E0003B63F6F767FCF862BB6B1B68002B28D1F3
:1008F000BB6BFA6A1A6000237B670AE0AB4A7B6F26
:1009000052F82320A4497B6F41F823207B6F0133E9
:100910007B677B6F032BF1DD00233B670DE0386FB6
:1009200002F0B2FBB0EE407B9C4A3B6FDB0013440D
:1009300083ED007B3B6F01333B673B6F032BEEDDA9
:10094000FDE1BB6B1B68FA6AD31A07EE903AB8EE6A
:10095000677ADFED976AC7EE267AC7ED1B7AD7ED87
:100960001B7A9FED947AF4EEC77AF1EE10FA01D873
:10097000914BFB66914B3C1D0FCB84E80F0000238D
:10098000BB66D2E14FF000024FF00003C7E9182325
:10099000012387F85F30BB6E9B0078333B4453F8EC
:1009A000743C1B78012B54D1B86E02F06DFB87EDBF
:1009B000060BBB6EDB00FA6B134493ED007B97EDE7
:1009C000066B36EE477B87ED147B97ED147B9FED2E
:1009D000686BB4EEC67BF1EE10FA08DD97ED147B80
:1009E0009FED656B37EE467B87ED147B10E097ED4E
:1009F000147B9FED636BB4EEC67BF1EE10FA07D566
:100A000097ED147B9FED5C6B37EE067B87ED147BD7
:100A1000D7ED1B7AB7EEE77A97ED145B85EE076B9F
:100A20009FED555B86EE057B9FED576B27EE067BB2
:100A300087ED187B97ED187BB1EE477B87ED187B30
:100A4000BB6EDB00FA6BD118D7E90623C1E900239E
:100A50000CE1564ABB6E52F82330BB62B86E02F00E
:100A600071FB87ED120B97ED127BB7EE006BB4EEC6
:100A7000C67BF1EE10FA04D54FF00002504BC7E9E7
:100A80001223BB6E9B003A6C13441B68BA6AD31ADC
:100A90007B62BB6E9B003A6C1344BA6A1A6097ED96
:100AA000127B9FED3B6BB4EEC67BF1EE10FA00F2C9
:100AB000B280D7ED1B7A9FED3E7A67EE877AFCEE27
:100AC000E77A17EE903A7B647B6C002B01D10A2306
:100AD0007B643C4ABB6E52F823207B6A1A44394936
:100AE000BB6E41F82320384ABB6E52F823207B6C42
:100AF0001A443549BB6E41F82320334ABB6E52F885
:100B00002330312B40F283802F4ABB6E52F82330C2
:100B100007EE903AF8EE677A9FED267A67EE877ACD
:100B2000C7ED087A97ED127BB5EEC07BF1EE10FAB7
:100B30004CDDD7ED087AF5EEC07AF1EE10FA45DD1E
:100B4000204ABB6E52F8233007EE903AB8EEE75BCE
:100B500097ED127B85EE076BD7ED087AB7EEE75A73
:100B60009FED094B84EE057B26EE077B30E000BF4E
:100B70000000000000806640000000000080764019
:100B800000000000008066C00000000000004E4031
:100B90000000000000005840F8AD002008AE002022
:100BA00028AE00202CAE00206CAE0020DCAE002071
:100BB00000007A446F12833A0AD7233CFC8603086C
:100BC0000000F03F3CAE00205CAE00209FED5E7B5D
:100BD00087ED187B7B6A002B0BD1634ABB6E52F802
:100BE0002330002B05D14FF000024FF00003C7E97E
:100BF00018235D4ABB6E002142F823105B4ABB6E8E
:100C0000002142F82310012387F85F302EE00023F3
:100C100087F85F302AE097ED127BB5EEC07BF1EEEE
:100C200010FA13DD7B6A07EE903AB8EEE75B97EDBA
:100C3000127B85EE076BD7ED1B7AB7EEE75A9FED77
:100C4000444B84EE057B26EE077B01E09FED3E7B67
:100C500087ED187B7B6A002B05D14FF000024FF027
:100C60000003C7E91823012387F85F3097ED187B4D
:100C70009FED396BB4EEC67BF1EE10FA08DC97ED10
:100C8000187B9FED376BB4EEC67BF1EE10FA05D5FD
:100C90004FF000024FF00003C7E9182397F85F30C8
:100CA000002B32D0324ABB6E9B0013441B687B6121
:100CB0003B6B1B78002B0AD1BB6E9B007A6B1344F5
:100CC00097ED187BF7EEC77BC3ED007A1DE0BB6E96
:100CD0009B007A6B134493ED007AD7ED057A67EEAB
:100CE000276AB7EE007AD7ED057A37EE676A97ED97
:100CF000187BF7EEC77B66EE277ABB6E9B007A6B9C
:100D0000134476EEA77AC3ED007ABB6E9B007A6B34
:100D10001344D3ED007AB7EEE77AB0EE470BB86E26
:100D200002F032F9BB6E0133BB66BB6E032B7FF75B
:100D300029AE3B6B01221A70BB6BFA6A1A607C37D2
:100D4000BD4690BDAFF30080000000000000000031
:100D50000000000000004E40000000000040BF40C6
:100D6000000000000040BFC03CAE00205CAE002090
:100D70001001002080B584B000AF7860FBF7ECF97B
:100D80000346FB6000F00CFFFFF79EFD09F0F8FB47
:100D900002F086FF07F10C0305211846FBF704F863
:100DA00000BFEFE780B584B000AF786001F07CFC55
:100DB000FBF7D2F90346BB600023FB6005E0F8684F
:100DC00001F0B0FBFB680133FB60FB68032BF6DD31
:100DD00001F094FD07F108030A211846FAF7E4FF31
:100DE000EAE780B582B000AF786001F001FE4FF411
:100DF0007A70FCF775FB00BFF7E780B400AF00BF67
:100E0000FDE780B400AF00BFFDE780B400AF00BFD6
:100E1000FDE780B400AF00BFFDE780B400AF00BFC6
:100E2000FDE780B400AF00BFBD465DF8047B7047AE
:100E300080B500AF0248F0F7EDF900BF80BD00BFFC
:100E400078AE002080B500AF0248F1F74FFC00BF3C
:100E500080BD00BF0091002080B500AF0248F7F7C9
:100E6000A8FA00BF80BD00BF4CAB002080B582B0A7
:100E700000AF7860786809F0BDF900BF0837BD465B
:100E800080BD80B582B000AF7860786809F004FA60
:100E900000BF0837BD4680BD80B582B000AF114BA2
:100EA0001B6C104A43F0805313640E4B1B6C03F011
:100EB00080537B607B680B4B5B6C0A4A43F4804336
:100EC0005364084B5B6C03F480433B603B68002237
:100ED0000F216FF00100F6F721F900BF0837BD467A
:100EE00080BD00BF0038024080B58CB000AF786094
:100EF00007F11C0300221A605A609A60DA601A61D6
:100F00007B681B68364A93423CD1364B5B6C354A52
:100F100043F480735364334B5B6C03F48073BB61A5
:100F2000BB69304B1B6B2F4A43F0010313632D4BFE
:100F30001B6B03F001037B617B692A4B1B6B294A06
:100F400043F002031363274B1B6B03F002033B6167
:100F50003B69C023FB6103233B6200237B6207F1F3
:100F60001C0319462048F5F7D7FC0323FB61032334
:100F70003B6200237B6207F11C0319461B48F5F70F
:100F8000CBFC28E07B681B68194A934223D1154BA0
:100F90005B6C144A43F400735364124B5B6C03F4B0
:100FA0000073FB60FB680F4B1B6B0E4A43F00103A1
:100FB00013630C4B1B6B03F00103BB60BB687E2308
:100FC000FB6103233B6200237B6207F11C0319468C
:100FD0000548F5F7A1FC00BF3037BD4680BD00BF16
:100FE000002001400038024000000240000402409E
:100FF0000021014080B58AB000AF786007F114038A
:1010000000221A605A609A60DA601A617B681B6875
:10101000294A93424CD1294B1B6C284A43F0007358
:101020001364264B1B6C03F000733B613B69234B3D
:101030001B6B224A43F002031363204B1B6B03F02C
:101040000203FB60FB681D4B1B6B1C4A43F008034B
:1010500013631A4B1B6B03F00803BB60BB684FF4B0
:1010600080737B610223BB610023FB6103233B622E
:1010700009237B6207F1140319461148F5F74CFC6C
:1010800002237B610223BB610023FB6103233B62DC
:1010900009237B6207F1140319460A48F5F73CFC63
:1010A00000220C211420F6F739F81420F6F752F834
:1010B00000BF2837BD4680BD0064004000380240B4
:1010C00000040240000C024080B5A6B000AF78607A
:1010D00007F1080390220021184614F06DF97B688F
:1010E0001B680E4A934214D12023BB604FF4007357
:1010F000BB6307F108031846F4F722FD0346002BF3
:1011000001D0FFF797F8064B1B6F054A43F40043E5
:10111000136700BF9837BD4680BD00BF0028004060
:101120000038024080B592B000AF786007F1340318
:1011300000221A605A609A60DA601A617B681B6844
:10114000B3F1804F45D1784B1B6C774A43F00103D4
:101150001364754B1B6C03F001033B633B6B724BD9
:101160001B6B714A43F0020313636F4B1B6B03F05D
:101170000203FB62FB6A6C4B1B6B6B4A43F001037F
:101180001363694B1B6B03F00103BB62BB6A08234B
:101190007B630223BB630023FB6300233B640123C7
:1011A0007B6407F1340319466048F5F7B5FB4FF44B
:1011B00000437B630223BB630023FB6300233B6488
:1011C00001237B6407F1340319465948F5F7A4FB62
:1011D000A5E07B681B68574A934228D1524B1B6C91
:1011E000514A43F0020313644F4B1B6C03F002039C
:1011F0007B627B6A4C4B1B6B4B4A43F002031363CD
:10120000494B1B6B03F002033B623B6A30237B6359
:101210000223BB630023FB6300233B6402237B6444
:1012200007F1340319464148F5F776FB77E07B6810
:101230001B68414A934245D13B4B1B6C3A4A43F0F1
:1012400008031364384B1B6C03F00803FB61FB6954
:10125000354B1B6B344A43F001031363324B1B6B5A
:1012600003F00103BB61BB692F4B1B6B2E4A43F09C
:10127000800313632C4B1B6B03F080037B617B6942
:1012800001237B630223BB630023FB6300233B64D6
:1012900002237B6407F1340319462548F5F73CFB2C
:1012A0004FF400637B630223BB630023FB630023D3
:1012B0003B6402237B6407F1340319461F48F5F7AA
:1012C0002BFB2CE07B681B681D4A934227D1164BF1
:1012D0005B6C154A43F002035364134B5B6C03F0E1
:1012E00002033B613B69104B1B6B0F4A43F4807355
:1012F00013630D4B1B6B03F48073FB60FB6860236F
:101300007B630223BB630023FB6300233B64032353
:101310007B6407F1340319460A48F5F7FDFA00BF6C
:101320004837BD4680BD00BF00380240000402407F
:101330000000024000040040000C0040001C02407D
:10134000000401400020024080B485B000AF786006
:101350007B681B68134A93420CD1134B5B6C124A97
:1013600043F480335364104B5B6C03F48033FB60B5
:10137000FB6810E07B681B680C4A93420BD10A4B58
:101380001B6C094A43F040031364074B1B6C03F0CA
:101390004003BB60BB6800BF1437BD465DF8047BEB
:1013A000704700BF00400140003802400018004074
:1013B00080B485B000AF78607B681B68134A9342A5
:1013C0000CD1134B5B6C124A43F480235364104BD3
:1013D0005B6C03F48023FB60FB6810E07B681B6898
:1013E0000C4A93420BD10A4B1B6C094A43F0800311
:1013F0001364074B1B6C03F08003BB60BB6800BF2A
:101400001437BD465DF8047B704700BF00480140BB
:1014100000380240001C004080B592B000AF7860F8
:1014200007F1340300221A605A609A60DA601A6188
:101430007B681B68B3F1804F3DD1704B1B6C6F4ACA
:1014400043F0010313646D4B1B6C03F001033B631A
:101450003B6B6A4B1B6B694A43F002031363674B98
:101460001B6B03F00203FB62FB6A644B1B6B634A5A
:1014700043F001031363614B1B6B03F00103BB6279
:10148000BB6A08237B630223BB630023FB63002347
:101490003B6401237B6407F1340319465848F5F790
:1014A0003BFA4FF400437B6307F134031946554878
:1014B000F5F732FA9DE07B681B68534A934228D1C6
:1014C0004E4B1B6C4D4A43F0020313644B4B1B6C99
:1014D00003F002037B627B6A484B1B6B474A43F075
:1014E00002031363454B1B6B03F002033B623B6A31
:1014F00030237B630223BB630023FB6300233B6435
:1015000002237B6407F1340319463D48F5F704FADA
:101510006FE07B681B683D4A93423DD1374B1B6CA3
:10152000364A43F008031364344B1B6C03F0080382
:10153000FB61FB69314B1B6B304A43F001031363C2
:101540002E4B1B6B03F00103BB61BB692B4B1B6B69
:101550002A4A43F080031363284B1B6B03F080037C
:101560007B617B6901237B630223BB630023FB63F5
:1015700000233B6402237B6407F1340319462148AE
:10158000F5F7CAF94FF400637B6307F1340319469A
:101590001F48F5F7C1F92CE07B681B681D4A934290
:1015A00027D1164B5B6C154A43F002035364134B6F
:1015B0005B6C03F002033B613B69104B1B6B0F4AF2
:1015C00043F4807313630D4B1B6B03F48073FB6058
:1015D000FB6860237B630223BB630023FB63002360
:1015E0003B6403237B6407F1340319460A48F5F78B
:1015F00093F900BF4837BD4680BD00BF00380240A8
:10160000000402400000024000040040000C0040C2
:10161000001C0240000401400020024080B58CB054
:1016200000AF786007F11C0300221A605A609A60CC
:10163000DA601A617B681B68454A93421CD1454BAE
:101640001B6B444A43F010031363424B1B6B03F0C4
:101650001003BB61BB692023FB6102233B620023B3
:101660007B620023BB620323FB6207F11C03194664
:101670003948F5F751F966E07B681B68374A9342B1
:101680001DD1344B1B6B334A43F002031363314BC0
:101690001B6B03F002037B617B694FF40073FB61FA
:1016A00002233B6200237B620023BB620323FB62B5
:1016B00007F11C0319462A48F5F72EF943E07B6829
:1016C0001B68284A93421CD1224B1B6B214A43F0D2
:1016D000800313631F4B1B6B03F080033B613B696B
:1016E0004023FB6102233B6200237B620023BB6239
:1016F0000923FB6207F11C0319461B48F5F70CF997
:1017000021E07B681B68194A93421CD1114B1B6B6B
:10171000104A43F0200313630E4B1B6B03F02003AE
:10172000FB60FB684FF48073FB6102233B62002384
:101730007B620023BB620923FB6207F11C0319468D
:101740000B48F5F7E9F800BF3037BD4680BD00BF54
:1017500000400140003802400010024000480140B3
:101760000004024000180040001C0240001C004021
:101770000014024080B582B000AF78607B681B68BF
:10178000B3F1804F0FD1244B1B6C234A23F001038C
:10179000136408212148F5F76BFA4FF40041204803
:1017A000F5F766FA33E07B681B681E4A93420AD15C
:1017B000194B1B6C184A23F002031364302117489D
:1017C000F5F756FA23E07B681B68174A93420FD15E
:1017D000114B1B6C104A23F00803136401211048BD
:1017E000F5F746FA4FF400611048F5F741FA0EE0BC
:1017F0007B681B680E4A934209D1074B5B6C064A13
:1018000023F00203536460210A48F5F731FA00BF60
:101810000837BD4680BD00BF0038024000040240CA
:101820000000024000040040000C0040001C024088
:10183000000401400020024080B58EB000AF786007
:101840000023FB620023BB62334B1B6C324A43F024
:1018500010031364304B1B6C03F01003FB60FB6838
:1018600007F1100207F1140311461846F4F736F990
:101870003B6AFB62FB6A002B03D1F4F71BF9786328
:1018800004E0F4F717F903465B007B637B6B234AA4
:10189000A2FB03239B0C013BBB62214B214A1A6034
:1018A0001F4B40F2E732DA601D4ABB6A53601C4BA3
:1018B00000221A611A4B00229A60194B00229A6189
:1018C0001748EEF72DFE034687F8333097F833308C
:1018D000002B1BD11248EEF77BFE034687F833300E
:1018E00097F83330002B11D13620F5F733FC7B68A5
:1018F0000F2B08D8002279683620F5F70FFC0A4A2A
:101900007B68136002E0012387F8333097F83330A7
:1019100018463837BD4680BD0038024083DE1B4381
:1019200078AE0020001000400400002080B586B092
:1019300000AF7860144A154BD31A7B617B693B6119
:10194000134B1B68002B02D1114B124A1A60104B2B
:101950001A687B6813443A699A4207D213F0FEFD75
:1019600003460C221A604FF0FF3309E0084B1B6856
:10197000FB60074B1A687B681344054A1360FB68D9
:1019800018461837BD4680BD00000820000400003E
:10199000C4AE0020903F012080B400AF0123184660
:1019A000BD465DF8047B704780B582B000AF7860BB
:1019B000396013F0D3FD034616221A604FF0FF334F
